:020000040000FA
:0400000A9900C0DEBB
:10000000004000200B010000C1000000C90D0000ED
:1000100000000000000000000000000000000000E0
:10002000000000000000000000000000C50000000B
:100030000000000000000000C7000000C900000030
:10004000CB000000CD000000CF000000D100000078
:10005000D3000000D5000000D7000000D900000048
:10006000DB0000008D0D0000DF000000E10000005B
:10007000E3000000E5000000E7000000E9000000E8
:10008000EB000000ED000000EF000000F1000000B8
:10009000F3000000F5000000F7000000F900000088
:1000A000FB000000FD000000FF0000000101000057
:1000B0000301000005010000070100000901000024
:1000C000FEE7FEE7FEE7FEE7FEE7FEE7FEE7FEE708
:1000D000FEE7FEE7FEE7FEE7FEE7FEE7FEE7FEE7F8
:1000E000FEE7FEE7FEE7FEE7FEE7FEE7FEE7FEE7E8
:1000F000FEE7FEE7FEE7FEE7FEE7FEE7FEE7FEE7D8
:10010000FEE7FEE7FEE7FEE7FEE70348854600F070
:1001100001F803E0704700000040002035493648F0
:100120000A1A02D0072291438D46344934480A1AEC
:1001300006D00722914381F30988022282F31488B2
:1001400030483149314A00F043F831483149324AA8
:1001500000F03EF831483249324A00F039F832486E
:100160003249334A00F034F832483349334A00F018
:100170002FF833483349344A00F02AF833483449D9
:10018000344A00F025F834483449002200F02BF8B6
:1001900033483449002200F026F833483349091A1D
:1001A000082903DB00220260043001601F48204957
:1001B000884205D00268043003B4904703BCF7E7D7
:1001C00000208646EC4600200021294A9047FEE7A1
:1001D000884207D0521A05D0037801300B700131E4
:1001E000013AF9D17047884202D002700130FAE733
:1001F0007047000000400020003C0020004000202C
:1002000000400020C82A0100000000200200002059
:1002100074020000740200003A0F0000C82A0100B6
:1002200000000020000000203C0F00003C0F0000F8
:100230003C0F00003C0F00003C0F00003C0F000092
:100240003C0F00003C0F0000C82A0100CC2A01002E
:10025000440100204401002004000020440100204B
:1002600044010020440100204801002048050020EE
:04027000F50900008C
:1002740082B002006B4607331A706B4607331B7853
:100284001A001F231A40044B012191400A001A60EE
:10029400C04602B07047C04600E100E0BFF34F8F94
:1002A400C046044B044ADA60BFF34F8FC046C046D1
:1002B400C046FCE700ED00E00400FA058023DA05FF
:1002C40080235B000021D1508023DB0501221A60CA
:1002D400C0468023DA0580235B00D358002BF8D076
:1002E4008023DA0580235B000021D150A023DB05A5
:1002F4000C49E02212025A50A023DA05A123DB00A4
:100304000949D150A023DA05A323DB00E021090227
:10031400D150A023DA05A323DB000349D150C04602
:100324007047C0460C050000F01F000010B5134ACA
:10033400A223DB000921D150104AA123DB000021B4
:10034400D1500E4A0E4B0021D1500C4AA823DB0099
:100354000C49D1500949C1239B0080225202CA5042
:10036400064A80239B000121D1500920FFF780FF1A
:10037400024B01221A60C04610BDC04600900040E6
:1003840004050000FFFF000084B001900091A02349
:10039400DB051A49E02212025A50A023DA05A123F0
:1003A400DB001749D1501749019A13009B009B1891
:1003B400009A9B18DB005B5803931249019A1300BF
:1003C4009B009B18009A9B18DB00CB1804331B6816
:1003D4000293039B0D33A022D20501219940A1234E
:1003E400DB00D150029B1A1DA023DB0501219140A3
:1003F4000A0002495A50C04604B070470C05000078
:10040400F01F0000E429010082B002006B460733AC
:100414001A70A023DB052A49E02212025A50A023B5
:10042400DA05A123DB002749D1506B4607331B783B
:10043400032B15D01CDC012B02D0022B08D017E0B3
:10044400A023DA05A123DB0080218901D15025E016
:10045400A023DA05A123DB008021C901D1501DE0CE
:10046400A023DA05A123DB0080210902D15015E085
:10047400A023DA05A123DB0080218901D150A02328
:10048400DA05A123DB008021C901D150A023DA05BC
:10049400A123DB0080210902D150C046A023DB0543
:1004A400074A10219950A023DB05054A20219950C1
:1004B400A023DB05024A40219950C04602B0704790
:1004C4000C050000F01F0000A023DB05114A0121E8
:1004D4009950A023DB050F498022D2055A500E4AB9
:1004E400A123DB000021D1500B4A0C4B1E21D1501B
:1004F40009490B4ACD23DB048B50074AB123DB00A7
:100504006021D150044AA023DB000521D150C0460C
:100514007047C0461C050000003000400C05000078
:100524002405000086B00190002305930023049362
:10053400002303933F4B0122DA613E4A84235B008C
:100544000021D1503B4B01221A60C046394A842312
:100554005B00D358002BF9D0364A84235B0000217A
:10056400D150344AA323DB00D3580393314B0122E7
:100574001A62059B01330593039B012B3ADDC046A8
:100584002C4A84235B00D358002BF9D0294A8423B6
:100594005B000021D150274AA323DB00D358DAB2F1
:1005A400019B1A70234B01221A62224B01225A61C9
:1005B400C046204A84235B00D358002BF9D01D4A3F
:1005C40084235B000021D1501A4AA323DB00D258B4
:1005D400019B0133D2B21A70C046164A82235B00D3
:1005E400D358002BF9D0134A82235B000021D15049
:1005F40001231CE00F4B01225A61C0460D4A84239B
:100604005B00D358002BF9D00A4A84235B000021F5
:10061400D150084AA323DB00D3580393019B002243
:100624001A70019B013300221A7001235B421800E7
:1006340006B07047003000401B4B02221A701A4B60
:1006440000225A70184B01229A70174B0122DA705B
:10065400154B02221A71144B01225A71124B0322B8
:100664009A71114B0122DA710F4B00221A720E4B50
:1006740002225A720C4B02229A720B4B0222DA7239
:10068400094B04221A73084B02225A73064B0222A6
:100694009A73054B0322DA73034B02221A74024B3A
:1006A40004225A74C046704770000020244B042270
:1006B4001A70234B00225A70214B03229A70204B4C
:1006C4000022DA701E4B02221A711D4B00225A714D
:1006D4001B4B01229A711A4B0022DA71184B00222B
:1006E4001A72174B01225A72154B02229A72144B3A
:1006F4000122DA72124B00221A73114B02225A732E
:100704000F4B02229A730E4B0222DA730C4B012216
:100714001A740B4B03225A74094B02229A74084B25
:100724000322DA74064B03221A75054B03225A7509
:10073400034B04229A75024B0322DA75C0467047B4
:1007440058000020154B04221A70144B00225A70D2
:10075400124B03229A70114B0122DA700F4B0322C1
:100764001A710E4B02225A710C4B03229A710B4BD5
:100774000322DA71094B04221A72084B04225A72BA
:10078400064B01229A72054B0122DA72034B0122B5
:100794001A73024B03225A73C04670474800002064
:1007A400154B03221A70144B00225A70124B042268
:1007B4009A70114B0122DA700F4B04221A710E4BFE
:1007C40002225A710C4B04229A710B4B0322DA71E8
:1007D400094B03221A72084B04225A72064B012257
:1007E4009A72054B0122DA72034B01221A73024BEF
:1007F40003225A73C046704738000020544B00222D
:100804001A70534B00225A70514B00229A70504B6D
:100814000122DA704E4B00221A714D4B02225A719A
:100824004B4B00229A714A4B0322DA71484B002247
:100834001A72474B04225A72454B01229A72444B56
:100844000422DA72424B02221A73414B04225A7375
:100854003F4B03229A733E4B0422DA733C4B04222F
:100864001A743B4B04225A74394B04229A74384B41
:100874000322DA74364B04221A75354B02225A7558
:10088400334B04229A75324B0122DA75304B042221
:100894001A762F4B00225A762D4B03229A762C4B34
:1008A4000022DA762A4B02221A77294B00225A7741
:1008B400274B01229A77264B0022DA77244B2022F9
:1008C40001219954224B212201219954204B2222A7
:1008D400012199541E4B2322022199541C4B24229A
:1008E400012199541A4B252203219954184B26228D
:1008F40002219954164B272203219954144B282280
:1009040003219954124B292203219954104B2A2272
:10091400032199540E4B2B22022199540C4B2C2267
:10092400032199540A4B2D2201219954084B2E225C
:1009340002219954064B2F2201219954044B302251
:1009440002219954024B312202219954C046704726
:100954000400002000B583B001900A006B46033305
:100964001A70204B1A88204B1B889A4222D11F4BA5
:100974001B785B00019AD3181B7818001B4B1B785B
:100984005B00019AD3185B781900FFF7FDFC174B45
:100994001B780133DAB2154B1A70144B1A786B4674
:1009A40003331B781900100000F090FA0B00DAB240
:1009B4000E4B1A700B4B1B8801339AB2094B1A80E9
:1009C400084B1B881A00084B1B88013319001000C0
:1009D40000F091FA0B009AB2024B1A80C04603B0A1
:1009E40000BDC046840000200000002082000020DA
:1009F40000B599B000231793002314930023139395
:100A04000023129300231193CC4B0193FFF756FC60
:100A140000210120FFF7B8FCFFF7F0FEFFF7C0FE4E
:100A2400FFF790FEFFF708FEFFF740FEFFF74CFDCF
:100A3400FFF77CFCA023DA05A323DB008021490314
:100A4400D150A023DA05A123DB0080214903D15032
:100A5400A023DB05BA49802292025A50B94B0122E5
:100A64001A6060231093B84B00221A60B74B00221F
:100A74001A60002316930023159300210020FFF72A
:100A840083FCA023DB05B24A00219950AF4B052219
:100A94001A60C04642E1AF4B0122DA60A023DA05B6
:100AA400A223DB00D25880239B02134020D1A74B02
:100AB4001B68052B03D0A54B1B68062B18D1C04619
:100AC400A023DA05A223DB00D25880239B02134023
:100AD400F6D09C4B01221A60602310939A4B00229B
:100AE4001A609A4B00221A60002316930023159370
:100AF400964B1B68062B00D910E19A00964BD3182D
:100B04001B689F46019B013B0193002B05DD934B22
:100B14000C211800FFF71EFF00E18C4B06221A601F
:100B2400864B0193FAE0019B013B0193002B05DD09
:100B34008B4B09211800FFF70DFFEFE0834B0522D3
:100B44001A607E4B0193E9E000231B061A0001237F
:100B54001B041900FF231B040B401A431A231B0216
:100B64001B041B0C13438E2213430F930F9B283B30
:100B74001793764B01221A6040231693CEE0794BEB
:100B840001229A6016E0784A159BD3181B78754A9F
:100B940019006B4BD150C046724A8E235B00D35868
:100BA400002BF9D06F4A8E235B000021D150159B96
:100BB40001331593159A169B9A42E4D3694B01228B
:100BC4005A61624B02221A60A8E004210420FFF754
:100BD400DBFB664B1800FFF7A5FC031E00DC9DE061
:100BE400624B1B781A00614B5B781B021B041B0CC5
:100BF4001A435F4B1A605E4B1B685E4A934200D0F7
:100C04008CE0524B03221A6088E00120FFF7FCFBC2
:100C1400564B1800FFF786FC031E00DC7EE0534BA6
:100C24001B781A00514B5B781B021B041B0C1A43E4
:100C34004F4B1A604E4B1B68002B28D1002100201B
:100C4400FFF7A2FB494B1800FFF76CFC474B1B78DE
:100C54001A00464B5B781B021B041B0C1A43444BC3
:100C64001A60434B1B68012B0ED1A023DB054249BC
:100C7400802252035A50374B01225A603F4B0721BE
:100C84001800FFF767FEF9E7304B05221A60384B6E
:100C94001B681A00169B9B1816932C4B04221A608F
:100CA4003CE0374B19211800FFF754FE354B002266
:100CB4001A60159A169B9A4226D02A4B01229A60F2
:100CC4001BE0294A159BD3181B78264A19001C4B94
:100CD400D150C046234A8E235B00D358002BF9D051
:100CE400204A8E235B000021D150159B01331593BC
:100CF400244B1B685A1C234B1A60159A169B9A4264
:100D0400DFD3184B01225A611E4B1B681A00179B34
:100D14009B1A17930D4B03221A60C046094B1B689C
:100D2400012B00D1B7E603210320FFF72DFBA023FD
:100D3400DB051149802252035A50FEE7A0860100C8
:100D44001C050000F0000020FC000020F80000203A
:100D54004407000000900040AC2A01005800002025
:100D640070000020003000403C0F00008C00002088
:100D7400F400002011FF00000C05000038000020E2
:100D8400040000208800002000B583B0FA239B00F3
:100D940001930B4AA0235B00D358012B0CD1084AC2
:100DA400A0235B000021D150FFF778FA044AA02366
:100DB4005B00D3580093009BC04603B000BDC046FF
:100DC4000090004004207146084202D1EFF30880ED
:100DD40001E0EFF30980014A10470000E50D00002F
:100DE40082B001902F4B1B882F4B1A682F4B1A622D
:100DF4002F4B1B78D9B22D4B242299542D4B1B78A1
:100E0400DBB21A00294B9A622B4B1A68274BDA6221
:100E14002A4B1B889AB2254B1A86224B1B889BB2FD
:100E24001A00224B5A63264B1B889BB21A001F4B95
:100E34009A63244B1B889BB21A001C4BDA63224B27
:100E440000221A60C046204B1B68002BFBD0019B7C
:100E54001A68164B1A60019B5A68144B5A60019B1E
:100E64009A68124B9A60019BDA68104BDA60019B16
:100E74001A690E4B1A61019B5A690C4B5A61019B0A
:100E84009A690A4B9A61019BDA69084BDA610E4B45
:100E940000221A60C0460C4B1B68002BFBD002B02A
:100EA4007047C0462CED00E024ED00E00401002072
:100EB40028ED00E029ED00E038ED00E02AED00E047
:100EC40030ED00E03CED00E0000100200A0010D00D
:100ED4000300400800E052008242FCD9002000E0F8
:100EE4005208934200D39B1A40418A42F8D1190018
:100EF400704700207047CA1751408B1A19D0C11788
:100F040006B44840411A48081A0000E052008242E0
:100F1400FCD9002000E05208914200D3891A4041D4
:100F24009A42F8D10CBC53405840C01A5140891A17
:060F340070470020704729
:100F3C0055555555555555554D43555048434D45AB
:100F4C00424C32428E1A010041E006C3BCEC7F4792
:100F5C00A6809473BC9D7273691500000A00020090
:100F6C000000000000000000000000000000000075
:100F7C00E8190100000000008602040000001018AF
:100F8C00001418001818001C1800201800781A00FB
:100F9C00241800781A002818002C18003018003477
:100FAC001800381800781A003C1800401800441833
:100FBC00004818004C18005018005418005818001D
:100FCC005C18006018006418006818006C18007039
:100FDC001800741800781800781A007C1800801813
:100FEC00008418008818008C1800901800941800C1
:100FFC009818009C1800781A00781A00781A00A02B
:10100C001800A41800720200AC1800781A00B0186E
:10101C00007C0200781A00B81800BC1800C0180038
:10102C00C41800C81800CC1800D01800D41800D868
:10103C001800DC1800781A00E01800781A00E41880
:10104C0000E81800EC1800F01800F41800F818006C
:10105C00FC1800001900041900081900781A000C7B
:10106C0019001019001419001819001C1900201966
:10107C00002419002819002C1900781A00301900C6
:10108C00341900381900781A003C19004019004432
:10109C0019004819004C190050190054190058191E
:1010AC00005C19006019006419006819006C1900C3
:1010BC007019007419007819007C190080190084CB
:1010CC0019008819008C19009019009419009819AE
:1010DC00009C1900A01900A41900A81900AC190053
:1010EC00B01900B41900B81900BC1900C01900C41B
:1010FC001900C81900CC1900D01900D41900D8193E
:10110C0000DC1900E01900E41900E81900EC1900E2
:10111C00F01900F41900F81900781A00781A007800
:10112C001A00781A00781A00781A00781A00781ABF
:10113C0000781A00781A00781A00781A00781A00C9
:10114C00FC1900001A00041A00781A00781A0078AA
:10115C001A00781A00081A000C1A00781A00101AD3
:10116C0000141A00781A00781A00781A00781A00FD
:10117C00781A00781A00181A001C1A00781A0078CD
:10118C001A00781A00781A00781A00781A00201AB7
:10119C0000241A00281A002C1A00301A00341A00E5
:1011AC00381A003C1A00401A00441A00481A004C25
:1011BC001A00501A00541A00581A00781A00781A9B
:1011CC0000781A00781A00781A00781A005C1A0055
:1011DC00601A00641A00681A006C1A00701A007405
:1011EC001A00FFFFFFFFFFFFFFFFFFFFFFFFFFFFE7
:1011FC00FFFFFFFFFFFFFFFFFFFFFFFFFFFFFFFFF3
:10120C00FFFFFFFFFFFFFFFFFFFFFFFFFFFFFFFFE2
:10121C00FFFFFFFFFFFFFFFFFFFFFFFFFFFFFFFFD2
:10122C00FFFFFFFFFFFFFFFFFFFFFFFFFFFFFFFFC2
:10123C00FFFFFFFFFFFFFFFFFFFFFFFFFFFFFFFFB2
:10124C00FFFFFFFFFFFFFFFFFFFFFFFFFFFFFFFFA2
:10125C00FFFFFFFFFFFFFFFFFFFFFFFFFFFFFFFF92
:10126C00FFFFFFFFFFFFFFFFFFFFFFFFFFFFFFFF82
:10127C00FFFFFFFFFFFFFFFF00180000BF0204BFCE
:10128C000214BF0224BF0228BF022CBF023CBF02C3
:10129C0040BF0244BF0248BF0200C0020000000C65
:1012AC00180000BF0204BF0218BF0224BF0228BFEF
:1012BC00022CBF023CBF0240BF0244BF0248BF0227
:1012CC000000000018000018000C180014BF0218D1
:1012DC00BF0200BF02060000FFFF00FFFFFF18BFA8
:1012EC0002120000050000FFFFFF461D00FFFFFF7C
:1012FC00FF7F00FFFFFF28BF02060000828000FF77
:10130C00FFFF3CBF02060000010000FFFFFF44BFCF
:10131C000203000077770014BF02060000FF7FFF76
:10132C00FFFFFF5010AFA81804000000A00304003A
:10133C0000005030AFB41804000000B814040000D2
:10134C00006F17210EFF260E018800000000002000
:10135C000000E00200320001202002881400070780
:10136C0001070000E003003AA03E2101002002002A
:10137C0037000020010020810F700100320F0007A0
:10138C000000200000E00200320000020000003CDF
:10139C000D020000000040DA0000FEA00120000059
:1013AC00E0020032002020900188000006A1028893
:1013BC008004780000EB1F0037E2844454A0B499F9
:1013CC0005BAE2844454A0B49906BAE2844454A009
:1013DC00B40006EB476FDEFD07B2AE0188636CE12B
:1013EC0003003A0AD8010000EB0E0037606CE108EC
:1013FC00003A004DEB0A05E80200393420EC0AF003
:10140C00A08B05E9F9FF3E0400376168E101003269
:10141C000086EB0B000719C7BA1905BA0E04E003D6
:10142C00003A0A00E0DBFF3A000006FE07B2AE020B
:10143C00888A0478F5FF370CD0A3E20F4D1C0039D5
:10144C00890278354DBA0A05E80200393420EC0AD5
:10145C00F0A08B05E90F0032254DBA0A05E8020011
:10146C00393420EC0AF0A08B05E90800320C00E0BE
:10147C0006003215CDBA0A05E80200393420EC0A10
:10148C00F0A08B05E98984E854A0B40B00E0E2FFDE
:10149C003A0000069902BA055D788B05E9F7FF3230
:1014AC00C82ADE055D788B05E9F3FF320C00E0F10C
:1014BC00FF3219DDBAEEFF37B015040000005416E8
:1014CC0004000000B814040000009A160400000088
:1014DC00A01604000000741104000000E0140400C5
:1014EC000000F40F04000000809FBE829FBE841F8A
:1014FC00780800FA04A8A90011800018A33E003255
:10150C00A311800001784202B2010220810F5138F0
:10151C00003AB189800110A0B18988218980A41278
:10152C0021948F50040039B189800140A0B1898881
:10153C000B0037318980835878318988628980140F
:10154C000241848F500100393289881200204112E7
:10155C0021910841D13424C1BF9F510525D1BF9F92
:10156C00813424E1BF9F5120B0F1BF9FE28A806794
:10157C000161834078688257E4417983CF500C0035
:10158C003A8200E8E18A88E88F500F003AB18980EE
:10159C000170A0B1898841122121838881132131E6
:1015AC0083880700370001EBE28A880FF99782CF16
:1015BC005002003A110020E18A88E50060E48F5067
:1015CC0032003A0058A30C003AC08980F08A88484F
:1015DC0000DE020032F00F20F08A88F48A80841139
:1015EC0088508A8000F0A0508A882400370000E0E0
:1015FC00220035F08A800000E00C003AC08980F0AF
:10160C008A884800DE020032F00F20F08A88F08AC7
:10161C0080801188508A8000F0A0508A881300378F
:10162C00E08980B080FB811188E08988018A80E2A2
:10163C001321128140820F50010039E18988110079
:10164C0020801321108810508A800000A0508A88B6
:10165C00F08A800000E9F08A88808B80010021905C
:10166C00806001003A10C0A00080FA4F02784F0150
:10167C00BE4F00BE00400600000541E00006C3005E
:10168C00BCEC007F4700A68000947300BC9D0072E8
:10169C0073000100003E7E00007C00FCFF00600037
:1016AC0000CF05B0889FBE8A9FBE8C9FBE8E1F78D0
:1016BC000005782083800000E002003A000D786974
:1016CC000237028021030020D28F9FE38F9F0204F8
:1016DC00BE8005EB2183801107781A01788001EB1D
:1016EC00E80F51E08F5954023E02060108003733CF
:1016FC000037BF0037E500371A0137770137A701EC
:10170C0037D00137EB0137F00220800F574E0236ED
:10171C00020320E0FB2F0F0040721002000000E0DB
:10172C00FB2F0F00400006EB30417821C4B3814FF2
:10173C005111003A90409021C3B2C3C4B390C16917
:10174C0083C070A0419002C16982C07008003A3118
:10175C0083801101780000EB7610020000001D0060
:10176C00200D0D780500370C06E8C10220810F56BC
:10177C00E7FF3A8006EB0C01782183800000EB76C2
:10178C001002000000130020DE01378001EB800600
:10179C00EBF00220800F57D90136020320E0FB2F1B
:1017AC000F0040761002000000030320E2FB2F0F15
:1017BC0001416000B8961202000000400D98510DD6
:1017CC00981FA097AFA0978002B10180B1200D980F
:1017DC00310D981C00204C1598E0FB2F0F0040E8B1
:1017EC000040020120C04A280E1602000000000032
:1017FC00E0060032A0FE2F401598800020000D78E6
:10180C008C0178B50137E406453FA897CFA8975FC0
:10181C00A997EFA997809EBE8296BE2401208000D6
:10182C00EB0801BEC0FA2F0F0040C01102000000EF
:10183C000000200000E0040032D02C21EF989780AB
:10184C008F50040032E0FD2F0F00407481571400BC
:10185C00372A0290BA02904A0390DA03906F90975D
:10186C00FF90970F99979F99970020E101A8E102AB
:10187C00B0E103B8E1EFFF3190FE2F4015987000F6
:10188C0020000D788C0178830678880137FFA897A3
:10189C00D08070F1AF9F820F50FBFF3A0100E0E95E
:1018AC00003A4065210000E00D00322A0990BA0987
:1018BC00900204B00380B00D0278318380208380C5
:1018CC005416020000000000E002003C50FE2FFF06
:1018DC0000379B8B800B00E01200320082200284C8
:1018EC00200001518000EB8016020000005030EF08
:1018FC005230EF0000EB908B883016020000002075
:10190C0083808A13020000003083808A1302000057
:10191C00000000EB3015986011B8620D98730D98AB
:10192C000080EB10159880002010059820002000F6
:10193C000D783083801000E007003A31F12FC18F11
:10194C009F22002081F92F8F804008120200000096
:10195C000B00E00100320060FE1A00906810B470B9
:10196C003EB1EA08900100404083886002200A00E2
:10197C0040060B020000000006781300208006EBE6
:10198C000C00E035013A10F12FC08F9F220020810E
:10199C00F92F8F80403083800812020000002083D2
:1019AC00801007782C1598400020000D782A08909C
:1019BC00BA0890430220830F50E08F5806003E4037
:1019CC000220301598600020100598130020290083
:1019DC00376A0990FA0990E00F51E08F5906003AE6
:1019EC008000203015983000201005981300201E20
:1019FC000037F03D206830B4200120301598800F5E
:101A0C00570100363E1598BA1090000320808F5075
:101A1C000100363015983A13906132B8820F528318
:101A2C008F5A0300396A0890301598050037620008
:101A3C00200500090283D80100533015985000206E
:101A4C001005981300200100378001EB2A6090E804
:101A5C004F400B003A2A10902A0A90BA0A90610360
:101A6C00B8840F53858F5B0100360400788006EB39
:101A7C008E0F50E5003A8207200200E02100323040
:101A8C008380B00090908050E58F501C00362183ED
:101A9C0080B10090810F510100360101782A12901B
:101AAC00848050828F500300313A1190840F511072
:101ABC000036F3CF5001003A8100E94809DEF34FBC
:101ACC005101003A0110B1048240241598C18F9F36
:101ADC0022002081F92F8F80400812020000001391
:101AEC0000203A11908006EB820F57BD00392A1066
:101AFC00900200502015982A0E90BA0E90218380E7
:101B0C00E0FB2F0F0040761002000000000656E0AC
:101B1C00865E2C0D983D0D98BA1190E2FB2F0F01AB
:101B2C00414A0890DA0890961202000000400D9885
:101B3C00510D981A0090000D78E30F50A0003A7CDC
:101B4C0000453A1190E1FB2F8F8040741502000084
:101B5C0000FA58903A609000C070960032B0FE2F98
:101B6C002400370B00E00100320060FE0003EB6044
:101B7C0022B8BA1190E2FB2F0F01410A10909A1073
:101B8C0090BE09020000000006BEE4F92F0F0242CD
:101B9C00BA1190E2FB2F0F01410A10909A1090E6B7
:101BAC000B020000000C15981D1598BA10906A09CC
:101BBC0090FA0990010151E08159620D98730D98CA
:101BCC00310020010D780000E007003D80FE2F4021
:101BDC001598700020000D781300208306786C0097
:101BEC00370000E068003270FE2F4015981300207B
:101BFC00830678650037F03D206830B44A0990DAE6
:101C0C000990C0F12D411422800F51818F591E0073
:101C1C003AD02C21E09F9F2A0090BA00904A019064
:101C2C00DA0190E0979FF1979F829F9F939F9F5F10
:101C3C00A897EFA8977FA9978FB197A09F9FB19F67
:101C4C009FC29F9FD39F9F0003EBD5EA2D0002EB11
:101C5C00230120C2FA2F0F01410800BEBE09020069
:101C6C000000DE150200000002003760FE2F401558
:101C7C00986430EF6830EF800020000D784A1090A7
:101C8C00CF80DEC000DD000020D08F9FE18F9F420F
:101C9C000020A1F92F8F80403083800812020000B1
:101CAC0000A28280B3828030838050120200000038
:101CBC00A00F205183800008B840140200000013CC
:101CCC0000208306781F00378001EB8006EB0E00A6
:101CDC00E01B00322A0990BA09906172B8820F5247
:101CEC00838F5A0500390207780000EB761002004A
:101CFC0000006430EF0E01782183800000EB761039
:101D0C00020000002A0890BA08900E0050E080589B
:101D1C00200D98310D981300208006EB020037132C
:101D2C000020830678F3B79F6814020000000002BD
:101D3C00BEFFB1970300E0020032000D98110D9820
:101D4C000A09909A099002015283815A6A0090FA0A
:101D5C000090800F51818F59210036C0FE2F401505
:101D6C00981A80E9E30F5018003E000020C1FE2FA6
:101D7C00D08F9FE18F9F420020A1F92F8F804030A0
:101D8C008380F4B79F85BF9F081202000000A282D7
:101D9C0080B382803083805012020000000081EBFF
:101DAC002183800000EB7610020000008FBA977F31
:101DBC00B297040D98150D98000DEB6430EF20834D
:101DCC00800000E00300328B8676ADFD3A090037C7
:101DDC000B00E00600326A0190FA019030838050CB
:101DEC0012020000000000FE000DEB00F0A7000046
:101DFC00EA0000E94F00DE0100370000EB4F0778E6
:101E0C004F06BE4F05BE4F04BECF05B10000060005
:101E1C0000FE6022B80300E0A00032C80BDE9E007A
:101E2C003A573E20871F785400F8889FBE8A9FBE81
:101E3C008C9FBE0178A306003A04D8A3020032D1CD
:101E4C0048AF0160A204C0A70160A03B00242D0094
:101E5C002004F0A02C8D200C00E006003204F0A130
:101E6C000B0024E8CF400200324D00201B0024065A
:101E7C0000FA0D06D08C87478E03788B1B78809BDD
:101E8C00BE0F04788004EBDCEA2D0C28E110003244
:101E9C00C22ADD0300328502E9058009B61F7800ED
:101EAC00C8FE852120860120D1E8AFFEFF37020055
:101EBC0037951FBAB59FBA0683E9FCFF3188845762
:101ECC006810F86830EF5500378F05780D06E90C6F
:101EDC008009809FEB0300E9008009B25D780381E3
:101EEC00558001EB8D00D00F00A78000EB0D00D1C9
:101EFC00020009B25B7880DBEB0000E9FBFF3A8162
:101F0C0087570D06E90C8009C70F483A0031C70501
:101F1C00784705788D004560864D640354890378B5
:101F2C00640343E883530700393608E136E0E1FAED
:101F3C00FF343650E136D8E1F8FF312A0037000083
:101F4C0020A10F2062034704F0A73600BEA102882F
:101F5C008D00D18E0378068D20D1E8AFFEFF3702BD
:101F6C000009371B783708BB3798BB8100E9FCFFA9
:101F7C003A6A3221FEB0977FB8970100B88A0350B5
:101F8C000A00201A00A00000EB1A00A7FEFF37047D
:101F9C00A0A70060FE8A1602000000070B78B109AA
:101FAC00B0010B78D1E8A800000000000004B8A331
:101FBC00D1E8AFFEFF3AAC1602000000E203470086
:101FCC0000EB979B46971B480D00D1008046808103
:101FDC0051B2FF31808141A5FF3A00FF23D028B6D2
:101FEC008027EB1E0090AE00900080FA4F06BE4F8B
:101FFC0005BE4F04BE5400F98027EB6830EF00009B
:10200C0006EE8747889FBE8A9FBE8C9FBE8E1F7828
:10201C000006780D80204E83806830EF0020200170
:10202C000020B0B79FC1B79F7A80575015020000AF
:10203C0000D0B79FE1B79FF2B79F83BF9F89002065
:10204C000004EB2E0037CFEA97E9CF42050036109B
:10205C000020960C020000000000EB4B00377FB50F
:10206C00978FBD970D00E97FB3978600600500320E
:10207C008000EB0A00708B8070610540E085486140
:10208C0068B85FB197EFB197000041818049D0B734
:10209C009FE1B79F8A0F508B8F58100039802120F9
:1020AC00010020BFB297808F523000317A80575098
:1020BC001502000000D0B79FE1B79FF2B79F83BF16
:1020CC009F800F55818F5D0100360804E90804E8F4
:1020DC001C0078800F54CFFF39000EE85FB097EFEB
:1020EC00B0970615020000000000E016003A5FB23F
:1020FC0097EFB2974200200300200023200100201C
:10210C00D812020000000000E00C003AE07B200036
:10211C0007474E83885FB097EFB097181402000002
:10212C00000000EB960C02000000100020050037A8
:10213C008904E9DEFF3A1000200100370000EB4F64
:10214C0007784F06BE4F05BE4F04BEEF00B100002E
:10215C00061600FA889FBE8A9FBE8C1F7882047870
:10216C0003057804047802F02B23002082B79F9398
:10217C00B79F0FB1979FB19792BF9FA3BF9F0800C6
:10218C00E001003A7C84570006EB8005EB8802786E
:10219C000B02788A0178090178DA0D020000000040
:1021AC0000E03600321802BE8200200300204023DB
:1021BC0020010020D812020000000000E01E003AAE
:1021CC001802BE1FB897AFB897E00F50E08F580FAA
:1021DC0000320400BE1FB997AFB997820F52838F9C
:1021EC005A0900390B00E01C003A2841909B002052
:1021FC000204E00100354B0020A80490DAFF37827E
:10220C000120030020802120010020D812020000B0
:10221C00000000E00F00321C0020E30F550D0036CB
:10222C002801900205556305550A854424002005B4
:10223C000020380042A8804AE30441C5FF37CCFF98
:10224C002F0100370086EB0C00784F06784F05BE47
:10225C004F04BE0080FA0000060A00FA889FBE8A6E
:10226C009FBE8C9FBE3007984F07986003200100DB
:10227C00209216020000000002BE8005788080E8E3
:10228C000100A18187474E05908000EBC2232003FB
:10229C0000200A0078C01102000000330037004013
:1022AC00EB5047980A0078B04078214798B04078B6
:1022BC00314798104078404798630045104F784A52
:1022CC0040901047982A4090E84F40040032140088
:1022DC00200004E005003D0100378400203E009002
:1022EC000000E01600321E0678E606451E0490AE8D
:1022FC0004908002EB8C01780D01780800BEDA0D99
:10230C00020000000000E00A0032F03D204083880B
:10231C000003EBD5EA2D0002EB8C01780D01780857
:10232C0000BEF60E020000001E0078808555E68582
:10233C0055660040000545E68F55CBFF3E6830EFF3
:10234C00CE07904F06BE4F05BE4F04BE0080FA006C
:10235C000006889FBE8A9FBE8C1F787231EF683052
:10236C00EF6430EF5C30EF5030EF5230EF8F0007FE
:10237C00600E210008EBC08280D18280908788A1FA
:10238C008788A08280B18280450ADDCB02DE85027F
:10239C00724502DD6033B86000B86011B8040250B9
:1023AC00858258060359878359015B21001121D678
:1023BC0001077503070004BE0A02200B82200C845F
:1023CC00200B06560060FE6E0307C28280D382800B
:1023DC004C1ADD4411DE020172C419DE0802508968
:1023EC008258820F52838F5A040036080441898424
:1023FC00491000207E0407C1728001006504003280
:10240C008000EBF082801108980E0037CD02070097
:10241C0000E00B0032F00F204004070C0178800024
:10242C00EB0B00785B040750B0EF52B0EF6030EF6D
:10243C006270EF1004070140FED8FF376022B888A5
:10244C009FBE8A9FBE5400F80500E04220AF8F0269
:10245C0078E482420178A306003A04D8A302003241
:10246C00D148AF0160A204C0A70160A0A10288807E
:10247C0000EBD1E8AFFEFF370300370080E84200E5
:10248C00AF5420EC8301E9290039821A78D100205D
:10249C00F6FF2FF70F203243788301E9050039B29C
:1024AC0048788301E9030039B243780200370430DD
:1024BC00A00420A01004BA9084BA889ABE869ABE52
:1024CC00E30F620B00320683EA87C3EA08056389CF
:1024DC0085630400A70A03BE08057389857304107D
:1024EC00A70A03BE6044B808035389835BEC0F62F0
:1024FC000300328003EB0430A7F60FB2EA82528756
:10250C000073D2FF32A602808622788022780100E6
:10251C00785400F94F05BE4F04BE000006889FBEDC
:10252C00B5EFA910002050200A860F00920120B0B0
:10253C00220A880F0050002064200A8A0F00120023
:10254C002020220A8A0F00A10920320020800720B7
:10255C0053F820804978814978824978227C80021E
:10256C0000A071052060042043F82080497881493F
:10257C0078824978840FABFEFF3A010220227C80DE
:10258C00028060FDFF3208A025292620C88288D948
:10259C008288C88288D9828800C429A08288563053
:1025AC00EF800220508388E202073E6EEF3A6EEF16
:1025BC00270EA8272EA81D0EA91D2EA90001EB5031
:1025CC00220A880D00D8220A880D002126840200D8
:1025DC0078460007401221F082880800BE4F04BEE6
:1025EC000000060000FE6022B80178A306003A0441
:1025FC00D8A3020032D148AF0160A204C0A7016089
:10260C00A0809FBE829FBE5400F8A102880300E008
:10261C002C0032670020E39F53268D200600E00437
:10262C000032F7BF9F0010A704F0A00010A100001B
:10263C00A1D1E8AFFEFF37FFBB978080EB90C0BA0B
:10264C00901FBACF9F600080E86638E105003A9091
:10265C00C0BACF9F609000BACF9F600080E80000A6
:10266C00E04220AF5420EC04F0A7E3835304F0A124
:10267C00CF8FEA04003A070141878151070036E702
:10268C00FF3700D9EB8301E90300328703E9FBFF35
:10269C003AE1FF378F87E95400F94F01BE4F00BE76
:1026AC00BE0904000000889FBE8A1F78000578814F
:1026BC00047818C0B3F00720808F5401003C00440C
:1026CC00EB6104644A44DD0860A008C0A00000204F
:1026DC00C12120010070808B880008EBA82FA80076
:1026EC0000EBF08A88A82FA90002EBA36921000156
:1026FC0020010020000178C11421801321941502BF
:10270C00000000046A218001EB80072001002000FA
:10271C000178E106214012219415020000005002BC
:10272C0020408A88A08988401721308A88004E2151
:10273C00908988808B800808782022EF2822EF2946
:10274C0011886A118804A8A910002074200A520864
:10275C0000B21602000000808B8010F0A04F0578AC
:10276C004F04BE00000660B0BF3A0032CFB897CD20
:10277C0008DE37003A4460AF35003A6210AC3300E3
:10278C003A3600F83200F83400F80000F8849FBEA6
:10279C00869FBE658380A68B80378B80950213370E
:1027AC0083189783184260EF040621840178148201
:1027BC00101B00326200423028E130B0E130B8E149
:1027CC00F8FF33849FBE869FBEB08210308318B052
:1027DC0083184220AF940978548A42540A4B548A85
:1027EC004B260521070020869FBEB01F78B01F78AE
:1027FC000040064260EF4F03BE4F02BE100A9880A5
:10280C0000EBE2FF374F03BE4F02BE0000F934006D
:10281C00F93200F93600F96210A94F01BECF0078E9
:10282C000040068002EB0F00A78082EBE081404263
:10283C0020AF000005851F78801FE8030090020080
:10284C00E14200AF020078230290B303904303905F
:10285C00070343CF00E91A00328403530038E142E6
:10286C0000AFE003500300328702E9058009B45839
:10287C00780620E14200AF430290870350030032F8
:10288C008702E9058009B458788080504F00E00237
:10289C000032930910A40198E303900700E0422052
:1028AC00AE0700010000060002420620E14200AF24
:1028BC00070252000178F1FF37C800DE2600321201
:1028CC0002804811DD4460AF0270A0CF1F7162001E
:1028DC00B84001B0C308AE1A003702F12B2100201A
:1028EC00810171160032801F7800F12B64160200F2
:1028FC000000809FEA00F02B2100206416020000EB
:10290C0000000178CF01E94F00788000EB02F0A6BF
:10291C000230A7060037F4FF218481610480200374
:10292C0021B8020040838048641602000000809F9A
:10293C00BE000006801FEB811F78801F78861F78F1
:10294C00851F78841F78C8150200000068140200E7
:10295C0000008003EB4F8253CF825B4F835BCF0130
:10296C00781400320706219719780B00338419402C
:10297C008599488619498499BE861978CF1978CFDC
:10298C001978000028801978F48B510000068419FE
:10299C00508599588619590200098019EBF4FF37B4
:1029AC00E48757000006889FBE8A1F780004BE0289
:1029BC000578080037080078201602000000000097
:1029CC00E0030032080890D610020000001800E066
:1029DC000F0032681402000000390150A98158BA66
:1029EC000F51AA8F59EFFF36070037681402000009
:1029FC0000390150A98158BA0F51AA8F5904003ED1
:102A0C002002ABF7FF3A1000200100370000EB4F1B
:102A1C0005784F04BE0000060400E021003280025D
:102A2C00786208B83600200500094688D8000141B4
:102A3C000380B00000EBA70280A30288D1E8AFFEB0
:102A4C00FF370100E00C00320402E90200A7060087
:102A5C0037D25ABA0402E90C0039020037B25ABA1A
:102A6C00925ABAC2DABA0281E854A0B4630252F99B
:102A7C00FF31620242020033048009B25ABAA70243
:102A8C0088000006E00140020078200032C3039069
:102A9C003303901302909302530683438403530031
:102AAC0028E14200AE0500788002780538E142004A
:102ABC00AE8702788503E9020039078009315A781C
:102ACC000620E14200AF430290050350030032861A
:102ADC0003E9078009315A78930940940198D3038C
:102AEC00908080500700E04220AE070001000006F5
:102AFC000000E04220AF100005881F78829FBE00C6
:102B0C000478681402000000809FBEF80390070050
:102B1C00E0070032080078E480576881570700010D
:102B2C00E887574F04780000061000201800E0FAE0
:102B3C00FF326814020000007FB997EFB9970200CA
:102B4C00508380585FB997CFB9970200E10388E1B1
:102B5C00F2FF340000EBEDFF370080EA8180EA855C
:102B6C00002006322887DB2E100037B25A78B2527A
:102B7C00780400688400208100D10080D3020039E1
:102B8C000600688780688100D10080D30200390676
:102B9C0000688780680402E9F4FF3AE28151EEFF95
:102BAC003BE28141040032124068440020030020C3
:102BBC00ECFF370080EA8180EA0000060400FA8806
:102BCC001F788A9FBE0003BEB0BF9FC1BF9F020487
:102BDC00780405BE0000EBE00F53E08F5B0B003A6E
:102BEC000F00376A8057501502000000800F558186
:102BFC008F5D030039820F55838F5D0500396404A6
:102C0C00540800E0F4FF3A0000EB010037100020FC
:102C1C004F05BE4F04780080FA0000060000FED17C
:102C2C00E8AFFEFF378046884783806830EF013B72
:102C3C00B8613221B709B08100538A160200000036
:102C4C00B146888000EBB74688D1E8A800000000A8
:102C5C0000000200A6AC16020000008003EB020884
:102C6C00A3D1E8AFFEFF3AD1C8A90200A7AC160267
:102C7C00000000000006A080210100206A0150E045
:102C8C0081580A00326416020000004800DEC808B1
:102C9C00DD010070D22C210000514220AE00000555
:102CAC00100005C0FF2B2100200160A0641602005B
:102CBC0000004C01DEC409DD0301710080EAF4FF61
:102CCC0020040060F0FF371100200F00A701002046
:102CDC000282200700371100200F00A701002000FE
:102CEC0000E04220AF0000050280208009904818C7
:102CFC00DE4220AE000005431ADE0400A1040141AF
:102D0C00EF81611218A50080D2E080401298AD00CE
:102D1C0000060001EB6022B80100E0110032B11F87
:102D2C00E90E0033F3FF20310378CC33DE03036369
:102D3C0002034300A8A51638A50428AD4200AA42F8
:102D4C0020AE1638AD8502E8CF1FE9F3FF3B8F8725
:102D5C00E90400780000065C10000200008000000E
:102D6C005010000400008000005C11000200008084
:102D7C0000007211000200008000006410000200CC
:102D8C000080000066100002000080000068100047
:102D9C000200008000000000000000FED1E8AFFE41
:102DAC00FF37A20280A102880308BBA202889046CA
:102DBC0088A14688200424D0C8A8D0C8AE1084B2FC
:102DCC000001EB513E201A1302000000D1E8AFFEC7
:102DDC00FF37D1C8A9000006889FBE8A9FBE000499
:102DEC00BE6814020000000005BE8001EB0300E089
:102DFC004220AE0140FE6814020000000A02508B13
:102E0C00825804015485815CF6FF314F05BE4F0496
:102E1C00BE0000066783800003EB651621A08B8043
:102E2C00150278170010B4001B34011B94011B64AD
:102E3C0002521520E1F7FF3A0480204400B01490B0
:102E4C00A6000006804B21741602000000ECFF3730
:102E5C000000EBA08B88001621308B88E09C206052
:102E6C0083880006210000E00200326030EF6270BF
:102E7C00EFBC29EFBE29EFD2A9EF20002074200A65
:102E8C005408002528A8BDE9A8000006811F7882F7
:102E9C009FBE8001EB318B806881683119E83199D4
:102EAC0049118949640151328B880180204100B05D
:102EBC001190A141FF200100E04220AE0104014F1E
:102ECC0001BECF0078004006881F780004781801F6
:102EDC00788800780000EB7610020000001808904B
:102EEC000040A1100C981808900050A1100C9818D4
:102EFC0008900060A1100C981000204F047800007E
:102F0C0006A20280A10288F37F208380EA00806001
:102F1C000082EBD1E8AFFEFF3710C2BAB000BA01A5
:102F2C0002628480EA04003A8381E9F9FF31A2024B
:102F3C0088100005A20288000005831F78821F7884
:102F4C00801F78681402000000CF83E86210AC1672
:102F5C000280370278A70278CF1B40CF9B48E01342
:102F6C00490610A76210A9470052D7805A000006E4
:102F7C00300278A00278A7028064184260884AA5C3
:102F8C0002880483E8E0824AD1E8AFFEFF371400E0
:102F9C00BA9480BAA502881601BA9681BAA702889B
:102FAC000000060000000202E905003981017003EF
:102FBC0000A603003704800931587800000682010E
:102FCC00D18301E90300390380093118780200A785
:102FDC003158780000068002EB05087832009841E1
:102FEC00009811009821009853009864009875007F
:102FFC00988080EB010898010028110898000006C1
:10300C006410E2080032600E2187F707A28280B3B9
:10301C0082808301D10281D3001121B4FF0700000B
:10302C00EB000006010621010037820078110178BF
:10303C000200E0040032800F51FAFF3A9008781039
:10304C000005000005D1E8AFFEFF37D1C8A9D2A812
:10305C00EFD4A8EFA1028054A0EFE2FF2F0209BB2E
:10306C00A10288000006AFFE070000E00600320255
:10307C0001FC2017210088EB0C1802000000000056
:10308C00FE000006B04178B1C15103003A0201E9DB
:10309C00FBFF310000050080EB4200AF1000050083
:1030AC0000060182200F00A7018020000990C311A7
:1030BC00DE67016161C0790200DE6100600000061C
:1030CC00C006210000E00400320082204000B01055
:1030DC0090A44200AE000005100005801F7800008F
:1030EC00EBA616020000004F0060A61602000000BE
:1030FC000080EA000006E582801600200500E00250
:10310C000032050001000378060078000006A202D8
:10311C0080A10288D1E8AFFEFF379080BA1000BAC8
:10312C00A20288000006110280C808DD4460AF01CD
:10313C0070A0CF9F700004010201E90200390280E7
:10314C0009015878000006000820CF1F701002807B
:10315C000040066300B88100D10080D3000006A1B6
:10316C0014211120A00000066113211130A00000D1
:10317C0006C14B28BC13040000004800DDCF1F70B3
:10318C0000400624A8A8000006FFFFFFFFFFFFFF7A
:10319C00FFFFFFFFFFFFFFFFFFFFFFFFFFFFFFFF33
:1031AC00FFFFFFFFFFFFFFFFFFFFFFFFFFFFFFFF23
:1031BC00FFFFFFFFFFFFFFFFFFFFFFFFFFFFFFFF13
:1031CC00FFFFFFFFFFFFFFFFFFFFFFFFFFFFFFFF03
:1031DC00FFFFFFFFFFFFFFFFFFFFFFFFFFFFFFFFF3
:1031EC00FFFFFFFFFFFFFFFFFFFFFFFFFFFFFFFFE3
:1031FC00FFFFFFFFFFFFFFFFFFFFFFFFFFFFFFFFD3
:10320C00FFFFFFFFFFFFFFFFFFFFFFFFFFFFFFFFC2
:10321C00FFFFFFFFFFFFFFFFFFFFFFFFFFFFFFFFB2
:10322C00FFFFFFFFFFFFFFFFFFFFFFFFFFFFFFFFA2
:10323C00FFFFFFFFFFFFFFFFFFFFFFFFFFFFFFFF92
:10324C00FFFFFFFFFFFFFFFFFFFFFFFFFFFFFFFF82
:10325C00FFFFFFFFFFFFFFFFFFFFFFFFFFFFFFFF72
:10326C00FFFFFFFFFFFFFFFFFFFFFFFFFFFFFFFF62
:10327C00FFFFFFFFFFFFFFFFFFFFFFFFFFFFFFFF52
:10328C00FFFFFFFFFFFFFFFFFFFFFFFFFFFFFFFF42
:10329C00FFFFFFFFFFFFFFFFFFFFFFFFFFFFFFFF32
:1032AC00FFFFFFFFFFFFFFFFFFFFFFFFFFFFFFFF22
:1032BC00FFFFFFFFFFFFFFFFFFFFFFFFFFFFFFFF12
:1032CC00FFFFFFFFFFFFFFFFFFFFFFFFFFFFFFFF02
:1032DC00FFFFFFFFFFFFFFFFFFFFFFFFFFFFFFFFF2
:1032EC00FFFFFFFFFFFFFFFFFFFFFFFFFFFFFFFFE2
:1032FC00FFFFFFFFFFFFFFFFFFFFFFFFFFFFFFFFD2
:10330C00FFFFFFFFFFFFFFFFFFFFFFFFFFFFFFFFC1
:10331C00FFFFFFFFFFFFFFFFFFFFFFFFFFFFFFFFB1
:10332C00FFFFFFFFFFFFFFFFFFFFFFFFFFFFFFFFA1
:10333C00FFFFFFFFFFFFFFFFFFFFFFFFFFFFFFFF91
:10334C00FFFFFFFFFFFFFFFFFFFFFFFFFFFFFFFF81
:10335C00FFFFFFFFFFFFFFFFFFFFFFFFFFFFFFFF71
:10336C00FFFFFFFFFFFFFFFFFFFFFFFFFFFFFFFF61
:10337C00FFFFFFFFFFFFFFFFFFFFFFFFFFFFFFFF51
:10338C00FFFFFFFFFFFFFFFFCD120E1E040000002A
:10339C00B62B04000000BC2B04000000CE2B040054
:1033AC000000C22B04000000C82B04000000CE2B30
:1033BC0004000000CE2B04000000CE2B0400000003
:1033CC00DE2504000000542704000000C225040080
:1033DC000000CE2B04000000CE2B040000005E2564
:1033EC0004000000CE2B04000000CE2B04000000D3
:1033FC00A42004000000442204000000CE2B040092
:10340C000000CE2B04000000CE2B04000000CE2BBD
:10341C0004000000CE2B040000002C25040000004A
:10342C00CA2804000000CE2B04000000CE2B0400A0
:10343C000000CE2B04000000762504000000CE2BEB
:10344C0004000000CE2B0400000038210400000012
:10345C008E2204000000CE2B04000000CE2B0400B2
:10346C000000CE2B04000000222504000000CE2B0F
:10347C0004000000081F04000000CE2B0400000014
:10348C00CE2B04000000B81404000000CE2B040066
:10349C000000CE2B04000000CE2B04000000CE2B2D
:1034AC0004000000CE2B04000000CE2B0400000012
:1034BC00CE2B04000000CE2B04000000CE2B040009
:1034CC000000CE2B04000000CE2B04000000CE2BFD
:1034DC0004000000BE2104000000D82204000000FB
:1034EC00CE2B04000000CE2B04000000CE2B0400D9
:1034FC000000CE2B04000000CE2B04000000CE2BCD
:10350C0004000000CE2B04000000CE2B04000000B1
:10351C00CE2B04000000CE2B04000000CE2B0400A8
:10352C000000CE2B04000000CE2B04000000CE2B9C
:10353C0004000000CE2B04000000402A0400000010
:10354C00CE2B04000000CE2B04000000CE2B040078
:10355C000000CE2B04000000CE2B04000000CE2B6C
:10356C0004000000CE2B04000000CE2B0400000051
:10357C00CE2B04000000CE2B04000000CE2B040048
:10358C000000CE2B04000000CE2B040000001A25F6
:10359C0004000000CE2B04000000222304000000D5
:1035AC00CE2B04000000CE2B04000000CE2B040018
:1035BC000000CE2B040000004C2304000000CE2B96
:1035CC0004000000CE2B0400000076230400000051
:1035DC00A02304000000CA2304000000F42304000C
:1035EC0000001E2404000000482404000000722483
:1035FC00040000009C2404000000C6240400000009
:10360C00F02404000000CE2B04000000CE2B04009C
:10361C000000CE2B04000000CE2B04000000CE2BAB
:10362C0004000000CE2B04000000CE2B0400000090
:10363C00CE2B04000000CE2B04000000CE2B040087
:10364C000000CE2B04000000CE2B04000000CE2B7B
:10365C0004000000CE2B04000000CE2B0400000060
:10366C00CE2B04000000CE2B04000000CE2B040057
:10367C000000CE2B04000000CE2B04000000CE2B4B
:10368C0004000000CE2B04000000CE2B0400000030
:10369C00CE2B04000000CE2B04000000CE2B040027
:1036AC000000CE2B04000000CE2B04000000CE2B1B
:1036BC0004000000CE2B04000000CE2B0400000000
:1036CC00CE2B04000000CE2B04000000CE2B0400F7
:1036DC000000CE2B04000000CE2B04000000CE2BEB
:1036EC0004000000CE2B04000000CE2B04000000D0
:1036FC00CE2B04000000CE2B04000000CE2B0400C7
:10370C000000CE2B04000000CE2B04000000CE2BBA
:10371C0004000000CE2B04000000CE2B040000009F
:10372C00CE2B04000000CE2B04000000CE2B040096
:10373C000000FFFF00FFFF00FF0000FFFF00FF0085
:10374C0000FFFF00FF0000FFFF00FF0000FFFF0075
:10375C00FF0000FFFF00FF0000FFFF00FF0000FF65
:10376C00FF00FF0000FFFF00FF0000FFFF00FF0055
:10377C0000FFFF00FF0000FFFF00FF0000FFFF0045
:10378C00FF0000FFFF00FF0000FFFF00FF0000FF35
:10379C00FF00FF0000FFFF00FF0000FFFF00FF0025
:1037AC0000FFFF00FF0000FFFF00FF0000FFFF0015
:1037BC00FF0000FFFF00FF0000FFFF00FF0000FF05
:1037CC00FF00FF0000FFFF00FF0000FFFF00FF00F5
:1037DC0000FFFF00FF0000FFFF00FF0000FFFF00E5
:1037EC00FF0000FFFF00FF0000FFFF00FF0000FFD5
:1037FC00FF00FF0000FFFF00FF0000FFFF00FF00C5
:10380C0000FFFF00FF0000FFFF00FF0000FFFF00B4
:10381C00FF0000FFFF00FF0000FFFF00FF0000FFA4
:10382C00FF00FF0000FFFF00FF0000FFFF00FF0094
:10383C0000FFFF00FF0000FFFF00FF0000FFFF0084
:10384C00FF0000FFFF00FF0000FFFF00FF0000FF74
:10385C00FF00FF0000FFFF00FF0000FFFF00FF0064
:10386C0000FFFF00FF0000FFFF00FF0000FFFF0054
:10387C00FF0000FFFF00FF0000FFFF00FF0000FF44
:10388C00FF00FF0000FFFF00FF0000FFFF00FF0034
:10389C0000FFFF00FF0000FFFF00FF0000FFFF0024
:1038AC00FF0000FFFF00FF0000FFFF00FF0000FF14
:1038BC00FF00FF0000FFFF00FF0000FFFF00FF0004
:1038CC0000FFFF00FF0000FFFF00FF0000FFFF00F4
:1038DC00FF0000FFFF00FF0000FFFF00FF0000FFE4
:1038EC00FF00FF0000FFFF00FF0000FFFF00FF00D4
:1038FC0000FFFF00FF0000FFFF00FF0000FFFF00C4
:10390C00FF0000FFFF00FF0000FFFF00FF0000FFB3
:10391C00FF00FF0000FFFF00FF0000FFFF00FF00A3
:10392C0000FFFF00FF0000FFFF00FF0000FFFF0093
:10393C00FF0000FFFF00FF0000FFFF00FF0000FF83
:10394C00FF00FF0000FFFF00FF0000FFFF00FF0073
:10395C0000FFFF00FF0000FFFF00FF0000FFFF0063
:10396C00FF0000FFFF00FF0000FFFF00FF0000FF53
:10397C00FF00FF0000FFFF0000000000000000003F
:10398C0000FFFF00FF0000FFFF00FF0000FFFF0033
:10399C00FF0000FFFF00FF0000FFFF00FF0000FF23
:1039AC00FF00FF0000FFFF00FF0000000000000010
:1039BC0000FF7F00000000FFFF00FF00000500007B
:1039CC00000000000000000000461D000000000088
:1039DC000000000000FF7F0000000000000000005D
:1039EC0000FFFF00FF0000000000000000828000CC
:1039FC00000000000000000000FFFF00FF000000BE
:103A0C000000000000FFFF00FF00000000000000AD
:103A1C0000FFFF00FF0000000000000000FFFF009F
:103A2C00FF0000000000000000010000000000008A
:103A3C000000000000D7FC00FF00000000000000A8
:103A4C0000777700000000000000000000FFFF007E
:103A5C00FF0000FFFF00FF0000FFFF00FF0000FF62
:103A6C00FF00FF0000FFFF00FF0000FFFF00FF0052
:103A7C0000FFFF00FF0000FFFF00FF0000FFFF0042
:103A8C00FF0000FFFF00FF0000FFFF00FF0000FF32
:103A9C00FF00FF0000FFFF00FF0000FFFF00FF0022
:103AAC0000FFFF00FF0000FFFF00FF0000FFFF0012
:103ABC00FF0000FFFF00FF0000FFFF00FF0000FF02
:103ACC00FF00FF0000FFFF00FF0000FFFF00FF00F2
:103ADC0000FFFF00FF0000FFFF00FF0000FFFF00E2
:103AEC00FF0000FFFF00FF0000FFFF00FF0000FFD2
:103AFC00FF00FF0000FFFF00FF0000FFFF00FF00C2
:103B0C0000FFFF00FF0000FFFF00FF0000FFFF00B1
:103B1C00FF0000FFFF00FF0000FFFF00FF0000FFA1
:103B2C00FF00FF0000FFFF00FF0000FFFF00FF0091
:103B3C0000FFFF00FF0000FFFF00FF0000FFFF0081
:103B4C00FF0000FFFF00FF0000FFFF00FF0000FF71
:103B5C00FF00FF0000FFFF00FF0000FFFF00FF0061
:103B6C0000FFFF00FF0000FFFF00FF0000FFFF0051
:103B7C00FF0000FFFF00FF0000FFFF00FF0000FF41
:103B8C00FF00FF0000FFFF00FF0000FFFF00FF0031
:103B9C0000FFFF00FF0000FFFF00FF0000FFFF0021
:103BAC00FF0000FFFF00FF0000FFFF00FF0000FF11
:103BBC00FF00FF0000FFFF00FF0000FFFF00FF0001
:103BCC0000FFFF00FF0000FFFF00FF0000FFFF00F1
:103BDC00FF0000FFFF00FF0000FFFF00FF0000FFE1
:103BEC00FF00FF0000FFFF00FF0000FFFF00FF00D1
:103BFC0000FFFF00FF0000FFFF00FF0000FFFF00C1
:103C0C00FF0000FFFF00FF0000FFFF00FF0000FFB0
:103C1C00FF00FF0000FFFF00FF0000FFFF00FF00A0
:103C2C0000FFFF00FF0000FFFF00FF0000FFFF0090
:103C3C00FF0000FFFF00FF0000FFFF00FF0000FF80
:103C4C00FF00FF0000FFFF00FF0000FFFF00FF0070
:103C5C0000FFFF00FF0000FFFF00FF0000FFFF0060
:103C6C00FF0000FFFF00FF0000FFFF00FF0000004F
:103C7C0000000000000007000A0D00000500080B02
:103C8C0000000600090C00000100031B000FD526E4
:103C9C000EFF260E01880000000000200000E0024C
:103CAC000032000120200288140007D7060700000C
:103CBC00E003003AC0702B01002002003700002006
:103CCC00010020810F700100320F0007000020005E
:103CDC0000E002003200000200000066BB0200009F
:103CEC00000040DA0000FE2039200000E002003223
:103CFC00002020900188000006A102888004780032
:103D0C0000EB1F0037E2844454A0B49905BAE28456
:103D1C004454A0B49906BAE2844454A0B40006EB0F
:103D2C00476FDEFD07B2AE0188636CE103003A0A0F
:103D3C00D8010000EB0E0037606CE108003A004D32
:103D4C00EB0A05E80200393420EC0AF0A08B05E9F7
:103D5C00F9FF3E0400376168E10100320086EB0B8D
:103D6C00000719C7BA1905BA0E04E003003A0A0095
:103D7C00E0DBFF3A000006FE07B2AE02888A047848
:103D8C00F5FF370CD0A3E20F4D1C003989027835B2
:103D9C004DBA0A05E80200393420EC0AF0A08B0574
:103DAC00E90F0032254DBA0A05E80200393420EC3F
:103DBC000AF0A08B05E90800320C00E00600321571
:103DCC00CDBA0A05E80200393420EC0AF0A08B05C4
:103DDC00E98984E854A0B40B00E0E2FF3A00000645
:103DEC009902BA055D788B05E9F7FF32C82ADE0522
:103DFC005D788B05E9F3FF320C00E0F1FF3219DD41
:103E0C00BAEEFF373600F8809FBE829FBE849FBEFD
:103E1C00869FBE0400FA04A8A9001180100798A17F
:103E2C001180010F781E00906400600000E0080013
:103E3C003A9E00900002200080600000E003003AEF
:103E4C00F611A81D82A8B000371E00906400600017
:103E5C0000E070003A9E009000022000806000009C
:103E6C00E06B0032F6D1BF6140600004E0440032E8
:103E7C00F611A9F631A81E00780040784EF0B74E26
:103E8C00D0BF0080FBE40F50310032E40F500C0027
:103E9C003CE10F50180032E10F5003003C0000E0F1
:103EAC001200322D0037E20F50140032E30F501580
:103EBC000032280037E70F50230032E70F50030081
:103ECC003CE60F50110032210037E80F501E003233
:103EDC00E90F501500321C0037DA39071A0037EF9A
:103EEC003907DA4D07170037E43907908F8814002B
:103EFC0037E01E21908F88110037033A071000BE5F
:103F0C00C08F88D18F88801F21908F88013A07C776
:103F1C004607080037094507908F880500370000D1
:103F2C0000030037000000010037000000000826E5
:103F3C00808F88EC71EF1D82A85F0037F6D1BF62CD
:103F4C0040600004E01000321E0090700060000021
:103F5C00E00C003A818F80ECD1BF0080FB008040E8
:103F6C009E0078814078014878ECD1BF0040E8ECA5
:103F7C00F1B71D82A80E0037F6D1BF624060000475
:103F8C00E00800321E00907000600000E004003277
:103F9C0010C0B3F4F1B7F631A90200371D82A83D69
:103FAC0000373C00371E00906400600000E01D00EC
:103FBC00329E00900002200080600000E018003A61
:103FCC0000000000000000000000000000000000E5
:103FDC000000908F801040780080FB801188908FBB
:103FEC00800000E8908F881D82A8000000001180DE
:103FFC006100600000E0FCFF3A00000000000000DF
:10400C0000000000001B00371E00906400600000E0
:10401C00E01700329E00900002200080600000E05B
:10402C001200329E00900000280080600000E00D1D
:10403C00003A908F801040780080FB801188908F20
:10404C00800000E8908F881D82A80000000011807D
:10405C006100600000E0FCFF3A0080FA4F03BE4FA5
:10406C0002BE4F01BE4F00BE3600F90040063600BE
:10407C00F8809FBE829FBE849FBE869FBE0200FAC0
:10408C00008080211280014178811D23827078008C
:10409C0080800000E8008088018080F07F20808F85
:1040AC00500100360030EF018080108080808F50EE
:1040BC0008003A1080800000E8108088118080F0A1
:1040CC007F20808F500100360230EF10C0B32125C5
:1040DC0007000F789E007800A7200080405001BE9A
:1040EC004000BE0000786100600040780004E016DB
:1040FC0000329E007880A6200080403002BE200353
:10410C00BE1000200100206011B800007281807286
:10411C000201738381739E027884A620048242007C
:10412C009ABE0292BE9E007870A62000804011C0FC
:10413C00B30148780168A90080FA4F03BE4F02BE54
:10414C004F01BE4F00BE3600F90040063600F88025
:10415C009FBE829FBE849FBE869FBE881F78000034
:10416C00FA60808061138001417881A52382707888
:10417C006080800000E8608088618080F03F208053
:10418C008F500100360C30EF618080708080808F02
:10419C005008003A7080800000E870808871808040
:1041AC00F03F20808F500100360E30EF20C0B3D688
:1041BC00240700047820C0B3D3240781A620010073
:1041CC00403002BE2003BE1000200100206011B858
:1041DC0000007281807202017383817384A62004B3
:1041EC000244009ABE0292BE20C0B3C2240771A63C
:1041FC002001004011C0B30148780368A90080FA7F
:10420C004F04784F03BE4F02BE4F01BE4F00BE3667
:10421C0000F90040063600F8809FBE829FBE849F46
:10422C00BE869FBE881F780000FAC08080617880AF
:10423C0001417881ED23827078C080800000E8C055
:10424C008088C18080F03F20808F5001003618306C
:10425C00EFC18080D08080808F5008003AD0808061
:10426C000000E8D08088D18080F03F20808F500102
:10427C0000361A30EF30C0B393240700047830C0F6
:10428C00B390240781A6200100403002BE2003BE5B
:10429C001000200100206011B800007281807202B1
:1042AC00017383817384A620040244009ABE029297
:1042BC00BE30C0B37F240771A62001004011C0B3EB
:1042CC000148780728A90080FA4F04784F03BE4FA5
:1042DC0002BE4F01BE4F00BE3600F900400636004C
:1042EC00F8809FBE829FBE849FBE869FBE0000FA50
:1042FC00518080408080808F501300320188A9004B
:10430C000000508080819D2361407880407810C0EF
:10431C00B3692C070004E0F8FF325080800000E8FD
:10432C00508088518080F00720808F500300360A1F
:10433C0030EF0100370188A90080FA4F03BE4F020D
:10434C00BE4F01BE4F00BE3600F90040063600F8E5
:10435C00809FBE829FBE849FBE869FBE0000FAB126
:10436C008080A08080808F501300320388A90000C9
:10437C0000B0808081E52361407880407820C0B314
:10438C00442C070004E0F8FF32B080800000E8B055
:10439C008088B18080F00720808F50030036163063
:1043AC00EF0100370388A90080FA4F03BE4F02BE0D
:1043BC004F01BE4F00BE3600F90040063600F880B3
:1043CC009FBE829FBE849FBE869FBE0000FA118155
:1043DC0080008180808F501300320748A9000000B4
:1043EC00108180812D2461407880407830C0B31FCB
:1043FC002C070004E0F8FF321081800000E81081E7
:10440C0088118180F00720808F500300362230EF16
:10441C000100370748A90080FA4F03BE4F02BE4F78
:10442C0001BE4F00BE3600F90040063600F8809FF2
:10443C00BE829FBE849FBE869FBE0200FA3A0807CA
:10444C00000F788160801E007871989810C0B310AE
:10445C00F2B70BA8A90080FA4F03BE4F02BE4F0162
:10446C00BE4F00BE3600F90040063600F8809FBEF5
:10447C00829FBE849FBE869FBE0200FA250807005D
:10448C000F78D160801E007861809810C0B310F254
:10449C00B70C48A90080FA4F03BE4F02BE4F01BEB5
:1044AC004F00BE3600F90040063600F8809FBE82F1
:1044BC009FBE849FBE869FBE0200FA100807000FA5
:1044CC00780161801E007801B89810C0B310F2B763
:1044DC000CA8A90080FA4F03BE4F02BE4F01BE4F7D
:1044EC0000BE3600F90040063600F8809FBE829F61
:1044FC00BE849FBE869FBE0200FAFB0707000F78A2
:10450C001161801E007811109910C0B310F2B70C15
:10451C00C8A90080FA4F03BE4F02BE4F01BE4F0028
:10452C00BE3600F90040063600F8809FBE829FBE62
:10453C00849FBE869FBE0200FAE60707000F782113
:10454C0061801E007841109810C0B310F2B70CE8CF
:10455C00A90080FA4F03BE4F02BE4F01BE4F00BEF2
:10456C003600F90040063600F8809FBE829FBE845C
:10457C009FBE869FBE0200FAD50707000F783161F7
:10458C00801E007811109910C0B310F2B70D08A955
:10459C000080FA4F03BE4F02BE4F01BE4F00BE3625
:1045AC0000F90040063600F8809FBE829FBE849FB3
:1045BC00BE869FBE0200FAC00707000F78416180DB
:1045CC001E007801B89810C0B310F2B70D28A900DE
:1045DC0080FA4F03BE4F02BE4F01BE4F00BE3600E5
:1045EC00F90040063600F8809FBE829FBE849FBEB5
:1045FC00869FBE0200FAAB0707000F785161801E40
:10460C00007861809810C0B310F2B70D48A90080F3
:10461C00FA4F03BE4F02BE4F01BE4F00BE3600F92B
:10462C000040063600F8809FBE829FBE849FBE86E7
:10463C009FBE0200FA920707000F786161801E008E
:10464C007851289810C0B310F2B70D68A90080FA01
:10465C004F03BE4F02BE4F01BE4F00BE3600F900E5
:10466C0040063600F8809FBE829FBE849FBE869F08
:10467C00BE0200FA810707000F787161801E007876
:10468C0071989810C0B310F2B70D88A90080FA4F3A
:10469C0003BE4F02BE4F01BE4F00BE3600F90040B4
:1046AC00063600F8809FBE829FBE849FBE869FBE4A
:1046BC000200FA6C0707000F788161801E007841B8
:1046CC00109810C0B310F2B70DA8A90080FA4F03D0
:1046DC00BE4F02BE4F01BE4F00BE3600F900400671
:1046EC003600F8809FBE829FBE849FBE869FBE020E
:1046FC0000FA570707000F789161801E0078512847
:10470C009810C0B310F2B70DC8A90080FA4F03BEC1
:10471C004F02BE4F01BE4F00BE3600F900400600EE
:10472C0000FA0B68A90080FA0040060000FA3AEE85
:10473C00A80468A90080FA0040063600F8809FBEE5
:10474C00829FBE849FBE869FBE0200FA4AD0BF00E5
:10475C0004E0060032DA6AA9616080010F784A70C1
:10476C00EFD80AA80200373AEEA9CA40070248A9B6
:10477C000080FA4F03BE4F02BE4F01BE4F00BE3643
:10478C0000F9004006801F780000FAC09026905671
:10479C0088E0C820A05688209080B056880108A9CF
:1047AC000080FA4F00780040063600F8809FBE82E9
:1047BC009FBE849FBE869FBE0000FA02D2BF00043B
:1047CC00E0110032009080800040004E26008040B6
:1047DC001000780000E00A00320090808000400059
:1047EC004E260080401000786B4807009080000037
:1047FC00E80090880500370032EF2308A92108A9AA
:10480C00A948070308A90080FA4F03BE4F02BE4F08
:10481C0001BE4F00BE3600F9004006809FBE00006E
:10482C00FA3156800002200080600000E003003264
:10483C00C40AA910C0B30AF2B70088A90080FA4FC5
:10484C0000BE0040063600F8809FBE829FBE849F4B
:10485C00BE869FBE0400FAB07080808188162EEF51
:10486C002070809081882E70EFA300378181802E7C
:10487C00D0BF0080FB0008DE6100600040780004BF
:10488C00E09800322ED0BF80407840E020B2220762
:1048AC0047981E00780000E08B00329181802ED05A
:1048BC00BF0080FB0008DE6100600040780004E06F
:1048CC004200329E007800A7200080403002BE20BB
:1048DC0003BE2000200100206011B800006281801E
:1048EC0062020163838163E00F50E08F58E00F593F
:1048FC00E08F597200329E0078A0A7200080409073
:10490C0000782E40900080FB0000E90008DE61007A
:10491C00600040780004E06600329E007880A7209A
:10492C000080409000782E40900080FB0000E9123F
:10493C0000200010DD8100701E017880A72000008F
:10494C00410108789E007880A6200080403002BE8D
:10495C002003BE2000200100206011B800007281ED
:10496C0080720201738381739E027884A620048274
:10497C0042009ABE0292BE9E007870A62000804033
:10498C0011C0B30148784100379E007800A7200081
:10499C0080403002BE2003BE400020010020601188
:1049AC00B8000062818062020163838163E00F5072
:1049BC00E08F58E00F59E08F593000329E0078E0BC
:1049CC00A7200080409000782E40900080FB0000D3
:1049DC00E90008DE6100600040780004E024003249
:1049EC009E0078C0A7200080409000782E40900058
:1049FC0080FB0000E91200200010DD8100701E0118
:104A0C0078C0A7200000410108789E007880A6207D
:104A1C000080403002BE2003BE4000200100206018
:104A2C0011B80000728180720201738381739E023F
:104A3C007884A620048242009ABE0292BE9E007820
:104A4C0070A62000804011C0B30148782ED0BF0062
:104A5C0040E82EF0B72ED0BFEF4F505AFF3600482B
:104A6C00A90080FA4F03BE4F02BE4F01BE4F00BEDD
:104A7C003600F90040063600F8809FBE829FBE8447
:104A8C009FBE869FBE0400FA907180B08188322E42
:104A9C00EF007180C081883470EFA30037B1818042
:104AAC0034D0BF0080FB0008DE610060004078005D
:104ABC0004E098003234D0BF80407800E220F72127
:104ACC0007000F7834D0BF80407800E220582207CE
:104ADC002047981E00780000E08B0032C1818034A2
:104AEC00D0BF0080FB0008DE61006000407800044D
:104AFC00E04200329E007800A7200080403002BEC9
:104B0C002003BE2000200100206011B8000062814B
:104B1C008062020163838163E00F50E08F58E00FE5
:104B2C0059E08F597200329E0078A0A72000804077
:104B3C009000782E40900080FB0000E90008DE61B8
:104B4C0000600040780004E06600329E007880A788
:104B5C00200080409000782E40900080FB0000E9FF
:104B6C001200200010DD8100701E017880A720004B
:104B7C0000410108789E007880A620008040300219
:104B8C00BE2003BE2000200100206011B80000727E
:104B9C008180720201738381739E027884A6200443
:104BAC008242009ABE0292BE9E007870A6200080BF
:104BBC004011C0B30148784100379E007800A7200F
:104BCC000080403002BE2003BE4000200100206067
:104BDC0011B8000062818062020163838163E00F7F
:104BEC0050E08F58E00F59E08F593000329E00781A
:104BFC00E0A7200080409000782E40900080FB00C1
:104C0C0000E90008DE6100600040780004E0240048
:104C1C00329E0078C0A7200080409000782E4090F3
:104C2C000080FB0000E91200200010DD8100701EE6
:104C3C000178C0A7200000410108789E007880A66A
:104C4C00200080403002BE2003BE40002001002026
:104C5C006011B80000728180720201738381739EAF
:104C6C00027884A620048242009ABE0292BE9E0064
:104C7C007870A62000804011C0B301487834D0BFB2
:104C8C000040E834F0B734D0BFEF4F505AFF360035
:104C9C0068A90080FA4F03BE4F02BE4F01BE4F0001
:104CAC00BE3600F90040063600F8809FBE829FBEDB
:104CBC00849FBE869FBE0400FA707280E081884E8D
:104CCC002EEFE07180F081883A70EFA30037E1811C
:104CDC00803AD0BF0080FB0008DE610060004078A5
:104CEC000004E09800323AD0BF804078C0E3203C0A
:104CFC002107000F783AD0BF804078C0E3209D2177
:104D0C00072047981E00780000E08B0032F181806C
:104D1C003AD0BF0080FB0008DE61006000407800E4
:104D2C0004E04200329E007800A720008040300250
:104D3C00BE2003BE2000200100206011B8000062DC
:104D4C00818062020163838163E00F50E08F58E041
:104D5C000F59E08F597200329E0078A0A720008076
:104D6C00409000782E40900080FB0000E90008DEA7
:104D7C006100600040780004E06600329E0078809C
:104D8C00A7200080409000782E40900080FB00000F
:104D9C00E91200200010DD8100701E017880A72030
:104DAC000000410108789E007880A62000804030E9
:104DBC0002BE2003BE2000200100206011B80000BC
:104DCC00728180720201738381739E027884A620A3
:104DDC00048242009ABE0292BE9E007870A6200009
:104DEC00804011C0B30148784100379E007800A77D
:104DFC00200080403002BE2003BE40002001002075
:104E0C006011B8000062818062020163838163E0FB
:104E1C000F50E08F58E00F59E08F593000329E0050
:104E2C0078E0A7200080409000782E40900080FB16
:104E3C000000E90008DE6100600040780004E02416
:104E4C0000329E0078C0A7200080409000782E4051
:104E5C00900080FB0000E91200200010DD81007042
:104E6C001E0178C0A7200000410108789E007880C0
:104E7C00A6200080403002BE2003BE40002001006E
:104E8C00206011B8000072818072020173838173FB
:104E9C009E027884A620048242009ABE0292BE9E94
:104EAC00007870A62000804011C0B30148783AD039
:104EBC00BF0040E83AF0B73AD0BFEF4F505AFF3638
:104ECC000268A90080FA4F03BE4F02BE4F01BE4FCD
:104EDC0000BE3600F90040063600F8809FBE829F67
:104EEC00BE849FBE869FBE0400FA507380108288D9
:104EFC006A2EEFC072802082884070EFA3003711B9
:104F0C00828040D0BF0080FB0008DE610060004062
:104F1C00780004E098003240D0BF80407880E520D3
:104F2C00812007000F7840D0BF80407880E520E2D8
:104F3C0020072047981E00780000E08B0032218269
:104F4C008040D0BF0080FB0008DE6100600040782C
:104F5C000004E04200329E007800A7200080403020
:104F6C0002BE2003BE2000200100206011B800000A
:104F7C0062818062020163838163E00F50E08F588D
:104F8C00E00F59E08F597200329E0078A0A72000E4
:104F9C0080409000782E40900080FB0000E90008D3
:104FAC00DE6100600040780004E06600329E00780C
:104FBC0080A7200080409000782E40900080FB005D
:104FCC0000E91200200010DD8100701E017880A71E
:104FDC00200000410108789E007880A620008040C7
:104FEC003002BE2003BE2000200100206011B8005A
:104FFC0000728180720201738381739E027884A691
:10500C0020048242009ABE0292BE9E007870A620B6
:10501C0000804011C0B30148784100379E007800F1
:10502C00A7200080403002BE2003BE4000200100BB
:10503C00206011B800006281806202016383816389
:10504C00E00F50E08F58E00F59E08F593000329E3E
:10505C000078E0A7200080409000782E40900080DF
:10506C00FB0000E90008DE6100600040780004E00D
:10507C002400329E0078C0A7200080409000782E3B
:10508C0040900080FB0000E91200200010DD810040
:10509C00701E0178C0A7200000410108789E00789E
:1050AC0080A6200080403002BE2003BE40002001BC
:1050BC0000206011B800007281807202017383813C
:1050CC00739E027884A620048242009ABE0292BE8D
:1050DC009E007870A62000804011C0B30148784033
:1050EC00D0BF0040E840F0B740D0BFEF4F505AFF60
:1050FC00360968A90080FA4F03BE4F02BE4F01BEAD
:10510C004F00BE3600F90040060000FAC028A9FF87
:10511C00FF370000FAC068A9FFFF370000FAC0484B
:10512C00A9FFFF370000FAC088A9FFFF370000FA7B
:10513C00FFFF3700000503F0A2889FBE8A9FBE8C3C
:10514C001F78FA00070101336450E14F00326420EC
:10515C00E152003203826C07003B0905D00306D0F4
:10516C00820F540C065D020039020032890178036B
:10517C00067885825504003D0003FD8103FD850200
:10518C00EA8B8542840F7202003B600010E08018AD
:10519C006011B80005EB7A28E10A0039060078C7DF
:1051AC005DDDF707B28780752D00378281710A01AA
:1051BC00786105608180D10080D38502E9F9FF3BDD
:1051CC0006044087844802003B600414E0841C09F8
:1051DC0088A30700328A817182817161016489041C
:1051EC00D10884D38B05E81700370978A313003A4C
:1051FC000B00E01300348B05E908044489844C0A45
:10520C0044740978A30D003A0B00E00700348B05B9
:10521C00E908044489844C01003A0B00200978A366
:10522C00F7FF320001EB0200378281710A017870BE
:10523C0000070CF0A701F0A0B900376420E10200D0
:10524C003A838F6CB900330801BE0200BEB200373E
:10525C00889FBE8A9FBE8C1F789D0007A4003303D5
:10526C00866C6450E12E00326420E13300326150D0
:10527C00E12F00326120E1310032858555EB07B01A
:10528C0009002008042005003708044489844C0ACE
:10529C00003106034387834B00015381815BF8FF88
:1052AC00330203BE0800A008044489844CF6FF397D
:1052BC00C639DD8301730100321300208904D10843
:1052CC0084D30998A30500320800A70300A0890421
:1052DC00D10884D38B05E88904D10884D30001EB71
:1052EC000281D234000701F0A10CF0A701F0A07CE0
:1052FC0000376420E17E00320801BE0200BEF7FFD9
:10530C00376120E17900326000B8F3FF37000020EC
:10531C0001F827F0FF37140020F30137F4FF2FF1C9
:10532C0001370001BE4400070470A703F0A103F885
:10533C00A313003A6509B11000320900356928E160
:10534C0002003501002800000500004081804885DE
:10535C0002E9FCFF3A000006F88F42050035810097
:10536C00D10080D38502E8FCFF3A0000068000EBF8
:10537C000000054F89DE820178EE01376011B8FC20
:10538C0001378100206180550B003D0B002061FE30
:10539C002F0100E11D00348281716101648904D107
:1053AC000884D30000E8FAFF3A710020610064031E
:1053BC000070020060090032610444E0844C0988EA
:1053CC00A50500328B05E86808E102003A8904D192
:1053DC000884D3F20F200258E105003DC75DDDF9CA
:1053EC0007B28980750800780000060BF8278B003F
:1053FC0078000005C70ADEF107B2F50FB2080032DB
:10540C00E1CF420200320170A0240005810F70012F
:10541C000032040805440005810F7002003A1400A4
:10542C00058502E900004081C048FCFF3B0170A0EB
:10543C002400050004BEE9FF070003BE0405BE02FC
:10544C0000BEE5FF07844F750000060200BE6450E5
:10545C00E10500366420E10200360968A301003A38
:10546C000800BE0160A04F06784F05BE4F04BE0079
:10547C000006F0FF2FF1FF27F9FF37889FBE8A9FA8
:10548C00BE8C1F78E4FF07EBFF3303866C6450E19E
:10549C002400326420E12700326150E122003261A5
:1054AC0020E12100328B8542EB07B10134B8003A80
:1054BC00B808044289844A013AB80030B888804060
:1054CC0009014A0400330000408180480201498BE5
:1054DC0005E9C909DD830170010032130020C814ED
:1054EC00DE4814DD4709DE1200B2C808DE088470FD
:1054FC0085FF0701F0A10CF0A701F0A0CDFF3761EB
:10550C0020E1CFFF320801BE0200BEF7FF37615029
:10551C00E1FCFF3AC9FF37889FBE8A9FBE8C1F787B
:10552C000004BE9AFF070478A326003A6120E12507
:10553C00003209F8A325003A6420E1210032F50776
:10554C00B10508A30200320000408180486044B8D5
:10555C000310200200200000408180480805448987
:10556C00854C0A05418B85490A05508B85580300EB
:10557C00330A00BE0204748384748301D10281D384
:10558C00830F71F0FF3A8904D10884D360014982FA
:10559C000178C1ADDEFB07B04DFF0798FF370960FE
:1055AC00A00800BE95FF37120220A29088F0FF2FB2
:1055BC00F1FF2790FF376022B80602200000D0814F
:1055CC0080D20482D28582D20000A0020252838251
:1055DC005A03003102024283824A0000A10603E909
:1055EC00F3FF3A000006EFFF070400BE0000068838
:1055FC009FBE8A9FBE300442B0844A30054B9085D2
:10560C004B6000B10898BE0A90BE0440E105C8E1A9
:10561C0006D0E107D8E10200316800401008E84FDD
:10562C0005BE4F04BE000006889FBE8A9FBE300494
:10563C00BE2005BE04185405985C06185D07985DDD
:10564C001100200440E105C8E106D0E107D8E101D2
:10565C0000398000EB1088104F05BE4F04BE0000CF
:10566C00061200FA889FBE8A9FBE8C9FBEE0B79F31
:10567C00F1B79F82BF9F93BF9F0605BE0404BE0077
:10568C0000EBD0B79FC0B79FB0B79FA0B79F90B7A4
:10569C009F0006785FB197CFB0978201413FB097DA
:1056AC000200E004003D3700077E8057C0FF07036F
:1056BC0000373300077E8057CFFF07DFB6970D000A
:1056CC00E00C00356FB297FFB2970FBB979FBB975B
:1056DC001000200100206011B80002728182720259
:1056EC0003738383731B00070C06E8010420810FEE
:1056FC0056E0FF3A0D00E004003D0802BE0A03BE6E
:10570C007E8057A3FF075FA8970000E005003A1FB3
:10571C00B297AFB2973FB397CFB3970900076FB06B
:10572C0097FFB0970FB9979FB9974F06BE4F05BE1D
:10573C004F04BE0080FA000006010007000006A41A
:10574C00B79FB5B79FC6B79FD7B79F0000064F0945
:10575C00DE828171B3B79F4F01DE81804082807001
:10576C00A1B79F8FB0974F09DE00004002007090E8
:10577C00B79F7FA8974F01DE81804082807081B7F0
:10578C009F0D00074F3ADE000040040070F0AF9F01
:10579C0008000704024285824A06034B87834BDFCD
:1057AC00FF070802BE0A03BE0000062FB297BFB265
:1057BC00974FB397DFB397000006881F7818002027
:1057CC00881F7889FF078F87E94F047800000680CF
:1057DC001FEB84FF078F87E9000006889FBE8A9F16
:1057EC00BEE00F50E08F58E00F59E08F590C003D90
:1057FC006044B86055B800005481805C02015D8340
:10580C00815D18002015000708003D1800070004F2
:10581C00EB0500370004EB0F000702003D120007F8
:10582C00180020DCFF070800E00600326022B86098
:10583C0033B800005281805A02015B83815B4F05B3
:10584C00BE4F04BE000006E00F52E08F5AE00F5B23
:10585C00E08F5B0000066044B86055B804025485C4
:10586C00825C06035D87835D000006889FBE8A9F6D
:10587C00BE8C1F78E00F50E08F58E00F59E08F5925
:10588C000D003D6044B86055B800005481805C0246
:10589C00015D83815D1C00200820E109A8E10AB0AC
:1058AC00E10BB8E10D003D0800370006EBE00F52AC
:1058BC00E08F5AE00F5BE08F5B06003D6044B86000
:1058CC0055B804025485825C06035D87835DAAFF8C
:1058DC00070C00E00600326022B86033B8000052BA
:1058EC0081805A02015B83815B4F06784F05BE4F66
:1058FC0004BE000006889FBE8A9FBE841F7866FE89
:10590C00074F0078110033F0FF2F838F6C06003B9C
:10591C000405650A00A708003709F0A61000200846
:10592C000037820F54838F5C030039100020010074
:10593C003E00002009F0A70000EA4F05BE4F04BE50
:10594C000000E0000006881F780304780300E007DD
:10595C00003D600010E08018600119E08119020020
:10596C003B01F02D03003704000708F0A701F0A05D
:10597C004F0478000006889FBE8A9FBE0082700488
:10598C0002710482712600320004BE0200BE601156
:10599C00B86B09209502200182CF0A00390541B16C
:1059AC000082CF0700390541B10982CF04003905C7
:1059BC0041B10882CF0100390541B10542521200B4
:1059CC00320A003B8281716101648100D10080D375
:1059DC008984D30884D38B05E80442E8F7FF3A079F
:1059EC00003708044489844C0000488180488B05AA
:1059FC00E90442E9F9FF3AD8FD074F05BE4F04BE52
:105A0C00000006800178020037B159780201E902E2
:105A1C0000E0FCFF3A000006800178020037815953
:105A2C00780201E90200E0FCFF3A0000068000EB7E
:105A3C00504A8B614A8B11C0B38094260148780080
:105A4C0000068094261004E002003A100020F4FFB7
:105A5C0007D2E624631C24504A83614A8309000759
:105A6C00920323030020000141818149524A8B6338
:105A7C004A8B03007800F0A1000006020AB9001B53
:105A8C00B90200B88100428100430000060C00FA04
:105A9C00881F78400798214F98324F984E01902ECE
:105AAC0048908080FB2003200088B900007800001B
:105ABC00413081883081801000788000783E489099
:105ACC000080FB000040008F40308180E00090118E
:105ADC0007981E00781000788080EA1E00900080E5
:105AEC00602007989E00783107982E0090BE009099
:105AFC00010478180C6838079800000000000000BA
:105B0C0000004F04780080FA0000060C00FA881F91
:105B1C0078400798214F98324F984E01902E48901C
:105B2C008080FB2003200088B90000780000413001
:105B3C0081883081801000788000783E4890008009
:105B4C00FB000040008F40308180E00090110798EE
:105B5C001E00789000781E00900080EA8080681EFD
:105B6C0000900080602007989E00783107982E00E6
:105B7C0090BE0090010478180C683807984F047890
:105B8C000080FA0000060C00FA881F784007982164
:105B9C004F98324F984E01902E48908080FB2003F6
:105BAC00200088B900007800004130818830818065
:105BBC001000788000783E48900080FB0000400088
:105BCC008F40308180E000901107989E0090210753
:105BDC00989E00783107982E0090BE0090010478B2
:105BEC00180C683807984F04780080FA00000604F7
:105BFC0000FA000F782147983247982E4090808009
:105C0C00FB1E01782003200088B9000078E20078A0
:105C1C003E40900080FB0000406101782E40908057
:105C2C0080FB9E01782003200088B90000786C006E
:105C3C00406300780001612E40908080FB9E0178CB
:105C4C002003200088B90000786E004063007800C3
:105C5C0010DE0040780080FA0000060200FA004FC7
:105C6C00781E80FBE189266140780080FA000006EE
:105C7C000600FA1007984147985247984E4090F307
:105C8C00FF07004F789E80FB1E01902003200088A8
:105C9C00B9000078C002B00000411001BE5E409017
:105CAC000080FBC200DDC08B260080401000BE02CD
:105CBC000278030178800178010078030262000009
:105CCC00618000EBC000DD0000200001BE6120B847
:105CDC00000171818171E00F51E08F590200321087
:105CEC00C0B30100370040EB0080FA000006000052
:105CFC00FAE022210080FA0000060000FAC0CB2155
:105D0C000080FA0000060000FAA074220080FA005D
:105D1C0000060000FAC0728011800A0000000080AA
:105D2C00FBC300DD007180AA800A0000000080FB2C
:105D3C004200DD808040007180BB800A00000000C2
:105D4C0080FB000040808040007180CC800A000005
:105D5C00000080FB0080400040786300B9000078B0
:105D6C00804078701D23014878701D231040788086
:105D7C0040E8B0CB21014878701D2310407880C0DA
:105D8C00E8907422014878701D231040780004E0DC
:105D9C0003003A10C0B3CB3B0702003720C0B3C896
:105DAC003B070080FA0000060200FA000F789E0004
:105DBC0078D0A8200080401040780080FA000006BF
:105DCC000000FAC4FF070400076307071C0607005E
:105DDC0080FA0000060000FA80E32070918800D958
:105DEC0020C09188100020D091880000EBE09188B1
:105DFC000000EBF09188000320009288C080208086
:105E0C009188C08220909188000820909288C0B818
:105E1C0020A091880000EB80928880252111C0B3CE
:105E2C0001487800B220B09188000021A0928860CF
:105E3C000421109288600421209288600421309201
:105E4C008860042140928880002060928880E32042
:105E5C0000938860D9205093880008206093887044
:105E6C0000207093881000208093887003209093FA
:105E7C0088C08020109388C08220209388008020C6
:105E8C0020948800B9203093880000EB109488A0EF
:105E9C00282111C0B301487820B22040938810000B
:105EAC0020309488600421A09388600421B09388EA
:105EBC00600421C09388600421D09388800020F076
:105ECC009388C0E12090948820D820E094884000EA
:105EDC0020F094882000200095880000EB10958815
:105EEC00200220209588C08020A09488C08220B0F9
:105EFC009488400020B0958860B820C09488100029
:105F0C0020A09588C02B2111C0B301487800B22085
:105F1C00D09488000820C095886004213095886052
:105F2C000421409588600421509588600421609577
:105F3C0088800020809588C0E12020968860D82039
:105F4C0070968800082080968870002090968810A3
:105F5C000020A09688700220B09688A080203096F1
:105F6C0088A0822040968800002240978820B82084
:105F7C005096880000EB309788E02E2111C0B301B9
:105F8C00487800B2206096884000205097886004C2
:105F9C0021C09688600421D09688600421E0968800
:105FAC00600421F09688800020109788C0E120B012
:105FBC00978880D82000988800102010988880003E
:105FCC00202098880000EB30988880022040988828
:105FDC00C08020C09788C08220D09788000220D033
:105FEC009888A0B820E097880000EBC09888003211
:105FFC002111C0B301487800B220F09788004020EE
:10600C00E09888600421509888600421609888602A
:10601C000421709888600421809888800020A098C2
:10602C0088C0E12040998880D82090998800202051
:10603C00A09988900020B09988100020C099889071
:10604C000220D09988C08020509988C08220609905
:10605C0088000420609A88A0B820709988100020CD
:10606C00509A8820352111C0B301487800B22080A5
:10607C009988008020709A88600421E099886004D7
:10608C0021F09988600421009A88600421109A8874
:10609C00800020309A8840E520D09A8840DA202071
:1060AC009B88000120309B88400020409B8800008A
:1060BC00EB509B88400420609B88600421E09A8808
:1060CC00600421F09A88100020F09B886004210065
:1060DC009B880000EBE09B8840382111C0B301483D
:1060EC0078600421109B88100020009C886004219B
:1060FC00709B88600421809B88600421909B886041
:10610C000421A09B88800020C09B8840E520609CD7
:10611C008820DA20B09C88800020C09C8830002029
:10612C00D09C88100020E09C88300420F09C886073
:10613C000421709C88600421809C88100020809D24
:10614C0088600421909C880000EB709D88603B2146
:10615C0011C0B3014878600421A09C8810002090E5
:10616C009D88600421009D88600421109D88600436
:10617C0021209D88600421309D88800020509D88BE
:10618C00C0E120F09D88C0D820409E88000021509E
:10619C009E88C00020609E880000EB709E88C00224
:1061AC0020809E88600421009E88600421109E88B7
:1061BC00100020109F88600421209E880000EB00B6
:1061CC009F88803E2111C0B3014878600421309E25
:1061DC0088100020209F88803620909E88003620D2
:1061EC00A09E88803820B09E88403820C09E888031
:1061FC000020E09E88403620D09E8880E320809F3F
:10620C0088E0D920D09F88000028E09F88F00020EB
:10621C00F09F8810002000A088F0032010A0886058
:10622C000421909F88600421A09F88100020A0A0CA
:10623C0088600421B09F880000EB90A088A04121C9
:10624C0011C0B3014878600421C09F88100020B0B1
:10625C00A08800442020A08880432030A0880046DD
:10626C002040A08840462050A08840002070A08884
:10627C00C0432060A08880E32010A188E0D9206072
:10628C00A18800002470A188E0002080A188000073
:10629C00EB90A188E00320A0A18860042120A188B4
:1062AC0060042130A18810002030A28860042140B5
:1062BC00A1880000EB20A288C0442111C0B3014882
:1062CC007860042150A18810002040A2880044204E
:1062DC00B0A188804320C0A188004620D0A188C0EE
:1062EC004520E0A18880002000A288C04320F0A1B6
:1062FC008880E320A0A288C0D920F0A288000022C8
:10630C0000A388D0002010A38810002020A388D0E0
:10631C00032030A388600421B0A288600421C0A2AD
:10632C0088100020C0A388600421D0A2880000EB54
:10633C00B0A388E0472111C0B3014878600421E084
:10634C00A288100020D0A388C04A2040A388404ACD
:10635C002050A388C04C2060A388004D2070A388D7
:10636C0040002090A388804A2080A38840E520E04C
:10637C00E588A0DA2030E68800402040E688A000BE
:10638C002050E6880000EB60E688A0042070E688C8
:10639C00C08020F0E588C0822000E6880000220042
:1063AC00E78820B92010E6880000EBF0E68860CE84
:1063BC002111C0B301487820B22020E6884000208B
:1063CC0010E78860042180E68860042190E68860EC
:1063DC000421A0E688600421B0E688800020D0E685
:1063EC008840E52070E788A0DA20C0E7880080208C
:1063FC00D0E788B00020E0E788100020F0E788B0F4
:10640C00042000E888C0802080E788C0822090E7C4
:10641C008800002490E88820B920A0E7881000208C
:10642C0080E88880D12111C0B301487820B220B017
:10643C00E788800020A0E88860042110E8886004C8
:10644C002120E88860042130E88860042140E88835
:10645C0080002060E88880E32000E98820D9205063
:10646C00E98880002060E98830002070E9881000FD
:10647C002080E98830032090E988C0802010E988CA
:10648C00C0822020E98800402020EA88E0B8203033
:10649C00E98810002010EA88A0D42111C0B301486B
:1064AC007800B22040E98800002830EA8860042196
:1064BC00A0E988600421B0E988600421C0E9886003
:1064CC000421D0E988800020F0E98880E32090EA5C
:1064DC008860D920E0EA88000420F0EA8860002077
:1064EC0000EB880000EB10EB8860032020EB88C0E9
:1064FC008020A0EA88C08220B0EA88000021B0EB9E
:10650C008800B920C0EA88100020A0EB88C0D721F1
:10651C0011C0B301487820B220D0EA88200020C0F6
:10652C00EB8860042130EB8860042140EB88600428
:10653C002150EB8860042160EB8880002080EB8880
:10654C0080E32020EC8820D92070EC88400020804B
:10655C00EC8820002090EC880000EBA0EC88200355
:10656C0020B0EC88C0802030EC88C0822040EC88C1
:10657C0000202040ED88E0B82050EC880000EB3083
:10658C00ED88E0DA2111C0B301487800B22060EC4C
:10659C008800002450ED88600421C0EC8860042140
:1065AC00D0EC88600421E0EC88600421F0EC888059
:1065BC00002010ED8880E320B0ED8800D92000EE9B
:1065CC008820002010EE8810002020EE881000207B
:1065DC0030EE8810032040EE88C08020C0ED88C0CB
:1065EC008220D0ED88001020D0EE88C0B820E0EDDD
:1065FC0088100020C0EE8800DE2111C0B30148785D
:10660C0000B220F0ED88000022E0EE8860042150FA
:10661C00EE8860042160EE8860042170EE886004CE
:10662C002180EE88800020A0EE8880E32040EF8857
:10663C0080D92090EF88001020A0EF88800020B037
:10664C00EF880000EBC0EF88800320D0EF88600457
:10665C002150EF8860042160EF8810002060F088E2
:10666C0060042170EF880000EB50F08820E12111CC
:10667C00C0B301487860042180EF8810002070F0CE
:10668C0088600421E0EF88600421F0EF8860042129
:10669C0000F08860042110F08880002030F08880A1
:1066AC00E320D0F08880D92020F18800202030F120
:1066BC008890002040F18810002050F18890032031
:1066CC0060F188600421E0F088600421F0F088100B
:1066DC000020F0F18860042100F1880000EBE0F16B
:1066EC008840E42111C0B301487860042110F1887E
:1066FC0010002000F28860042170F1886004218071
:10670C00F18860042190F188600421A0F188800058
:10671C0020C0F188C0E12060F288C0D820B0F28897
:10672C00000022C0F288D00020D0F288100020E0B7
:10673C00F288D00220F0F28860042170F2886004A4
:10674C002180F28810002080F38860042190F28868
:10675C000000EB70F38860E72111C0B3014878604A
:10676C000421A0F28810002090F38880362000F3DA
:10677C008800362010F38880382020F388C0382019
:10678C0030F38840002050F38840362040F388C016
:10679C00E120F0F388E0D82040F48800002450F485
:1067AC0088E0002060F4880000EB70F488E00220A0
:1067BC0080F48860042100F48860042110F48810AF
:1067CC00002010F58860042120F4880000EB00F50F
:1067DC008880EA2111C0B301487860042130F48824
:1067EC0010002020F58820332090F488A03220A0BF
:1067FC00F488203520B0F488E03420C0F488800080
:10680C0020E0F488E03220D0F488C0E12080F588C4
:10681C00E0D820D0F588000028E0F588F00020F0C2
:10682C00F58810002000F688F0022010F68860042D
:10683C002190F588600421A0F588100020A0F6882E
:10684C00600421B0F5880000EB90F688A0ED2111D2
:10685C00C0B3014878600421C0F588100020B0F660
:10686C008820332020F688A0322030F6882035206E
:10687C0040F68860352050F68840002070F688E09D
:10688C00322060F68880E32010F788C0D92060F7AA
:10689C008800002170F788C0002080F7880000EB8A
:1068AC0090F788C00320A0F78860042120F7886047
:1068BC00042130F78810002030F88860042140F75C
:1068CC00880000EB20F888C0F02111C0B301487893
:1068DC0060042150F78810002040F888C04A20B08E
:1068EC00F788404A20C0F788C04C20D0F788804CED
:1068FC0020E0F78880002000F888804A20F0F78894
:10690C0000E020503A89600421A03A89100020B0A0
:10691C003A890000EBC03A890000EBD03A890000BC
:10692C00EBE03A89A08020603A89A08220703A89F5
:10693C00008020703B8900B820803A890000EB6011
:10694C003B8940772261C1B301487800B220903A6C
:10695C0089100020803B89600421F03A8960042171
:10696C00003B89600421103B89600421203B898015
:10697C000020403B8980E320E03B89A0D820303CBC
:10698C0089004020403C89A00020503C890000EB4D
:10699C00603C89A00220703C89600421F03B896036
:1069AC000421003C89100020003D89600421103C2A
:1069BC00890000EBF03C89607A2211C0B301487861
:1069CC00600421203C89100020103D896004218046
:1069DC003C89600421903C89600421A03C896004BE
:1069EC0021B03C89800020D03C8940E520703D8955
:1069FC0000DA20C03D89100020D03D890000EBE07A
:106A0C003D890000EBF03D89000420003E896004C4
:106A1C0021803D89600421903D89100020903E89A1
:106A2C00600421A03D890000EB803E89807D22110D
:106A3C00C0B3014878600421B03D89100020A03E0D
:106A4C0089600421103E89600421203E8960042164
:106A5C00303E89600421403E89800020603E898060
:106A6C00E320003F8980DA20503F89002020603FDE
:106A7C0089900020703F89100020803F899004206D
:106A8C00903F89600421103F89600421203F8900D8
:106A9C000022204089600421303F890000EB104027
:106AAC0089A0802211C0B3014878600421403F893D
:106ABC00400020304089600421A03F89600421B04F
:106ACC003F89600421C03F89600421D03F89800048
:106ADC0020F03F89602121904089600421E04089A9
:106AEC00100020F040890000EB0041890000EB1001
:106AFC0041890000EB204189600421A04089600499
:106B0C0021B04089000220B04189600421C0408935
:106B1C000000EBA04189C0832211C0B3014878600A
:106B2C000421D04089004020C041896004213041BB
:106B3C00896004214041896004215041896004210D
:106B4C006041898000208041896021212042896038
:106B5C0004217042891000208042890000EB904291
:106B6C0089100020A042890000EBB042896004210A
:106B7C0030428960042140428900042040438960EE
:106B8C000421504289100020304389E0862211C034
:106B9C00B301487860042160428900802050438909
:106BAC00600421C04289600421D04289600421E044
:106BBC004289600421F042898000201043896021C1
:106BCC0021B04389600421004489100020104489BD
:106BDC000000EB2044891000203044890000EB4079
:106BEC004489600421C04389600421D0438910008A
:106BFC0020D04489600421E043890000EBC0448923
:106C0C00008A2211C0B3014878600421F043891036
:106C1C000020E044896004215044896004216044D0
:106C2C00896004217044896004218044898000209B
:106C3C00A044896021214045896004219045891038
:106C4C000020A045890000EBB045890000EBC04551
:106C5C00890000EBD04589600421504589600421EE
:106C6C006045894000206046896004217045891088
:106C7C000020504689208D2211C0B3014878600451
:106C8C0021804589000820704689600421E04589EF
:106C9C00600421F0458960042100468960042110BC
:106CAC00468980002030468940E520D0468960DA4C
:106CBC002020478900042030478960002040478904
:106CCC000000EB504789600420604789600421E094
:106CDC004689600421F04689100020F04789600441
:106CEC00210047890000EBE0478940902211C0B396
:106CFC000148786004211047891000200048896001
:106D0C0004217047896004218047896004219047E1
:106D1C0089600421A04789800020C0478940E52074
:106D2C0060488960DA20B04889000820C048897022
:106D3C000020D04889100020E04889700420F048D9
:106D4C0089600421704889600421804889100020E2
:106D5C008049896004219048890000EB7049896062
:106D6C00932211C0B3014878600421A04889100017
:106D7C0020904989600421004989600421104989C7
:106D8C006004212049896004213049894000205049
:106D9C004989602121F04989600421404A89100009
:106DAC0020504A890000EB604A890000EB704A8948
:106DBC000000EB804A89600421004A89600421109C
:106DCC004A89100020104B89600421204A89000058
:106DDC00EB004B8980962211C0B3014878600421E6
:106DEC00304A89100020204B89600421904A896028
:106DFC000421A04A89600421B04A89600421C04A58
:106E0C0089800020E04A8940E520804B8920DA20E7
:106E1C00D04B89400020E04B89200020F04B8900AA
:106E2C0000EB004C89200420104C89600421904B0D
:106E3C0089600421A04B89100020A04C896004219A
:106E4C00B04B890000EB904C89A0992211C0B30182
:106E5C004878600421C04B89100020B04C89600434
:106E6C0021204C89600421304C89600421404C89DC
:106E7C00600421504C89400020704C89F0E72501BA
:106E8C000020D09288E19288F0E7250100206094E0
:106E9C0088719488F0E725010020F0958801968888
:106EAC00F0E725010020809788919788F0E725016D
:106EBC000020109988219988F0E725010020A09ADC
:106ECC0088B19A88E0EF25010020309C88419C888D
:106EDC00E0F725010020C09D88D19D88E0E72701BF
:106EEC000020509F88619F88E0E727010020E0A0E8
:106EFC0088F1A088E0E72701002070A28881A28891
:106F0C00E0E72701002000A48811A488F0E7250100
:106F1C00002040E78851E788F0E725010020D0E801
:106F2C0088E1E888F0E72501002060EA8871EA88AA
:106F3C00F0E725010020F0EB8801EC88F0E7250153
:106F4C00002080ED8891ED88F0E72501002010EFFE
:106F5C008821EF88E0EF25010020A0F088B1F088AF
:106F6C00E0F72501002030F28841F288E0E72701A4
:106F7C000020C0F388D1F388E0E72701002050F50A
:106F8C008861F588E0E727010020E0F688F1F688B3
:106F9C00E0E72701002070F88881F88810002001B4
:106FAC000020B03B89C13B89600020010020403D9E
:106FBC0089513D89600020010020D03E89E13E8945
:106FCC000001200100206040897140896000B8F008
:106FDC0041890142896000B88043899143896000EE
:106FEC00B81045892145896000B8A04689B1468909
:106FFC0060202001002030488941488960402001F0
:10700C000020C04989D149896000B8504B89614B37
:10701C0089600024010020E04C89F14C890080FA41
:10702C000000060000FAE0252111C0B301487812D7
:10703C00C0B311C0B3E022212A370700292131C087
:10704C00B301487821C0B3E02221133607202C214C
:10705C0041C0B301487831C0B3E022214414074049
:10706C002F2151C0B301487841C0B3E02221C41391
:10707C000760322161C0B301487851C0B3E02221CE
:10708C0064130780352171C0B301487861C0B3E047
:10709C002221F51307A0382181C0B3014878B1C073
:1070AC00B3E022216C1407C03B2191C0B301487896
:1070BC00C1C0B3E022217F1407E03E21A1C0B3017F
:1070CC004878D1C0B3E022210F1307004221B1C090
:1070DC00B3014878E1C0B3E02221AF12072045216B
:1070EC0021C0B3014878F1C0B3E02221703507F11B
:1070FC00C0B3E02221793507404821E1C0B30148F3
:10710C007801C1B3E02221D43507C0CE2111C0B320
:10711C0001487812C0B311C0B3C0CB21DE3607E0F2
:10712C00D12131C0B301487821C0B3C0CB21C735C0
:10713C000700D52141C0B301487831C0B3C0CB2181
:10714C00F8130720D82151C0B301487841C0B3C00F
:10715C00CB2178130740DB2161C0B301487851C0C3
:10716C00B3C0CB2118130760DE2171C0B30148787E
:10717C0061C0B3C0CB21A9130780E12181C0B30149
:10718C004878B1C0B3C0CB21201407A0E42191C032
:10719C00B3014878C1C0B3C0CB21331407C0E72179
:1071AC00A1C0B3014878D1C0B3C0CB21C31207E052
:1071BC00EA21B1C0B3014878E1C0B3C0CB2163125E
:1071CC000700EE2121C0B3014878F1C0B3C0CB2138
:1071DC00243507F1C0B3C0CB212D350720F121E1B7
:1071EC00C0B301487801C1B3C0CB21883507A07763
:1071FC002211C0B30148780041EB11C0B3A0742236
:10720C00923607C07A2231C0B301487821C0B3A0AE
:10721C00742286350721C0B3A07422783507E07D2F
:10722C002231C0B301487831C0B3A074227D350738
:10723C0031C0B3A074226F350700812251C0B30155
:10724C00487841C0B3A074222613072084228040C2
:10725C00EB0148784087228040EB014878608A2215
:10726C008040EB014878808D228040EB014878A06B
:10727C009022A1C0B3014878D1C0B3A074227D1272
:10728C0007C09322B1C0B3014878E1C0B3A0742207
:10729C001D1207E096228040EB014878009A22806C
:1072AC0040EB0148780080FA0000061000FA6007F5
:1072BC0098614F980000EB000F7880D2201007984F
:1072CC00A0D220200798A0D320300798E80047A22E
:1072DC00E029030009B25878EE009030A820008015
:1072EC0040EE48900148786E48900080FB000040CA
:1072FC00EE00786E019000A8200000410108786E25
:10730C0048900080FB0000478048906E019020A8B8
:10731C00200000410148780080FA0000061800FAAD
:10732C00200F986157980000EB000F78C0D2201006
:10733C00079800D320200798E0D320300798E80066
:10734C0047E2DF29030009B25878EC004722E02914
:10735C00030009B25878F0004762E029030009B233
:10736C005878AE089090A820008040EE50900148CC
:10737C00786E50900080FB000040EE00782E099053
:10738C0040A8200000410108786E50900080FB005E
:10739C0000478048902E099060A8200000410148C9
:1073AC00786E50900080FB000047C048902E0990EA
:1073BC0070A8200000410148786E50900080FB00BE
:1073CC0000478050902E099080A820000041014871
:1073DC00780080FA0000060400FA000F7821479824
:1073EC009E0078B0A820008040AE40900148780004
:1073FC0080FA0000060000FA31C0B3E022218EFFB3
:10740C000721C0B3C0CB218BFF0711C0B3A07422DE
:10741C0088FF0731C0B3E02221ABFF0721C0B3C006
:10742C00CB21A8FF0711C0B3A07422A5FF0731C060
:10743C00B3E02221E0FF0711C0B3C0CB21DDFF0771
:10744C000080FA0000060200FA000F788125201E49
:10745C0080400080FA0000060200FA000F78806578
:10746C00201E00400080FA0000060200FA000F788F
:10747C009E007880A5200080401000780080FA00E3
:10748C0000060200FA000F789E0078A0A52000806C
:10749C00401000780080FA0000060200FA000F7815
:1074AC009E007880A5200080408000EB01087800C9
:1074BC0080FA0000060200FA000F789E0078A0A562
:1074CC00200080408000EB0108780080FA00000664
:1074DC000400FA000F782147989E007880A52000C0
:1074EC0080401000789E00780080408025B0AE402F
:1074FC00900148789E007880A5200080401000788C
:10750C008000E81E017880A5200000410108780069
:10751C0080FA0000060400FA000F782147989E00BC
:10752C0078A0A5200080401000789E0078808040D4
:10753C00806520008040AE40900148789E0078A085
:10754C00A5200080401000788000E81E0178A0A5DE
:10755C00200000410108780080FA0000060600FABD
:10756C001007982107980040EB004F781E81FB9E76
:10757C000090E052200000410000406100780000C3
:10758C00E00C003A1E81FB9E0090E052200000416E
:10759C00000040008040AE00900108782E009080E2
:1075AC0000EB2100981000371E81FB9E0090F052DA
:1075BC0020000041000040610078AE00903100983E
:1075CC001E81FB9E0090F05220000041000040E123
:1075DC0000782E00902100981E81FB9E0090F052A6
:1075EC0020000041000040008040AE00900108786F
:1075FC002E00908000EB3100981E80FB1E01904104
:10760C00A620810040E2C0788140E81E0190000174
:10761C004140A6200000410148780080FA00000695
:10762C000600FA1007982107980040EB004F781ECF
:10763C0081FB9E009000532000004100004061003F
:10764C00780000E00C003A1E81FB9E009000532055
:10765C00000041000040008040AE00900108782EF0
:10766C0000908000EB2100981000371E81FB9E00DB
:10767C0090105320000041000040610078AE009053
:10768C003100981E81FB9E00901053200000410099
:10769C000040E100782E00902100981E81FB9E0096
:1076AC0090105320000041000040008040AE00903C
:1076BC000108782E00908000EB3100981E80FB1E94
:1076CC00019041A620810040810041914090814071
:1076DC00E81E019000014140A62000004111409895
:1076EC009E009060A6200080401040788040E81EEC
:1076FC00019060A6200000410148780080FA00004B
:10770C00060800FA1007982107983207980040EBFA
:10771C00004F783E0090B000902E00903100982ED3
:10772C000090BE00902100983E0090300090000028
:10773C00E00500323E0090300090AE0090210098A1
:10774C000800371E81FB9E0090F052200000410083
:10775C000040008040AE00900108783E0090AE00E2
:10776C00903100981E80FB1E019041A620810040A4
:10777C00E2C0788140E81E019000014140A6200043
:10778C0000410148780080FA0000060800FA100752
:10779C00982107983207980040EB004F783E0090F4
:1077AC00B000902E00903100982E0090BE009021D9
:1077BC0000983E00903000900000E00500323E0042
:1077CC0090300090AE00902100980800371E81FB8D
:1077DC009E0090105320000041000040008040AEFD
:1077EC0000900108783E0090AE00903100981E8009
:1077FC00FB1E019041A620810040810041914090E8
:10780C008140E81E019000014140A620000041117A
:10781C0040989E009060A6200080401040788040E8
:10782C00E81E019060A6200000410148780080FA13
:10783C000000060600FA1007982107980040EB009C
:10784C004F782E00902000900000E00A003A9E81B4
:10785C00FB2E0090B000901E0190E0522000804161
:10786C000000400000410108780500372E009020F0
:10787C000090AE0090B100903100982E0090300036
:10788C00900000E00A003A9E81FB2E0090A0009030
:10789C001E0190F052200080410000400000410188
:1078AC0008780500372E0090300090AE0090A100B3
:1078BC00902100981E80FB1E019041A62081004063
:1078CC00E2C0788140E91E019000014140A62000F1
:1078DC0000410148780080FA0000060600FA100703
:1078EC00982107980040EB004F781E81FB9E00907A
:1078FC00005320000041000040E100789E81FB1EF7
:10790C000190105320008041000040620078808F6D
:10791C00502F003A1E81FB9E009000532000004126
:10792C00000040E100782E0090808F5026003A1E17
:10793C0081FB9E009000532000004100004000801D
:10794C00408000EB0108781E81FB9E0090105320B4
:10795C000000410000400080408000EB0108781ED0
:10796C0080FB1E019041A620810040810041914086
:10797C00908140E91E019000014140A62000004189
:10798C001140989E009060A62000804010407880A6
:10799C0040E91E019060A6200000410148783B00A0
:1079AC00372E00902000900000E00A003A9E81FBE8
:1079BC002E0090B000901E019000532000804100DA
:1079CC0000400000410108780500372E009020008F
:1079DC0090AE0090B100903100982E009030009045
:1079EC000000E00A003A9E81FB2E0090A000901E41
:1079FC00019010532000804100004000004101081C
:107A0C00780500372E0090300090AE0090A10090C9
:107A1C002100981E80FB1E019041A6208100408110
:107A2C0000419140908140E91E019000014140A627
:107A3C00200000411140989E009060A620008040DC
:107A4C001040788040E91E019060A62000004101A2
:107A5C0048780080FA0000060600FA1007984147A3
:107A6C00985247984E4090FBF507004F789E80FB4C
:107A7C001E01902003200088B9000078000041000E
:107A8C0003B0DE40900148780080FA000006060042
:107A9C00FA1007984147984E4090EAF507004F7846
:107AAC009E80FB1E01902003200088B90000780006
:107ABC0003B06240780080FA0000060600FA100756
:107ACC00984147984E4090DBF507004F78CE409098
:107ADC001E0090E8FF070080FBCF80DEF200200341
:107AEC000020820F50838F584A003E0006014A0046
:107AFC00370E00371100371700371A00371D0037C3
:107B0C002000372300372600372800372A00372D6E
:107B1C000037300037330037320037350037CE406E
:107B2C00901E0090FA3307380037CE40901E00901C
:107B3C003F3207CE40901E0090543207310037CEB2
:107B4C0040901E0090A532072D0037CE40901E00AD
:107B5C0090D51007290037CE40901E009054100786
:107B6C00250037CE40901E0090F50F07210037CE30
:107B7C0040901E00908910071D00371E0090DE10EB
:107B8C00071A00371E0090F41007170037CE4090EC
:107B9C001E0090AB0F07130037CE40901E00904C88
:107BAC000F070F0037CE40901E0090F610070B0009
:107BBC0037CE40901E0090F71007070037CE40904C
:107BCC001E0090E00E070300370000000100370094
:107BDC0000000080FA0000064E00FA889FBE502775
:107BEC00986127980000EB3007986E209010009059
:107BFC004007984E0090904078214F984E009090FE
:107C0C004190334F984E00901002906407984E00AC
:107C1C00906400407007982E48900080FB6101B979
:107C2C000080EB8080EB020040838048F200200350
:107C3C000020820F50838F58AA0D3E0006010F00C2
:107C4C00372C0237A80D372903378D033716053724
:107C5C006B05370D06372A0737B60737A00D379F48
:107C6C000D379E0D372308379C0D37050A373E48D4
:107C7C00900080FB6101B9E0FF2FF1FF2F02004063
:107C8C00838048B20020030020820F50838F58104D
:107C9C00023E0006010B00370E003711003775004D
:107CAC0037B80037FB00373E013741013744013705
:107CBC00470137AC0137AF0137000000000000006E
:107CCC000000000237000000000000000000FC0172
:107CDC00376E00908000EB5081886181880000EB4A
:107CEC00100798100020000F783900375081806100
:107CFC0081801E01E98201788301E9030033810050
:107D0C00D10080D3FBFF3700007861006000407821
:107D1C000004E02A00321E007800407822C0B380B4
:107D2C0040785E209018F5070004E02200321E0017
:107D3C00780040788040785E20901BFF07E24F501F
:107D4C001000321E00780040788040785E2090232E
:107D5C00FF071E00780040788040785E20906E31DE
:107D6C00071E007800407822C0B38040785E2090D7
:107D7C00F7FE071E00780040788040785E20909EC9
:107D8C0031078080FB1E00E90008DD9E0090010099
:107D9C00701007981E0FE81E0078F00F50C4FF36C5
:107DAC005E209005FD071E00900040788040785EB4
:107DBC00209020FD071E00904800DE004078804097
:107DCC00785E20901AFD071939070004E00F003285
:107DDC00123907000F985E2090E2FC078E08908005
:107DEC0008785E2090D0FC078E08909000980E08C2
:107DFC00901D39078E08905E209061FD0797013722
:107E0C006E00908000EB508188618188100020000A
:107E1C000F783900375081806181801E01E90202A0
:107E2C00780402E90300338100D10080D3FBFF37D3
:107E3C000000786100600040780004E02A00321EE7
:107E4C00007800407832C0B38040785E2090B5F462
:107E5C00070004E02200321E007800407880407851
:107E6C005E2090B8FE07E34F501600321E007800DB
:107E7C0040788040785E2090C0FE071E007800405D
:107E8C00788040785E20905431071E00780040784E
:107E9C008040785E20905A31071E0078004078327E
:107EAC00C0B38040785E20908FFE070500371E001F
:107EBC00780040788040785E20904E31071E0FE8A5
:107ECC001E0078F00F50C4FF365301376E009080BF
:107EDC0000EB508188618188100020000F783900F8
:107EEC00375081806181801E01E98201788301E92C
:107EFC000300338100D10080D3FBFF370000786191
:107F0C0000600040780004E02A00321E0078004037
:107F1C007832C0B38040785E209071F4070004E0A2
:107F2C002200321E00780040788040785E209074E9
:107F3C00FE07E34F501600321E0078004078804058
:107F4C00785E20907CFE071E007800407880407898
:107F5C005E20901031071E00780040788040785EDB
:107F6C0020902231071E007800407832C0B3804048
:107F7C00785E20904BFE070500371E007800407895
:107F8C008040785E20901631071E0FE81E0078F0B6
:107F9C000F50C4FF360F01376E00908000EB5081FC
:107FAC0088618188100020000F783900375081805B
:107FBC006181801E01E90202780402E90300338129
:107FCC0000D10080D3FBFF370000786100600040D7
:107FDC00780004E02A00321E007800407832C0B3EA
:107FEC008040785E20902DF4070004E02200321EC1
:107FFC0000780040788040785E209030FE07E34F98
:10800C00501600321E00780040788040785E209038
:10801C0038FE071E00780040788040785E2090CCB7
:10802C0030071E00780040788040785E2090EA305F
:10803C00071E007800407832C0B38040785E2090F4
:10804C0007FE070500371E00780040788040785EF8
:10805C002090DE30071E0FE81E0078F00F50C4FF92
:10806C0036CB0037000000000000000000C70037CE
:10807C00000000000000000000C3003700000000FA
:10808C000000000000BF00376E00908000EB5081B4
:10809C00886181887E009010407828F0B71000200D
:1080AC00000F785800375081806181801E01E98271
:1080BC0001788301E90300338100D10080D3FBFFF9
:1080CC00370000786100600040780004E04900321D
:1080DC001E007800407822C0B38040785E2090DA91
:1080EC00F3070004E04100321E0078004078804025
:1080FC00785E2090DDFD07E24F501000321E0078B4
:10810C000040788040785E2090E5FD071E007800E6
:10811C0040788040785E20903030071E0078004018
:10812C007822C0B38040785E2090B9FD0728D0BF7C
:10813C000080FBE20F500F0032E30F50180032E1C9
:10814C000F5021003A1E00780040788040785E2065
:10815C00903430071E00780040788040785E209084
:10816C003B30071700371E00780040788040785E5F
:10817C0020904130071E00780040788040785E20C7
:10818C00901830070C00371E00780040788040783B
:10819C005E20901E30071E00780040788040785E8C
:1081AC0020903130070100370000001E0FE81E0040
:1081BC0078F00F50A5FF3659003700000000000082
:1081CC000000005500376E00908000EB50818861F4
:1081DC0081887E009010407828F0B7100020000FA6
:1081EC00784600375081806181801E01E902027857
:1081FC000402E90300338100D10080D3FBFF370078
:10820C0000786100600040780004E03700321E0006
:10821C007800407832C0B38040785E209070F307CD
:10822C000004E02F00321E00780040788040785E19
:10823C00209073FD07E34F501000321E0078004071
:10824C00788040785E20907BFD071E007800407897
:10825C008040785E20900F30071E00780040783206
:10826C00C0B38040785E20904FFD071E0078004020
:10827C00788040785E20901B300728D0BF0080FBB0
:10828C000000E0080032E10F500C003A1E007800AC
:10829C0040788040785E20902830070700371E0019
:1082AC00780040788040785E20902E3007010037AF
:1082BC000000001E0FE81E0078F00F50B7FF3601CB
:1082CC000037000000820B373E48900080FBE40F23
:1082DC0050510032E40F5007003CE20F5045003281
:1082EC00E20F5047003C0000E00A0032F00037E695
:1082FC000F50730032E60F505D0035E70F509A00B7
:10830C0032E80F50E20032E700375E209037FB076F
:10831C00DE209030A82000804010407850180710C4
:10832C000F98DE209030A820008040104078C018B4
:10833C0007200F981E08900040788040785E2090AF
:10834C0046FB071E08904800DE0040788040785EAF
:10835C00209040FB072E08900040788040785E20EB
:10836C00903BFB072E08904800DE00407880407858
:10837C005E209035FB073437070004E00F00322DE8
:10838C003707000F985E2090FDFA078E0890800842
:10839C00785E2090EBFA078E08909000980E08906B
:1083AC003837078E08905E20907CFB07B1003700B1
:1083BC000000000000000000AD00370000000000CD
:1083CC0000000000A90037DE209030A8200080407B
:1083DC00104078CC15077E00900000E81040780023
:1083EC0080FBC800DD7E00901040780080FB808010
:1083FC00405E219030A820000041104078D715072E
:10840C00DE209030A820008040104078A015079006
:10841C0000376E2090100078E40F500F00326E2061
:10842C0090100078E400505E219030A820000041AC
:10843C00104078010178FE0090011907DE20903081
:10844C00A820008040104078AF19077C00375E20D0
:10845C0090CBFA07DE209030A820008040104078A6
:10846C00E41707300F980000EB000F78090037DE97
:10847C00209030A820008040104078AF1907804031
:10848C00785E2090DAFA071E0FE83E08909E00787E
:10849C00808F50F3FF39D436070004E00F0032CD43
:1084AC003607000F985E20909DFA078E0890800882
:1084BC00785E20908BFA078E08909000980E0890AA
:1084CC00D836078E08905E20901CFB075100375E53
:1084DC002090A0FA077E00900000E8104078008001
:1084EC00FBC800DD7E00901040780080FB008040CF
:1084FC00400F98DE209030A820008040104078AFCC
:10850C001707300F98CE08903E0890808F501100BE
:10851C003E0000EB000F78090037DE209030A820D9
:10852C000080401040787619078040785E2090A13A
:10853C00FA071E0FE84E08909E0078808F50F3FFCC
:10854C00391000370000EB000F78090037DE20905F
:10855C0030A8200080401040786519078040785E74
:10856C00209090FA071E0FE83E08909E0078808FAE
:10857C0050F3FF398A36070004E00F0032833607C8
:10858C00000F985E209053FA078E08908008785E52
:10859C00209041FA078E08909000980E08908E3625
:1085AC00078E08905E2090D2FA07070037DE2090E5
:1085BC0030A8200080401040785F1607010037007B
:1085CC000000830A37DE2090B0A8200080401040C5
:1085DC00780E2207E14F5058003A3E48900080FB3D
:1085EC00E20F501B0032E20F5003003CE10F50062B
:1085FC0000324D0037E30F50290032E40F503500A4
:10860C00324800376E209010007800407866425057
:10861C007E00908081E87E00900000E81041787E1A
:10862C000090904078DE2290B0A82000804210404C
:10863C0078E51D073800375E209028FA07DE209079
:10864C00B0A820008040104078D220077E00900017
:10865C0080E89041787E00900000E81041787E0020
:10866C00909040785E2290B0A82000004210407894
:10867C005E1E072300377E00900080E89041787ED4
:10868C0000900000E81041787E00909040785E22C7
:10869C0090B0A820000042104078121E0715003739
:1086AC005E209005FA07DE2090B0A82000804010D4
:1086BC004078A320077E00900000E81041787E00EF
:1086CC0090904078DE2190B0A82000804110407836
:1086DC008241780041EB3C1E07010037000000246A
:1086EC000A37DE2090C0A82000804011C0B301489A
:1086FC00781E0A373E48900080FBE40F50E90032A8
:10870C00E40F5007003CE20F50310032E20F50747E
:10871C00003CE10F500A00327B0137E60F50140188
:10872C0032E60F50110135E70F505C0132E80F5063
:10874C0040780004E0070032DE2090A0A8200080D2
:10875C00401040788040785E20907A2E077E009002
:10876C001040788080FB5E219090A8200000411082
:10877C0040783E3107DE2090A0A8200080401040B9
:10878C00780004E0070032DE2090A0A82000804092
:10879C001040788040785E2090592E075001377E2B
:1087AC000090904078215F985E2090ADF907DE2014
:1087BC0090A0A8200080401040780004E007003210
:1087CC00DE2090A0A8200080401040788040785E89
:1087DC002090522E070000EB000F780C00377E0023
:1087EC00909040785E219090A82000004110407835
:1087FC006C3107305F98BE58905E2090B2F9071E1E
:10880C000FE82E58900080FB9E0F50F0FF3EDE20AC
:10881C0090A0A8200080401040780004E0070032AF
:10882C00DE2090A0A8200080401040788040785E28
:10883C002090262E079F35070004E00F0032983554
:10884C0007000F985E209068F9078E0890800878D2
:10885C005E209056F9078E08909000980E0890A311
:10886C0035078E08905E2090E7F9070B01377E00E4
:10887C00900000E81041787E0090904078DE2190C6
:10888C0090A820008041104078E82F070001376E37
:10889C0000908000EB5081886181885081806181DB
:1088AC0080E00F50E08F5815003A31C0B35E209035
:1088BC0049FB07E44F500A003231C0B35E2090539D
:1088CC00FB0731C0B35E2090200C0742C0B331C00F
:1088DC00B35E20902BFB07DE2090A0A820008040E8
:1088EC008040EB014878450037100020000F783F9E
:1088FC0000375081806181801E01E98201788301FB
:10890C00E90300338100D10080D3FBFF37000078EE
:10891C006100600040780004E03000321E007800F6
:10892C00407832C0B38040785E209016F107000486
:10893C00E02800321E00780040788040785E20905D
:10894C0019FB07E34F501600321E00780040788068
:10895C0040785E209021FB071E0078004078804014
:10896C00785E2090B52D071E007800407880407806
:10897C005E2090BB2D071E007800407832C0B3807B
:10898C0040785E2090F0FA070500371E0078004012
:10899C00788040785E2090AF2D071E00788040785C
:1089AC005E2190A0A8200000410148781E0FE81E0F
:1089BC000078F00F50BEFF369C00376E20901000F0
:1089CC0078E40F503000326E209010007800407820
:1089DC00644050205F98DE2090A0A82000804010BA
:1089EC0040780004E0070032DE2090A0A820008030
:1089FC00401040788040785E20909A2D070000EB64
:108A0C00000F780A00377E00901E004010407880DE
:108A1C0080FB5E219090A8200000411040785A30D5
:108A2C00071E0FE82E58900080FB9E0F50F2FF3E61
:108A3C00DE2090A0A8200080401040780004E007C1
:108A4C000032DE2090A0A8200080401040788040AA
:108A5C00785E2090702D076700376600376E209087
:108A6C00100078E40F504700326E20901000780010
:108A7C004078644050205F985E2090BDF807DE205F
:108A8C0090A0A8200080401040780004E00700323D
:108A9C00DE2090A0A8200080401040788040785EB6
:108AAC002090622D070000EB000F780D00377E0040
:108ABC00901E00409040785E219090A820000041CC
:108ACC001040787B3007305F98BE58905E2090C184
:108ADC00F8071E0FE82E58900080FB9E0F50EFFFFA
:108AEC003EDE2090A0A8200080401040780004E0DA
:108AFC00070032DE2090A0A8200080401040788033
:108B0C0040785E2090352D07AE34070004E00F004E
:108B1C0032A73407000F985E209077F8078E0890E4
:108B2C008008785E209065F8078E08909000980E6B
:108B3C000890B234078E08905E2090F6F8071A0061
:108B4C0037DE209090A820008040104078582F07E6
:108B5C007E00900000E81040780080FBC800DD7EAD
:108B6C0000901040780080FB8080405E219090A89F
:108B7C00200000411040787C2F07DE209090A82028
:108B8C000080401040785E2F0701003700000094F1
:108B9C0008377BF007B0F0070044785E2090ADF00A
:108BAC0007804F548A083A3E48900080FBE20F50F1
:108BBC00140032E20F5003003CE10F50060032412A
:108BCC000037E30F50210032E40F503B00323C00E1
:108BDC00376E2090100090640040104078E14F50A8
:108BEC0002003A8225070100377A25073600376ED6
:108BFC002090100090640040104278445F986E20E2
:108C0C0090100090650040904078515F986E2090D5
:108C1C00100090660040904178635F986E5990DE2A
:108C2C0058904E5890FA24072200375E20902CF86A
:108C3C00076E25078040785E209048F8078040EB4F
:108C4C005E209045F8074434070004E00F00323DE5
:108C5C003407000F985E20900DF8078E089080085E
:108C6C00785E2090FBF7078E08909000980E089085
:108C7C004834078E08905E20908CF8070600375A0F
:108C8C002507040037000000000000000000000071
:108C9C00003E083725F0075AF0070044785E209014
:108CAC0057F007804F5436083A3E48900080FBE45A
:108CBC000F50880032E40F5007003CE20F50500078
:108CCC0032E20F505F003CE10F500800328D00374C
:108CDC00E60F50270032E60F507D0035E70F508528
:108CEC000032860037C029072007985E2090ECF7E9
:108CFC00072E00900040788040785E209007F8079F
:108D0C002E00904800DE0040788040785E20900174
:108D1C00F8070034070004E00F0032F93307000FA6
:108D2C00985E2090C9F7078E08908008785E209096
:108D3C00B7F7078E08909000980E08900434078EB1
:108D4C0008905E209048F8076500378A29072007AD
:108D5C00985E2090CAF7072E0090004078804078EB
:108D6C005E2090E5F7072E00904800DE00407880EA
:108D7C0040785E2090DFF707DE33070004E00F0039
:108D8C0032D73307000F985E2090A7F7078E089014
:108D9C008008785E209095F7078E08909000980ECA
:108DAC000890E233078E08905E209026F807430067
:108DBC00376E20901000906500401040780080FBCA
:108DCC00C800DD6E209010009064004010407800C8
:108DDC0080FB0080403007983E00907F2907712966
:108DEC00073200379429073007985E209097F707D1
:108DFC003E00900040788040785E2090B2F7073EAD
:108E0C0000904800DE0040788040785E2090ACF7FF
:108E1C0007AB33070004E00F0032A43307000F98B0
:108E2C005E209074F7078E08908008785E20906220
:108E3C00F7078E08909000980E0890AF33078E08B5
:108E4C00905E2090F3F7074E29070F00377C290717
:108E5C000D00376E20901000906400401040780098
:108E6C0004E002003A062907010037FD2807030039
:108E7C00373429070100370000009B07373E489024
:108E8C000080FBE10F50030032E20F5083003216DA
:108E9C0001376E02900417987E00900000E8104095
:108EAC00780080FBC800DD7E00901040780080FBCD
:108EBC000080408000EB41EC0710179821179810A8
:108ECC000020000F786C00371E00E98E109000080F
:108EDC00DE6100600040780004E06400321E00781F
:108EEC00004078E2C0B38040785E20902BEF070002
:108EFC0004E02800321E00780040788040785E2024
:108F0C00902EF907EE4F501000321E00780040787A
:108F1C008040785E209036F9071E007800407880FB
:108F2C0040785E2090CA2B071E0078004078E2C083
:108F3C00B38040785E20900AF907020020A34724F2
:108F4C001E1090AE1090ADEB071E01780242780017
:108F5C0001BE8440785E20907424071E0078004087
:108F6C00788040785E20905D23073400371E0078AF
:108F7C00004078D2C0B38040785E2090FBEE0700B2
:108F8C0004E02C00321E00780040788040785E208F
:108F9C0090FEF807ED4F501500321E007800407817
:108FAC008040785E209006F9071E0078004078809B
:108FBC0040785E20909A2B071E0078004078804005
:108FCC00785E20907725071E0078004078D2C0B3D9
:108FDC008040785E2090D5F807020020A347241E1D
:108FEC001090AE109078EB071E01780242780001C9
:108FFC00BE8440785E20903F24071E0078004078A5
:10900C008040785E20900026071E0FE81E0078F046
:10901C000F5091FF36940037EE00900117987E00A8
:10902C00906300401040780080FB8000EBC801DDAD
:10903C000200207E00900080E81040780080FB80C9
:10904C0000EBC000DD0000200201408381487E005F
:10905C00900000E81040780082FB8002EB4828DD8D
:10906C00C820DE8100704820DD0201408381487EEB
:10907C0000901040780080FB8000EB020040838061
:10908C0048301798411798100020000F7868003767
:10909C001E00E98E10900008DE6100600040780030
:1090AC0004E06000321E0078004078E2C0B38040DB
:1090BC00785E209093EE070004E02600321E0078C4
:1090CC000040788040785E209096F807EE4F501064
:1090DC0000321E00780040788040785E20909EF828
:1090EC00071E00780040788040785E2090322B0775
:1090FC001E0078004078E2C0B38040785E20907209
:10910C00F8071E00780040783E1190CE11908040F8
:10911C00785E20901322071E007800407802002011
:10912C0003F0238040785E2090D923073200371E4D
:10913C000078004078D2C0B38040785E209065EE15
:10914C00070004E02A00321E007800407880407846
:10915C005E209068F807ED4F501500321E00780025
:10916C0040788040785E209070F8071E00780040B0
:10917C00788040785E2090042B071E0078004078A1
:10918C008040785E2090E124071E0078004078D261
:10919C00C0B38040785E20903FF8071E00780040F6
:1091AC00783E1190CE11908040785E2090FE23077F
:1091BC001E007800407802002003F0238040785E87
:1091CC002090A623071E0FE81E0078F00F5095FF85
:1091DC00360000007D06373E48900080FBCF80DED5
:1091EC00020120030020820F50838F5883003E0021
:1091FC0006011000378000371200371500371800B1
:10920C00371B00377B00371D00371D00371D00371B
:10921C001D003776003775003774003773003772CE
:10922C0000371800370000000000000000006E003E
:10923C00370000000000000000006A00370000004A
:10924C000000000000006600370000000000000075
:10925C0000006200370000000000000000005E000B
:10926C00375D00375C00375B00375A0037EE0190F2
:10927C00531798100020000F785000371E00E9DEBD
:10928C0010900008DE6100600040780004E04800A7
:10929C00321E007800407812C0B38040785E209077
:1092AC00EFED070004E01F00321E007800407880CC
:1092BC0040785E2090F2F707E14F501100321E000B
:1092CC00780040788040785E2090FAF7071E00788E
:1092DC0000407812C0B38040785E20909E2B071E11
:1092EC00007800407812C0B38040785E2090CDF7B3
:1092FC00071E00780040788040785E20902E2B0767
:10930C002007980200370000EB2007985E2090E1C0
:10931C00F5072E00900040788040785E2090FCF598
:10932C00072E00904800DE0040788040785E209048
:10933C00F6F507F531070004E00F0032EE310700B7
:10934C000F985E2090BEF5078E08908008785E20FE
:10935C0090ACF5078E08909000980E0890F93107A4
:10936C008E08905E20903DF6071E0FE81E0078F0E8
:10937C000F50ADFF36010037000000F005373E48B6
:10938C00900080FBE40F503E0032E40F5007003C8D
:10939C00E20F50140032E20F5022003CE10F500853
:1093AC000032620037E60F50400032E60F505C008E
:1093BC0035E70F503100325B00377E00901040785B
:1093CC000004E0020032632F07010037652F0754B9
:1093DC0000376E209010009065004010407800809F
:1093EC00FBC800DD6E2090100090640040104078A7
:1093FC000080FB0080406017986E1090C82E0744C8
:10940C0000377E00901040780004E0110032672E87
:10941C00077017980000EB000F780700377E10904C
:10942C001E0040FE00909E80409140780148781EBE
:10943C000FE86E20901000786400509E0F50F4FFDF
:10944C003E2E0037252F072C00377E0090104078D9
:10945C000004E00600327E00901042780477980EEB
:10946C0070900080FBC32E072100377E0090000017
:10947C00E81040780080FBC800DD7E00901040783A
:10948C000080FB0080400017987E00906300401025
:10949C0040780080FBC800DD7E00900080E8104022
:1094AC00780080FB0080406017986E1090712E073A
:1094BC000E1090D22E0700000000000000000000EB
:1094CC000000030037122F070100370000007F0552
:1094DC00373E48900080FB6101B90080EB8080EB47
:1094EC00020040838048C20020030020820F50837A
:1094FC008F58D6013E0006010C0037650137680114
:10950C0037930137930137960137990137C50137E6
:10951C00C801370C0137B300373D00377F0037EEF9
:10952C000090111F987E00909041784377987E00B0
:10953C00900000E8104278547798100020000F78C3
:10954C002C00371E00E99E18900008DE61006000B8
:10955C0040780004E02400321E0078004078F2C00D
:10956C00B38040785E209002ED070004E01C0032CE
:10957C001E00780040788040785E209005F707EF59
:10958C004F501500321E00780040788040785E20E5
:10959C00900DF7075E70908084FB1E007800447875
:1095AC005E209056ED078901784E7190884078AE18
:1095BC0014071E0078004078F2C0B38040785E201B
:1095CC0090DCF6071E0FE81E0078F00F50D1FF3626
:1095DC008D0137EE0090111F987E00900000E8106E
:1095EC0040780080FBC800DD7E0090104078008041
:1095FC00FB008040301F987E009063004010407844
:10960C000080FBC800DD7E00900080E810407800F0
:10961C0080FB008040401F98100020000F78250030
:10962C00371E00E99E18900008DE6100600040784B
:10963C000004E01D00321E0078004078F2C0B380B8
:10964C0040785E2090B8EC070004E01500321E0054
:10965C00780040788040785E2090BBF607EF4F5042
:10966C000E003A1E00780044785E209013ED0788B7
:10967C0040784F1407501F985E18900000E00400CB
:10968C00323E1990CE18905E18901E15071E0FE8EA
:10969C001E0078F00F50D8FF364A0137EE019013B8
:1096AC001F987E0090104278447F98100020000F85
:1096BC00782600371E00E99E18900008DE610060D5
:1096CC000040780004E01E00321E0078004078F262
:1096DC00C0B38040785E209087EC070004E0160051
:1096EC00321E00780040788040785E20908AF60721
:1096FC00EF4F500F003A1E00780044785E2090E245
:10970C00EC078840781E1407501F985E18900000D4
:10971C00E00500324E78900080FB8000785E189057
:10972C007615071E0FE81E0078F00F50D7FF36187D
:10973C000137EE0090111F987E009063004010409E
:10974C00780080FB8000EBC801DD0200207E0090D9
:10975C000080E81040780080FB8000EBC000DD004A
:10976C0000200201408381487E00900000E81040F8
:10977C00780082FB8002EB4828DDC820DE81007077
:10978C004820DD0201408381487E00901040780023
:10979C0080FB8000EB020040838048701F980127FB
:1097AC00987E009064004090417823C79810002068
:1097BC00000F782800371E00E99E18900008DE6123
:1097CC0000600040780004E02000321E0078004069
:1097DC0078F2C0B38040785E209031EC070004E052
:1097EC001800321E00780040788040785E2090345B
:1097FC00F607EF4F5011003A1E00780044785E20B7
:10980C00908CEC07884078C81307501F985E18900E
:10981C000000E00700322EC0900080FB7E19908E75
:10982C0021908000785E18909B15071E0FE81E0093
:10983C0078F00F50D5FF36C000376E0290141F9889
:10984C007E00906300401040780080FB8000EBC8E5
:10985C0001DD0200207E00900080E810407800803E
:10986C00FB8000EBC000DD0000200201408381483A
:10987C007E00900000E81040780082FB8002EB48EC
:10988C0028DDC820DE8100704820DD020140838184
:10989C00487E00901040780080FB8000EB02004076
:1098AC00838048701F98012798100020000F78259E
:1098BC0000371E00E99E18900008DE610060004031
:1098CC00780004E01D00321E0078004078F2C0B32E
:1098DC008040785E2090DDEB070004E01500321E1E
:1098EC0000780040788040785E2090E0F507EF4FDC
:1098FC00500E003A1E00780044785E209038EC0739
:10990C00884078741307501F985E18900000E0048C
:10991C0000327E19908E21905E1890D413071E0F82
:10992C00E81E0078F00F50D8FF366F0037000000AB
:10993C000000000000006B0037EE0090111F981023
:10994C000020000F782300371E00E99E18900008B5
:10995C00DE6100600040780004E01B00321E0078DD
:10996C00004078F2C0B38040785E2090ABEB0700EB
:10997C0004E01300321E00780040788040785E20AE
:10998C0090AEF507EF4F500C003A1E00780044786B
:10999C005E209006EC07884078421307501F985EB3
:1099AC0018900000E00200325E18909D13071E0F05
:1099BC00E81E0078F00F50DAFF363F00373E0037D4
:1099CC000000000000000000003A0037000000001A
:1099DC000000000000360037EE0190131F981000B5
:1099EC0020000F782400371E00E99E18900008DE36
:1099FC006100600040780004E01C00321E0078001A
:109A0C004078F2C0B38040785E209076EB0700047B
:109A1C00E01400321E00780040788040785E209080
:109A2C0079F507EF4F500D003A1E00780044785E30
:109A3C002090D1EB078840780D1307501F985E18C3
:109A4C00900000E0030032FE00905E189043150772
:109A5C001E0FE81E0078F00F50D9FF3609003700B2
:109A6C0000000000000000000500370000000000AE
:109A7C00000000000100370000009B03373E4890B7
:109A8C000080FB6101B90080EB8080EB0200408319
:109A9C008048920A20030020820F50838F5886033F
:109AAC003E000601A90037C20037E100371101372B
:109ABC002C01379C0137B70137C80137F001372526
:109ACC0002375B0237860237B20237E702371D03D3
:109ADC00374803377403377303377203377103370F
:109AEC007003376F03376E03376D03376C03376BB7
:109AFC0003376A033769033768033767033766032D
:109B0C003765033764033763033762033761033701
:109B1C006003375F03375E03375D03375C03375BE6
:109B2C0003375A033759033758033757033756034C
:109B3C003755033754033753033752033751033721
:109B4C005003374F03374E03374D03374C03374B16
:109B5C0003374A033749033748033747033746036C
:109B6C003745033744033743033742033741033741
:109B7C004003373F03373E03373D03373C03373B46
:109B8C0003373A033739033738033737033736038C
:109B9C003735033734033733033732033731033761
:109BAC003003372F03372E03372D03372C03372B76
:109BBC0003372A03372903372803372703372603AC
:109BCC003725033724033723033722033721033781
:109BDC002003371F03371E03371D03371C03371BA6
:109BEC0003371A03371903371803371703371603CC
:109BFC0037150337140337130337120337110337A1
:109C0C001003370F03370E03370D03370C03370BD5
:109C1C0003370A03370903370803370703370603EB
:109C2C0037050337040337030337020337010337C0
:109C3C00000337FF0237FE0237FD0237FC0237FB09
:109C4C000237FA0237F90237F80237F70237F60211
:109C5C0037F50237F40237F30237F20237F10237E5
:109C6C00F00237EF0237EE0237ED0237EC0237EB3A
:109C7C000237EA0237E90237E80237E70237E60231
:109C8C0037E50237E40237E30237E20237E1023705
:109C9C00E00237DF0237DE0237DD0237DC023769DC
:109CAC0000375E2090AFF2075E2090FEEA078040FE
:109CBC00785E2090CAF207C92E070004E00F00322C
:109CCC00C22E07000F985E209092F2078E089080AB
:109CDC0008785E209080F2078E08909000980E080D
:109CEC0090CD2E078E08905E209011F307C202379C
:109CFC005E209095F207BE25071040788040785E74
:109D0C002090B0F207B925070000E8104078804099
:109D1C00785E2090AAF207A92E070004E00F00320B
:109D2C00A22E07000F985E209072F2078E0890808A
:109D3C0008785E209060F2078E08909000980E08CC
:109D4C0090AD2E078E08905E2090F1F207A202379C
:109D5C007E00901040780080FB0000408000787EF0
:109D6C0000900000E81040780080FB4800DD008087
:109D7C00402027982E20901002783427985E20904F
:109D8C0066F2073E20900040788040785E209081FB
:109D9C00F2073E20904800DE0040788040785E203C
:109DAC00907BF2077A2E070004E00F0032732E0727
:109DBC00000F985E209043F2078E08908008785E22
:109DCC00209031F2078E08909000980E08907E2E0D
:109DDC00078E08905E2090C2F2077302370000FED7
:109DEC007102377E00901040780080FB00004080AC
:109DFC0000787E00900000E81040780080FB48005E
:109E0C00DD0080402027987E009063004010407851
:109E1C000080FBC800DD7E00900080E810407800D8
:109E2C0080FB0080403027982E2090BE20900108A7
:109E3C00780000FE5502375E209028F207DE209055
:109E4C0080A6200080405001BE4000BE00407880BB
:109E5C0040785E20903FF207DE209080A6200080A4
:109E6C00405001BE4000BE4800DE480ADD000072D2
:109E7C000040788040785E209033F207DE2090809E
:109E8C00A6200080405001BE4000BE01007800407A
:109E9C00788040785E209029F207DE209080A62002
:109EAC000080405001BE4000BE4808DE4812DD0074
:109EBC0000720040788040785E20901DF207DE2012
:109ECC009080A6200080405001BE4000BE02007869
:109EDC000040788040785E209013F207DE2090805E
:109EEC00A6200080405001BE4000BE4810DE481A3B
:109EFC00DD0000720040788040785E209007F20709
:109F0C00DE209080A6200080405001BE4000BE03A1
:109F1C0000780040788040785E2090FDF107DE20CC
:109F2C009080A6200080405001BE4000BE4818DE44
:109F3C000040788040785E2090F3F107DE2090801E
:109F4C00A6200082406000B86011B8009ABE029250
:109F5C00BEEB2D070004E00F0032E42D07000F9834
:109F6C005E2090B4F1078E08908008785E2090A255
:109F7C00F1078E08909000980E0890EF2D078E0830
:109F8C00905E209033F207E401377E00905001BEC2
:109F9C004000BEDE229004A720048242009ABE023A
:109FAC0092BEDE209080A6200080403002BE2003AE
:109FBC00BEDE209000A7200080405001BE4000BEB5
:109FCC00000062818062020163838163DE229084DF
:109FDC00A620048242009ABE0292BEC80137DE203F
:109FEC009000A7200080403002BE2003BE7E00906F
:109FFC005001BE4000BE000072818072020173836A
:10A00C008173DE229004A720048242009ABE029241
:10A01C00BEB60137DE209000A7200080403002BE83
:10A02C002003BE7E00905001BE4000BE0080EA813D
:10A03C0080EA0281EA8381EA000062818062020187
:10A04C0063838163DE229004A720048242009ABEBF
:10A05C000292BEDE209080A6200080403002BE20FE
:10A06C0003BEDE209000A7200080405001BE4000BF
:10A07C00BE000062818062020163838163DE2290F4
:10A08C0084A620048242009ABE0292BE8D01375EE5
:10A09C00209060F107DE209080A720008040100007
:10A0AC00788040786E009000407800C060804078E6
:10A0BC005E209075F107DE209080A72000804090F4
:10A0CC0000786E00900080604800DE004078804090
:10A0DC00785E20906AF107DE209080A720008040F7
:10A0EC009000786E00900080EA8080605E21908005
:10A0FC00A7200000410108785E2D070004E00F0046
:10A10C0032572D07000F985E209027F1078E08908C
:10A11C008008785E209015F1078E08909000980EBC
:10A12C000890622D078E08905E2090A6F1075701CB
:10A13C0037DE2090A0A720008040EE009001087828
:10A14C00100020000F782B00371E00780040780399
:10A15C00E90700CF981E00E9EE00900008DE6100D0
:10A16C00600040780004E01000320EC8900004E05B
:10A17C0008003A1E0078E10F5019003A82C0B38EE5
:10A18C00C8905E209057E80714003782C0B38EC881
:10A19C00905E209052E8070F00370EC8900004E044
:10A1AC0008003A1E0078E10F5009003A82C0B38EC5
:10A1BC00C8905E209071E80704003782C0B38EC847
:10A1CC00905E20906CE8071E0FE81E0078F00F5090
:10A1DC00D2FF36200137DE2090A0A72000804090CF
:10A1EC0000786E00908100705E2190A0A720000086
:10A1FC0041010878100020000F781B00371E0078F2
:10A20C00004078C7E80700CF981E00E9EE009000E8
:10A21C0008DE6100600040780004E00F00320EC8D8
:10A22C00900004E008003A1E0078E10F5009003A53
:10A23C0082C0B38EC8905E20901BE8070400378262
:10A24C00C0B38EC8905E209016E8071E0FE81E0063
:10A25C0078F00F50E2FF36F40037DE2090A0A720F4
:10A26C000080409000786E00900080EA8080605EF4
:10A27C002190A0A720000041010878100020000FB9
:10A28C00781B00371E00780040789AE80700CF98BA
:10A29C001E00E9EE00900008DE61006000407800CE
:10A2AC0004E00F00320EC8900004E008003A1E00D3
:10A2BC0078E10F5009003A82C0B38EC8905E2090AE
:10A2CC0018E80704003782C0B38EC8905E20901344
:10A2DC00E8071E0FE81E0078F00F50E2FF36C700AB
:10A2EC00375E20909AF007DE2090C0A720008040B7
:10A2FC001000788040786E009000407800C060803C
:10A30C0040785E2090AFF007DE2090C0A720008040
:10A31C00409000786E00900080604800DE0040782D
:10A32C008040785E2090A4F007DE2090C0A720002B
:10A33C0080409000786E00900080EA8080605E2102
:10A34C0090C0A720000041010878982C070004E079
:10A35C000F0032912C07000F985E209061F0078E51
:10A36C0008908008785E20904FF0078E089090003F
:10A37C00980E08909C2C078E08905E2090E0F007B9
:10A38C00910037DE2090E0A720008040EE01900382
:10A39C000878100020000F782B00371E0078004042
:10A3AC00783DE80700CF981E00E9EE00900008DE2B
:10A3BC006100600040780004E01000320EC890008C
:10A3CC0004E008003A1E0078E10F5019003AA2C0D0
:10A3DC00B38EC8905E209091E707140037A2C0B3EB
:10A3EC008EC8905E20908CE7070F00370EC8900047
:10A3FC0004E008003A1E0078E10F5009003AA2C0B0
:10A40C00B38EC8905E2090ABE707040037A2C0B3B0
:10A41C008EC8905E2090A6E7071E0FE81E0078F00D
:10A42C000F50D2FF365A0037DE2090E0A720008074
:10A43C00409000786E00908100705E2190E0A72023
:10A44C00000041010878100020000F781B00371E17
:10A45C00007800407801E80700CF981E00E9EE0074
:10A46C00900008DE6100600040780004E00F0032CC
:10A47C000EC8900004E008003A1E0078E10F500965
:10A48C00003AA2C0B38EC8905E209055E707040036
:10A49C0037A2C0B38EC8905E209050E7071E0FE81D
:10A4AC001E0078F00F50E2FF362E0037DE2090E0D1
:10A4BC00A7200080409000786E00900080EA808099
:10A4CC00605E2190E0A72000004101087810002078
:10A4DC00000F781B00371E0078004078D4E7070087
:10A4EC00CF981E00E9EE00900008DE61006000408D
:10A4FC00780004E00F00320EC8900004E008003A27
:10A50C001E0078E10F5009003AA2C0B38EC8905ECD
:10A51C00209052E707040037A2C0B38EC8905E208B
:10A52C00904DE7071E0FE81E0078F00F50E2FF3643
:10A53C00010037000000070037000000050037005D
:10A54C0000000300370000000100370000004F043A
:10A55C00BE0080FA0000061A00FA400F980000EBCB
:10A56C00100798CE089070A620008040104078E12B
:10A57C004F501B003A4E08900FE8074047984E404A
:10A58C00908080FB0068200100703007980000EB81
:10A59C007007983E00908000EB0001EB821F7880E2
:10A5AC0003EB7E01908E09901E0A90AE0A903E0B32
:10A5BC00905F06078F87E9CE089070A62000804038
:10A5CC008040EB0148780040EB004F78AE00371E1E
:10A5DC0081FBCE0890005320000041000040610137
:10A5EC00784207984E00900000E0A300324E08908D
:10A5FC00E7E7074047984E089082EF075007984EC0
:10A60C00089071EF071007985E00904300DE404FF2
:10A61C00985E0090004078674060504F980040EB87
:10A62C00004F784B00371E80FB4300DD9E009000EE
:10A63C0080401040780057981E80FB4300DD0000DE
:10A64C00E89E00900080401040781057981E80FBC8
:10A65C004300DD0080E89E00900080401040782090
:10A66C0057981E80FB4300DD6300409E00900080E5
:10A67C00401040783057981E80FB4300DD6400404A
:10A68C009E00900080401040784057981E80FB43FD
:10A69C0000DD6500409E00900080401040785057CF
:10A6AC00981E80FB4300DD6600409E0090008040B9
:10A6BC001040786057981E80FB4300DD6700409E79
:10A6CC0000900080401040787057984E40908080E9
:10A6DC00FB0048200100703007988000207007981C
:10A6EC003E00908000EB0001EB821F788003EB7E34
:10A6FC0001908E09901E0A90AE0A903E0B90F005C8
:10A70C00078F87E91E4FE84E48909E407880CF50C7
:10A71C00B1FF390040EB004F780D00371E80FBCEA7
:10A72C0048908180FBC308DD0101789E80FB81008D
:10A73C00411E0190810041914078000047015098E2
:10A74C001E4FE85E48909E407880CF50EFFF394E08
:10A75C0040908080FB0048200100703007985E48D4
:10A76C00900080FB7007983E00908000EB0001EB9E
:10A77C00821F788003EB7E01908E09901E0A90AEAA
:10A78C000A903E0B90C305078F87E94E409080805E
:10A79C00FB0078200100703007980000EB700798E0
:10A7AC003E00908000EB0001EB821F788003EB7E73
:10A7BC0001908E09901E0A90AE0A903E0B90B00547
:10A7CC00078F87E9CE00904E08905AF0074E009004
:10A7DC001A2B070400371E4FE81E40780004E04F88
:10A7EC00FF320080FA0000060600FA2007980040AD
:10A7FC00EB004F782000371E81FBAE0090E052201A
:10A80C000000410000406101781207981E00900082
:10A81C0000E01500329E00902E00903EF107AE0035
:10A82C0090C0A8200080401040780004E006003A58
:10A83C009E00902E0090FEEF071E0090F62A070A4D
:10A84C000037AE0090C0A8200080408040EB01484B
:10A85C00780400371E4FE81E40780004E0DDFF321C
:10A86C000080FA0000060600FA1007984147984E3F
:10A87C004090A2E607004F78217C80F00B200081ED
:10A88C006060042071052043F82080497881497864
:10A89C008249789E80FB1E01902003200088B9001D
:10A8AC0000786A00406200780001789E80FB9E016F
:10A8BC00902003200088B900007870004063007875
:10A8CC000000418040EB014878207C800001780238
:10A8DC0060A060042071052043F8208049788149EC
:10A8EC00788249780080FA0000060600FA10079872
:10A8FC00414798CE40901E0090C12207CE40901E3A
:10A90C000090CA22074E409070E607004F78217CD9
:10A91C0080F00B2000816060042071052043F8203A
:10A92C008049788149788249789E009000A820005F
:10A93C0080401001789E009000A8200080401000FC
:10A94C007890007800F02F8081609E80FB1E029032
:10A95C002003200088B9000078720040640078035E
:10A96C000070000978207C800001780260A06004EF
:10A97C002071052043F820804978814978824978F4
:10A98C000080FA0000060600FA1007984147984E1E
:10A99C00409042E607004F78217C80F00B2000812C
:10A9AC006060042071052043F82080497881497843
:10A9BC008249789E009000A8200080401000781EEC
:10A9CC00019001A82081004191007811017801F0DB
:10A9DC002F810061010878207C800001780260A042
:10A9EC0060042071052043F82080497881497882E1
:10A9FC0049780080FA0000060600FA1007984147D3
:10AA0C0098CE40901E0090672207CE40901E00907A
:10AA1C007C22074E409016E607004F78217C80F090
:10AA2C000B2000816060042071052043F8208049D0
:10AA3C00788149788249789E80FB1E019020032002
:10AA4C000088B90000786A00406200780001789EA6
:10AA5C0080FB9E01902003200088B90000787000D4
:10AA6C00406300780000411E019021A82081004124
:10AA7C00914078014878207C800001780260A060C9
:10AA8C00042071052043F820804978814978824957
:10AA9C00780080FA0000060400FA000F782147982D
:10AAAC00AE40901E00783FFF070080FA00000606BB
:10AABC0000FA100798414798CE40901E00902A2229
:10AACC0007CE40901E00903322074E4090D9E507E8
:10AADC00004F78217C80F00B200081606004207195
:10AAEC00052043F8208049788149788249789E0076
:10AAFC009040A8200080401001789E009040A82033
:10AB0C0000804010007890007800F02F8081609ECB
:10AB1C0080FB1E02902003200088B9000078720090
:10AB2C0040640078030070000978207C8000017874
:10AB3C000260A060042071052043F82080497881D0
:10AB4C0049788249780080FA0000060600FA10075E
:10AB5C00984147984E4090ABE507004F78217C8098
:10AB6C00F00B2000816060042071052043F82080E8
:10AB7C0049788149788249789E009040A8200080CD
:10AB8C00401000781E019041A8208100419100786E
:10AB9C0011017801F02F810061010878207C800080
:10ABAC0001780260A060042071052043F8208049E0
:10ABBC00788149788249780080FA0000060600FA0C
:10ABCC00100798414798CE40901E0090D02107CE98
:10ABDC0040901E0090E521074E40907FE507004F06
:10ABEC0078217C80F00B20008160600420710520AE
:10ABFC0043F8208049788149788249789E80FB1EF1
:10AC0C0001902003200088B90000786A004062009F
:10AC1C00780001789E80FB9E01902003200088B96B
:10AC2C000000787000406300780000411E019081A4
:10AC3C00A820810041914078014878207C80000157
:10AC4C00780260A060042071052043F820804978C8
:10AC5C008149788249780080FA0000060400FA00E5
:10AC6C000F78214798AE40901E0078A8FE07008010
:10AC7C00FA0000060600FA100798414798CE40905B
:10AC8C001E0090932107CE40901E0090A821074EE5
:10AC9C00409042E507004F78217C80F00B2000812A
:10ACAC006060042071052043F82080497881497840
:10ACBC008249789E80FB1E01902003200088B900F9
:10ACCC0000786A00406200780001789E80FB9E014B
:10ACDC00902003200088B900007870004063007851
:10ACEC000000411E019071A8208100419140780123
:10ACFC004878207C800001780260A06004207105F7
:10AD0C002043F8208049788149788249780080FA7C
:10AD1C000000060400FA000F78214798AE40901E00
:10AD2C0000786BFE070080FA0000060600FA100798
:10AD3C0098414798CE40901E0090562107CE4090E7
:10AD4C001E00906B2107CE40901E0090C821074E2C
:10AD5C00409002E507004F78217C80F00B200081A9
:10AD6C006060042071052043F8208049788149787F
:10AD7C008249789E80FB1E01902003200088B90038
:10AD8C0000786A00406200780001789E80FB9E018A
:10AD9C00902003200088B900007870004063007890
:10ADAC000000411E019061A8208100419140780172
:10ADBC004878207C800001780260A0600420710536
:10ADCC002043F8208049788149788249780080FABC
:10ADDC000000060400FA000F78214798AE40901E40
:10ADEC0000782BFE070080FA0000060400FA000F22
:10ADFC0078214798AE40901E0078162107AE4090FF
:10AE0C001E00782B21079E0078B0A82000804010EF
:10AE1C004078D811070080FA0000060200FA000FF3
:10AE2C00789E0078B0A8200080401040780112076E
:10AE3C000080FA0000060400FA000F78214798AE53
:10AE4C0040901E0078FD2007AE40901E0078122125
:10AE5C00079E0078B0A820008040104078BF1107F2
:10AE6C000080FA0000060200FA000F789E0078B00D
:10AE7C00A820008040104078E811070080FA0000FC
:10AE8C00060400FA000F782147980080FA000006AB
:10AE9C000400FA000F782147980080FA000006049D
:10AEAC0000FA000F78214798E2C0B3AE40901E0024
:10AEBC007894E4070004E0040032AE40901E007861
:10AECC00A61807030037AE40901E0078D91B070068
:10AEDC0080FA0000060800FA300798BE0090B0A86F
:10AEEC00200080401040786814071007981E0090CE
:10AEFC007040900080FBE20F50070032E20F50636D
:10AF0C000034E30F502A0032E40F502C00325F0063
:10AF1C00371E00901040900004E00F003A1E009085
:10AF2C00B041901E00906801401E00909040783E09
:10AF3C000290B0A820000042104078EA12071E00D0
:10AF4C009031C0B37140984C00371E00908040EB9C
:10AF5C004140981E00903042901E0090E801401E27
:10AF6C0000902041901E0090904078BE0290B0A8B6
:10AF7C00200080421040782413071E009031C0B38B
:10AF8C007140983800371E009041C0B3714098341E
:10AF9C0000371E0090104090E14F5024003A3E00C4
:10AFAC00905BEC070040EB004F780900371E0090D7
:10AFBC00E800401E80FB0080401040788040783EC6
:10AFCC00009070EC071E4FE81E00904040909E4F82
:10AFDC0050F3FF3E6A28070004E00F003263280795
:10AFEC002007983E009033EC07AE00908008783E26
:10AFFC00009021EC07AE00909000982E00906E28E7
:10B00C0007AE00903E0090B2EC071E00908040EB23
:10B01C003140981E00908040EB4140981E009011EA
:10B02C00C0B37140980000000100370000000080A0
:10B03C00FA0000060400FA20479843E407000F7852
:10B04C009E007830A8200080409040782E40908060
:10B05C00CF5002003A1E007817003730E407000F7B
:10B06C00789E007830A8200080409040782E409048
:10B07C0080CF5002003A1E00780C003729E40700FC
:10B08C000F789E007830A8200080409040782E40A9
:10B09C009080CF5002003A1E00780100370000EB80
:10B0AC000080FA0000060800FA2007986147981CF7
:10B0BC00E4071007980040EB004F781800379E808B
:10B0CC00FB1E01902003200088B90000786E004020
:10B0DC00E200786E40900080FB808F500C003A9E0E
:10B0EC0080FB1E01902003200088B90000786200CC
:10B0FC0078E400402E0090808F5002003A1E0090A1
:10B10C004500371E4FE81E4078EB4F50E5FF36F4F4
:10B11C00E3071007980040EB004F781800379E802B
:10B12C00FB1E01902003200088B90000786E0040BF
:10B13C00E200786E40900080FB808F500C003A9EAD
:10B14C0080FB1E01902003200088B900007862006B
:10B15C0078E400402E0090808F5002003A1E009040
:10B16C002500371E4FE81E4078EB4F50E5FF36D8D0
:10B17C00E3071007980040EB004F781800379E80CB
:10B18C00FB1E01902003200088B90000786E00405F
:10B19C00E200786E40900080FB808F500C003A9E4D
:10B1AC0080FB1E01902003200088B900007862000B
:10B1BC0078E400402E0090808F5002003A1E0090E0
:10B1CC000500371E4FE81E4078EB4F50E5FF360068
:10B1DC0000EB0080FA0000060800FA20079861478F
:10B1EC0098B6E3071007980040EB004F781A003729
:10B1FC009E80FB1E01902003200088B90000786E11
:10B20C000040E200786E40900080FB808F500E0072
:10B21C003A9E80FB1E01902003200088B900007824
:10B22C00620078E400402E0090808F5004003A1E9B
:10B23C0080FBF18A266140784900371E4FE81E409A
:10B24C0078EB4F50E3FF368CE3071007980040EB88
:10B25C00004F781A00379E80FB1E019020032000BF
:10B26C0088B90000786E0040E200786E4090008053
:10B27C00FB808F500E003A9E80FB1E019020032015
:10B28C000088B9000078620078E400402E009080BD
:10B29C008F5004003A1E80FBF18A2661407827000B
:10B2AC00371E4FE81E4078EB4F50E3FF366EE30736
:10B2BC001007980040EB004F781A00379E80FB1E59
:10B2CC0001902003200088B90000786E0040E20055
:10B2DC00786E40900080FB808F500E003A9E80FB71
:10B2EC001E01902003200088B9000078620078E4E9
:10B2FC0000402E0090808F5004003A1E80FBF18A93
:10B30C00266140780500371E4FE81E4078EB4F5001
:10B31C00E3FF360040EB0080FA0000060000FA5B09
:10B32C008EA90080FA0000060400FA80352410076C
:10B33C00984201208000EB80352449E2071200205E
:10B34C008000EBE01A2145E2071200208000EBF0B0
:10B35C001A2141E207B071EFB171EF0040EB004FE1
:10B36C00780600371E00907C00071E009074004089
:10B37C001007981E4FE81E40780004E0F7FF3D00D0
:10B38C0080FA0000060000FA508D800080FA000060
:10B39C00060400FA1007980040EB004F781E80FB63
:10B3AC00800040201A210080401000780000E00A44
:10B3BC00003A1E80FB800040201A210080409E0035
:10B3CC00900108781E00908000EB0108980E003761
:10B3DC001E80FB800040401A210080401000789EA7
:10B3EC0000901108981E80FB800040401A210080BC
:10B3FC00409000781E00900108981E80FB80004051
:10B40C00401A210080409E00900108781E00908018
:10B41C0000EB1108981E80FBE11A2181004091403D
:10B42C00788140E8E21A210200400148780080FA55
:10B43C000000060400FA1007980040EB004F781E3D
:10B44C0080FB800040601A210080401000780000D2
:10B45C00E00A003A1E80FB800040601A2100804008
:10B46C009E00900108781E00908000EB0108980E59
:10B47C0000371E80FB800040801A210080401000A5
:10B48C00789E00901108981E80FB800040801A2145
:10B49C000080409000781E00900108981E80FB8070
:10B4AC000040801A210080409E00900108781E0008
:10B4BC00908000EB1108981E80FBF11A218100404E
:10B4CC009140788140E8F21A21020040014878B09E
:10B4DC00D1BF0040E8B0F1B70080FA0000060200CE
:10B4EC00FA000F784201208000EB1E0078B8E107CB
:10B4FC00508D800000E006003A9E0078518D881E29
:10B50C0000788000EB010898060037608D809E0063
:10B51C0078110898618D801E00780108989E00783B
:10B52C00618D881E00788000EB110898B1D1BF00A6
:10B53C0040E8B1F1B70080FA0000060600FA1007E7
:10B54C00982107980040EB004F782E0090900890BF
:10B55C001E00901108981E0090AE00900108982EC5
:10B56C0000901008900000E00500322E00901008AA
:10B57C00909E00900108980600371E80FB800040CA
:10B58C00401A210080409E00900108782E00909E69
:10B59C0000901108981E80FBE11A21810040914017
:10B5AC00788140E8E21A210200400148780080FAD4
:10B5BC000000060600FA1007982107980040EB00DF
:10B5CC004F782E00909008901E00901108981E0045
:10B5DC0090AE00900108982E00901008900000E0AA
:10B5EC000500322E00901008909E009001089806DD
:10B5FC0000371E80FB800040801A210080409E0096
:10B60C00900108782E00909E00901108981E80FBE7
:10B61C00F11A218100409140788140E8F21A210210
:10B62C000040014878B0D1BF0040E8B0F1B70080CD
:10B63C00FA0000060400FA000F7811079822002087
:10B64C008000EB1E007845E1071E00909008901ECC
:10B65C0000781108981E00789E00900108981E0032
:10B66C00901008900000E00500321E009010089029
:10B67C009E00780108980200379E0078618D881E24
:10B68C0000909E0078110898B1D1BF0040E8B1F14C
:10B69C00B70080FA0000060400FA1007980040EB8F
:10B6AC00004F781E00900008900000E008003A1E41
:10B6BC0080FB9E0090910890000140201A21000010
:10B6CC00410108780500371E00900008909E0090FC
:10B6DC009108901108981E00901008900000E00846
:10B6EC00003A1E80FB9E0090810890000140401A99
:10B6FC00210000410108780500371E0090100890C9
:10B70C009E00908108900108981E80FBE11A21810F
:10B71C0000409140788140E9E21A21020040014842
:10B72C00780080FA0000060400FA1007980040EB3D
:10B73C00004F781E80FB800040601A2100804090F2
:10B74C0000781E80FB000140801A2100004110008F
:10B75C0078808F5020003A1E80FB800040601A21B8
:10B76C000080409000781E0090808F5018003A1E88
:10B77C0080FB800040601A210080408000EB0108B3
:10B78C00781E80FB800040801A210080408000EBF6
:10B79C000108781E80FBF11A2181004091407881CC
:10B7AC0040E9F21A21020040014878B0D1BF0040B4
:10B7BC00E9B0F1B72D00371E00900008900000E0B2
:10B7CC0008003A1E80FB9E0090910890000140609A
:10B7DC001A210000410108780500371E009000086E
:10B7EC00909E00909108901108981E00901008905F
:10B7FC000000E008003A1E80FB9E0090810890003B
:10B80C000140801A210000410108780500371E0014
:10B81C00901008909E00908108900108981E80FB63
:10B82C00F11A218100409140788140E9F21A2102FD
:10B83C000040014878B0D1BF0040E9B0F1B70080BA
:10B84C00FA0000060200FA000F781E00780008903B
:10B85C000000E004003A1E0078100890508D880516
:10B86C0000371E00780008909E007891089011080F
:10B87C00981E00781008900000E004003A1E007832
:10B88C00000890608D880500371E00781008909E87
:10B89C000078810890010898B1D1BF0040E9B1F15E
:10B8AC00B70080FA0000060200FA000F78B1D1BF91
:10B8BC000004E00600321E0078D8FF071E00784511
:10B8CC00FE0710C0B30100370040EB0080FA000007
:10B8DC00061200FA10079821079832079843079828
:10B8EC00540798650798760798070F98B1D1BF0051
:10B8FC0004E02400322FFE07000F78CE00901E00CB
:10B90C0078410098DE00901E0078510098EE00906F
:10B91C001E0078610098FE00901E00787100983E21
:10B92C0000908040781E00784140981E00781E01DF
:10B93C0090AE01900288BE0E08908040781E007870
:10B94C006140984EB8978040781E00785140981E00
:10B95C000078A5FF071E007848FE0710C0B3010051
:10B96C00370040EB0080FA0000060800FA0000EBFC
:10B97C00000F780000EB100798B1D1BF0004E081F4
:10B98C000032203180200798FEFD073007982E00EA
:10B99C009020009044800A0000000080FB000F788B
:10B9AC002E009020009055800A0000000080FB10B3
:10B9BC0007981E00780000E00B003A2E0090100053
:10B9CC0078A0800A0000008000EB3E01900089BE48
:10B9DC003E00908040EB6140981A00372E0090108A
:10B9EC000078A0800A0000008000EBC202DD040099
:10B9FC00202E0190920178CB19DE920390F67F20D5
:10BA0C000683634533DD868171030078120190CB88
:10BA1C00810A0200000400408580483E01900089A4
:10BA2C00BE3E009011C0B36140981E0090E10F50D3
:10BA3C0004003A3E009011C0B35140984000373E8C
:10BA4C0000908040EB5140983E00901001BE404069
:10BA5C0020010020800F51818F5905003A00000011
:10BA6C000000000000000000000000002E009068A4
:10BA7C0000409040783E00900148982E009069005C
:10BA8C00409040783E00901148982E00906A0040FB
:10BA9C009040783E00902148982E00906B0040908A
:10BAAC0040783E00903148982E00906C00409040B9
:10BABC00783E00904148982E00906D004090407860
:10BACC003E00905148982E00906E00409040783E79
:10BADC0000906148982E00906F00409040783E0096
:10BAEC00907148982E009020009030800A00000041
:10BAFC008040783E00904140983E009038FF0710FF
:10BB0C00C0B30100370040EB0080FA0000060400CF
:10BB1C00FA000F781107981E00901000BE1E0178D5
:10BB2C000089BE1E0090E040901E00786140981E77
:10BB3C000090D040901E00785140981E0090C0405C
:10BB4C00901E00784140981E00908048901E00780E
:10BB5C000148981E00909048901E00781148981E3D
:10BB6C000090A048901E00782148981E0090B04884
:10BB7C00901E00783148981E0090C048901E0078A6
:10BB8C004148981E0090D048901E00785148981E4D
:10BB9C000090E048901E00786148981E0090F04894
:10BBAC00901E00787148980080FA0000060C00FA8C
:10BBBC005007985E00904000901007985E009050DF
:10BBCC0000902007985E00906000903007985E000F
:10BBDC00907000904007985E00904040900080FB71
:10BBEC00000F785E00905040908081FB5E0090606A
:10BC0C00780E01788220070080FA0000060400FA02
:10BC1C000040EB004F781100371E80FB8000402065
:10BC2C001A210080409000781107981E00900000A7
:10BC3C00E00700321E00900B00071E00901DFE074F
:10BC4C001E009088FD070400371E4FE81E40780048
:10BC5C0004E0ECFF320080FA0000061600FA881FA0
:10BC6C0078200F980000EB000F78AE089021079811
:10BC7C002E00901000BEC08C88D18C88C08C80D1D6
:10BC8C008C800040780074A19CF1B7C08C80D18C62
:10BC9C00804909DD4700DE000071C708DE004078EE
:10BCAC006140609DF1B7C08C80D18C800040789F42
:10BCBC00F1B7C08C80D18C804809DD4800DE0000D3
:10BCCC0071C808DE004078A0F1B7A0D1BF67406012
:10BCDC00A1F1B7C08C80D18C804809DD4800DE0012
:10BCEC000071C808DE0040786740609EF1B7F61B13
:10BCFC0007C11921914078814F500D0032DF1B078D
:10BD0C00C11921914078814F50080032E31B07C1C3
:10BD1C001921914078814F50030032F01B07E14FFD
:10BD2C005066013A9DD1BF0004E02A013A9ED1BF72
:10BD3C000080FBE20F504E0132E20F5005003C0038
:10BD4C0000E00A0032E10F50200032580137E40FB6
:10BD5C00508A0032E40F50330035E70F50D10032D7
:10BD6C00510137CF1B07C11921914078814F5003E6
:10BD7C00003ADBDF07B6E707490137B51B07C119E6
:10BD8C0021914078814F5003003ACBDF07AEE70793
:10BD9C00410137B61B07C11921914078814F502DB5
:10BDAC00013AC7DF07A6E707390137B71B07C119E7
:10BDBC0021914078814F5003003AC3DF07A7E70772
:10BDCC003101379D1B07C11921914078814F5003D8
:10BDDC00003AB3DF079FE7072901379E1B07C119FC
:10BDEC0021914078814F5017013AAFDF0797E70751
:10BDFC002101379F1B07C11921914078814F5004B5
:10BE0C00003AABDF077EE707000F78110037841B81
:10BE1C0007C11921914078814F5004003A9ADF07ED
:10BE2C0075E707000F78080037841B07C1192191AB
:10BE3C004078814F5003003A95DF076CE707000FFD
:10BE4C00789CD1BF0074A00080FB3007980000EBF9
:10BE5C005007983E00908000EB0001EB821F788029
:10BE6C0003EB5E0190EE01907E02908E0A901E0B09
:10BE7C00901FFE078F87E99E00786107989CD1BFC1
:10BE8C008080FB0048200100703007982000205073
:10BE9C0007983E00908000EB0001EB821F78800336
:10BEAC00EB5E0190EE01907E02908E0A901E0B903C
:10BEBC000AFE078F87E99CD1BF8080FB00782001A8
:10BECC0000703007980000EB5007983E00908000FF
:10BEDC00EB0001EB821F788003EB5E0190EE01908A
:10BEEC007E02908E0A901E0B90F7FD078F87E9CC8F
:10BEFC0000374A1B07C11921914078814F5014001B
:10BF0C003A0000EB1007980A0037AE00901E009024
:10BF1C006800406144784FDF078840783BE7071E94
:10BF2C0000900000E81007982E0090404090808010
:10BF3C00FB1E0090808F50F0FF3EB300371F1B0795
:10BF4C00C11921914078814F5014003A0000EB1038
:10BF5C0007980A0037AE00901E00906800406144BC
:10BF6C00782EDF0788407822E7071E00900000E853
:10BF7C001007982E00904040908080FB1E0090800F
:10BF8C008F50F0FF3E9A00370F1B07C119219140CB
:10BF9C0078814F508A003A0000EB1007980A00375E
:10BFAC00AE00901E009068004061447819DF07884D
:10BFBC00407809E7071E00900000E81007982E0053
:10BFCC00904040908080FB1E0090808F50F0FF3E90
:10BFDC00810037FF1A07C11921914078814F501306
:10BFEC00003A1023070004E07000320923074007D1
:10BFFC009806DF07D1E607CE009080087802DF07AD
:10C00C00C1E607CE00909000984E0090142307FCD8
:10C01C00DE07CE009017E707690037D51A07C1195C
:10C02C0021914078814F5013003AF822070004E028
:10C03C005A0032F12207400798E6DE07B9E607CE30
:10C04C000090800878E2DE07A9E607CE0090900009
:10C05C00984E0090FC2207DCDE07CE0090FFE6072E
:10C06C00510037C61A07C11921914078814F5047AA
:10C07C00003AE022070004E0460032D922074007CC
:10C08C0098D2DE07A1E607CE0090800878CEDE07B6
:10C09C0091E607CE00909000984E0090E42207C8DD
:10C0AC00DE07CE0090E7E607390037C01A07E14FEC
:10C0BC005036003A9ED1BF0080FBE40F500700328F
:10C0CC00E40F502F0034E60F50180032E70F5013D6
:10C0DC0000322B00370000EB100798080037AE0039
:10C0EC00901E00906800406140789A0E071E0090E8
:10C0FC000000E81007982E00904040908080FB1EB6
:10C10C000090808F50F2FF3E190037870E077A227D
:10C11C00071600379CD1BF960E076A1B070000005C
:10C12C001100370000000F00370000000D00370031
:10C13C0000000B003700000009003700000007006A
:10C14C003700000005003700000003003700000036
:10C15C000100370000004F04780080FA0000060050
:10C16C0000FA281F07461F073BFB070080FA000058
:10C17C00060000FA0031806100600000E00C003223
:10C18C004DFD070004E0040032100020B08C881D27
:10C19C0006A80500370000000000000000000000A9
:10C1AC00000000000031806100600000E00C0032F3
:10C1BC003DFD070004E0040032100020B08C881D07
:10C1CC0006A8050037000000000000000000000079
:10C1DC00000000000031806100600000E00C0032C3
:10C1EC002DFD070004E0040032100020B08C881DE7
:10C1FC0006A8050037000000000000000000000049
:10C20C00000000000031806100600000E00C003292
:10C21C001DFD070004E0040032100020B08C881DC6
:10C22C0006A8050037000000000000000000000018
:10C23C00000000000080FA0000060600FAD41E0779
:10C24C000004E07E003A0040EB004F787800371E87
:10C25C0080FB800040601A2100804090007811071C
:10C26C00981E00900000E06E00322B1A07E24F502F
:10C27C0003003A1E0090BCFD076300371E009010AF
:10C28C0001BEF00720010020020278030178800132
:10C29C00780100780302620000618000EBC000DDD1
:10C2AC000000200001BE6120B8000171818171E0A5
:10C2BC000F51E08F590B003AB1D1BF0004E04C0094
:10C2CC0032EBFA072007989E00902E00906AFD072B
:10C2DC002E00909BFC074400371E00901001BEF00E
:10C2EC000720010020020278030178800178010008
:10C2FC00780302620000618000EBC000DD000020CA
:10C30C000001BE6120B80001718181711000200113
:10C31C000020800F51818F590B003AB1D1BF00041E
:10C32C00E02B0032CAFA072007989E00902E00904E
:10C33C0049FD072E00907AFC072300371E00901051
:10C34C0001BEF00720010020020278030178800171
:10C35C00780100780302620000618000EBC000DD10
:10C36C000000200001BE6120B800017181817120A4
:10C37C000020010020800F51818F590B003AB1D160
:10C38C00BF0004E00A0032A9FA072007989E00902B
:10C39C002E009028FD072E009059FC070200371E36
:10C3AC00009058FD071E0090D4FB071E00900FFB59
:10C3BC00070400371E4FE81E40780004E085FF326A
:10C3CC000080FA0000060400FA2047982E409000E6
:10C3DC0080FBE20F50070032E30F50080032E10FF0
:10C3EC005009003A802320000F78060037002620E1
:10C3FC00000F7803003700F020000F780000001EBB
:10C40C00007890007801F0A10108781E0078304087
:10C41C000A1000001E007890007801D0A101087865
:10C42C001E007890007801C0A10108781E00789059
:10C43C0000780160A10108789E007831409021407D
:10C44C000A000000B040981E007890009001B0A047
:10C45C001100981E0078B115204100989E0078219B
:10C46C00409054400A000000A040981E00789000B4
:10C47C00900120A11100989E007871409064400AB0
:10C48C00000000F040989E007871409020400A0017
:10C49C000000F040982E4090F800072E40900701C5
:10C4AC00072E40901601072E40902501072E409034
:10C4BC007000072E40907F00072E4090B000072E92
:10C4CC004090BF00071E007890007801F0A0010892
:10C4DC00781E00789000780150A00108781E007832
:10C4EC009000780140A00108780080FA0000060452
:10C4FC0000FA2047982E40900080FBE20F50070076
:10C50C0032E30F50080032E10F5009003A8023202B
:10C51C00000F78060037002620000F780300370044
:10C52C00F020000F780000001E007890007801F0D9
:10C53C00A00108780080FA0000060400FA20479851
:10C54C002E40900080FBE20F50070032E30F5008A2
:10C55C000032E10F5009003A802320000F780600CA
:10C56C0037002620000F7803003700F020000F78EA
:10C57C000000001E007890007801F0A101087800FE
:10C58C0080FA0000060600FA2047982107982E40F2
:10C59C00900080FBE20F50070032E30F500800328E
:10C5AC00E10F5009003A802320000F780600370075
:10C5BC002620000F7803003700F020000F780000D1
:10C5CC00001E0078AE00904100980080FA00000632
:10C5DC000200FA004F781E80FBE20F50060032E397
:10C5EC000F50060032E10F5006003A0188A80400F3
:10C5FC00370388A80200370748A80000000080FA1B
:10C60C000000060200FA004F781E80FBE20F500675
:10C61C000032E30F50060032E10F5006003A018859
:10C62C00A90400370388A90200370748A9000000B5
:10C63C000080FA0000060200FA004F781E80FBE230
:10C64C000F50060032E30F50060032E10F50060087
:10C65C003A2188A80400372388A80200372748A865
:10C66C000000000080FA0000060200FA004F781E5D
:10C67C0080FBE20F50060032E30F50060032E10F50
:10C68C005006003A2188A90400372388A9020037F4
:10C69C002748A90000000080FA0000060200FA00FA
:10C6AC004F781E80FBE20F50060032E30F5006005D
:10C6BC0032E10F5006003A0168A80400370368A85D
:10C6CC000200370728A80000000080FA00000602CC
:10C6DC0000FA004F781E80FBE20F50060032E30F89
:10C6EC0050060032E10F5006003A0168A9040037E9
:10C6FC000368A90200370728A90000000080FA008F
:10C70C0000060200FA004F781E80FBE20F50090071
:10C71C0032E30F500C0032E10F500F003A2168A8A1
:10C72C00510020EC210A4408000A00372368A85164
:10C73C000020EC210A4C08000500372728A85100DE
:10C74C002064210A5C08000000000080FA0000064A
:10C75C000200FA004F781E80FBE20F50060032E315
:10C76C000F50060032E10F5006003A2168A9040070
:10C77C00372368A90200372728A90000000080FA97
:10C78C000000060200FA004F781E80FBE20F5006F4
:10C79C000032E30F50060032E10F5006003A003031
:10C7AC00EF0400370C30EF0200371830EF000000B8
:10C7BC000080FA0000060200FA004F781E80FBE2AF
:10C7CC000F50060032E30F50060032E10F50060006
:10C7DC003A0230EF0400370E30EF0200371A30EF18
:10C7EC000000000080FA0000060200FA004F781EDC
:10C7FC0080FBE20F50060032E30F50060032E10FCF
:10C80C005006003A0830EF0400371430EF020037BE
:10C81C002030EF0000000080FA0000060200FA0051
:10C82C004F781E80FBE20F50060032E30F500600DB
:10C83C0032E10F5006003A0A30EF0400371630EFA1
:10C84C000200372230EF0000000080FA00000602E0
:10C85C0000FA004F781147981E80FBE20F500F0032
:10C86C0032E30F50180032E10F5021003AF01180E2
:10C87C007000600000E00200320040EB1C00371E2C
:10C88C0040900080FB40128810C0B3170037301363
:10C89C00807000600000E00200320040EB110037B5
:10C8AC001E40900080FB80138810C0B30C00373002
:10C8BC0078807000600000E00200320040EB06005F
:10C8CC00371E40900080FB80788810C0B301003781
:10C8DC000040EB0080FA0000060200FA004F781EC0
:10C8EC0080FBE20F50110032E30F501C0032E10FBD
:10C8FC005027003A0141800080200080600000E059
:10C90C000500322168A90080801080882168A81D4C
:10C91C0000370080801080881A0037114180008019
:10C92C00200080600000E00500322368A960808050
:10C93C007080882368A81000376080807080880D14
:10C94C0000373141800020200080600000E00500AD
:10C95C00322728A9C08080D080882728A8030037D8
:10C96C00C08080D080880000000080FA00000602A1
:10C97C0000FA004F781E80FBE20F50110032E30FDB
:10C98C00501C0032E10F5027003A01418000002179
:10C99C000080600000E00500322188A940808050B2
:10C9AC0080882188A81D00374080805080881A001C
:10C9BC00371141800000210080600000E00500324A
:10C9CC002388A9A08080B080882388A8100037A075
:10C9DC008080B080880D003731418000402000807D
:10C9EC00600000E00500322748A900818010818892
:10C9FC002748A803003700818010818800000000C0
:10CA0C0080FA0000060400FA2047982E409000801F
:10CA1C00FBE20F50110032E30F501C0032E10F50BB
:10CA2C0027003A0141800080200080600000E00572
:10CA3C0000322168A9108080000F782168A81D00A1
:10CA4C0037108080000F781A003711418000802049
:10CA5C000080600000E00500322368A9708080002F
:10CA6C000F782368A8100037708080000F780D00B5
:10CA7C00373141800020200080600000E00500324A
:10CA8C002728A9D08080000F782728A8030037D04A
:10CA9C008080000F780000001E00780080FA0000F3
:10CAAC00060400FA2047982E40900080FBE20F50BD
:10CABC00110032E30F501C0032E10F5027003A01F5
:10CACC0041800000210080600000E00500322188D8
:10CADC00A9508080000F782188A81D0037508080D5
:10CAEC00000F781A0037114180000021008060008F
:10CAFC0000E00500322388A9B08080000F782388DD
:10CB0C00A8100037B08080000F780D0037314180BD
:10CB1C000040200080600000E00500322748A9108A
:10CB2C008180000F782748A8030037108180000F00
:10CB3C00780000001E00780080FA0000060200FA5F
:10CB4C00004F781E80FBE20F50110032E30F501C97
:10CB5C000032E10F5027003A014180008020008014
:10CB6C00600000E00500322168A9008080108088F8
:10CB7C002168A81D00370080801080881A003711AA
:10CB8C0041800080200080600000E00500322368B6
:10CB9C00A96080807080882368A81000376080802E
:10CBAC007080880D003731418000202000806000AB
:10CBBC0000E00500322728A9C08080D08088272873
:10CBCC00A8030037C08080D080880000000080FA65
:10CBDC000000060200FA004F781E80FBE20F50079F
:10CBEC000032E30F50080032E10F5009003A408048
:10CBFC0080508088060037A08080B0808803003782
:10CC0C000081801081880000000080FA000006047A
:10CC1C0000FA2047982E40900080FBE20F5027002E
:10CC2C0032E30F50480032E10F5069003A01418065
:10CC3C000080200080600000E01000322168A91103
:10CC4C008080008080808F5004003E0180801080A6
:10CC5C0080008F50050037018080108080808050CC
:10CC6C00008020008F402168A8540037118080007C
:10CC7C008080808F5004003E018080108080008F67
:10CC8C00504C0037018080108080808050008020C4
:10CC9C00008F4046003711418000802000806000EA
:10CCAC0000E01000322368A9718080608080808F42
:10CCBC005004003E618080708080008F50050037EA
:10CCCC00618080708080808050004020008F4023E5
:10CCDC0068A8310037718080608080808F5004009C
:10CCEC003E618080708080008F5029003761808089
:10CCFC00708080808050004020008F4023003731AE
:10CD0C0041800020200080600000E01000322728C5
:10CD1C00A9D18080C08080808F5004003EC180806B
:10CD2C00D08080008F50050037C18080D0808080FB
:10CD3C008050004020008F402728A80E0037D1805B
:10CD4C0080C08080808F5004003EC18080D0808065
:10CD5C00008F50060037C18080D0808080805000CA
:10CD6C004020008F400000001E00780080FA000078
:10CD7C00060400FA2047982E40900080FBE20F50EA
:10CD8C00270032E30F50480032E10F5069003A019E
:10CD9C0041800000210080600000E01000322188FA
:10CDAC00A9518080408080808F5004003E4180805B
:10CDBC00508080008F50050037418080508080006B
:10CDCC008050010820010F402188A8540037518061
:10CDDC0080408080808F5004003E41808050808055
:10CDEC00008F504C00374180805080800080500173
:10CDFC000820010F404600371141800000210080BF
:10CE0C00600000E01000322388A9B18080A08080EF
:10CE1C00808F5004003EA18080B08080008F500530
:10CE2C000037A18080B08080008050010820010F65
:10CE3C00402388A8310037B18080A08080808F503B
:10CE4C0004003EA18080B08080008F50290037A163
:10CE5C008080B08080008050010820010F402300AA
:10CE6C00373141800040200080600000E01000322B
:10CE7C002748A9118180008180808F5004003E01D9
:10CE8C008180108180008F500500370181801081D6
:10CE9C0080008050010820010F402748A80E003761
:10CEAC00118180008180808F5004003E01818010B0
:10CEBC008180008F500600370181801081800080B6
:10CECC0050010820010F400000001E00780080FA7D
:10CEDC000000060200FA004F781E80FBE20F50069D
:10CEEC000032E30F50060032E10F5006003A801D6D
:10CEFC002305003780A52303003780ED230100377D
:10CF0C000000EB0080FA0000060200FA004F781EC9
:10CF1C0080FBE20F50060032E30F50060032E10FA7
:10CF2C005006003A809D2305003780E52303003727
:10CF3C00802D240100370000EB0080FA0000060869
:10CF4C0000FA2047982107983207982E40900080CD
:10CF5C00FBE20F503B0032E30F50700032E10F50F8
:10CF6C00A5003A0000EB000F782F0037408080AE10
:10CF7C0000909E8040114178819D23827078408082
:10CF8C00800000E8408088418080F00720808F502E
:10CF9C000100360830EF0141800000210080600064
:10CFAC0000E00F00322188A9418080508080808F62
:10CFBC005008003A5080800000E8508088518080F2
:10CFCC00F00720808F500100360A30EF2188A80C22
:10CFDC000037418080508080808F5008003A50800C
:10CFEC00800000E8508088518080F00720808F50AE
:10CFFC000100360A30EF1E0FE83E00909E0078804C
:10D00C008F50CDFF396E00370000EB000F782F00EA
:10D01C0037A08080AE00909E804011417881E5233E
:10D02C00827078A080800000E8A08088A18080F0C9
:10D03C000720808F500100361430EF114180000022
:10D04C00210080600000E00F00322388A9A18080BD
:10D05C00B08080808F5008003AB080800000E8B02B
:10D06C008088B18080F00720808F50010036163008
:10D07C00EF2388A80C0037A18080B08080808F506F
:10D08C0008003AB080800000E8B08088B18080F061
:10D09C000720808F500100361630EF1E0FE83E003F
:10D0AC00909E0078808F50CDFF393700370000EB11
:10D0BC00000F782F0037008180AE00909E804011C9
:10D0CC004178812D248270780081800000E80081F5
:10D0DC0088018180F00720808F500100362030EFCE
:10D0EC003141800040200080600000E00F003227BA
:10D0FC0048A9018180108180808F5008003A1081EE
:10D10C00800000E8108188118180F00720808F500A
:10D11C000100362230EF2748A80C0037018180101F
:10D12C008180808F5008003A1081800000E81081C7
:10D13C0088118180F00720808F500100362230EF5B
:10D14C001E0FE83E00909E0078808F50CDFF390076
:10D15C0000000080FA0000060200FA004F781E80E2
:10D16C00FBE20F50060032E30F50060032E10F5085
:10D17C0006003A0188A80400370388A80200370784
:10D18C0048A80000000080FA0000060400FA2047BE
:10D19C00982E40900080FBE20F50320032E30F508B
:10D1AC005E0032E10F508A003A014180008020007D
:10D1BC0080600000E01600322168A9118080008098
:10D1CC0080808F500E0032108080811D23614F783B
:10D1DC001080800000E8108088118080F07F208013
:10D1EC008F500100360230EF2168A81E4078730082
:10D1FC00372168A80040EB700037118080008080D8
:10D20C00808F500D0032108080811D23614F78106B
:10D21C0080800000E8108088118080F07F20808F53
:10D22C00500100360230EF1E40785F00370040EBB3
:10D23C005D00371141800080200080600000E01606
:10D24C0000322368A9718080608080808F500E002E
:10D25C003270808081A523614F787080800000E857
:10D26C00708088718080F03F20808F500100360ED6
:10D27C0030EF2368A81E40784500372368A800408B
:10D28C00EB420037718080608080808F500D0032BF
:10D29C0070808081A523614F787080800000E870D9
:10D2AC008088718080F03F20808F500100360E30D6
:10D2BC00EF1E40783100370040EB2F0037314180B2
:10D2CC000020200080600000E01600322728A9D141
:10D2DC008080C08080808F500E0032D0808081EDA5
:10D2EC0023614F78D080800000E8D08088D1808086
:10D2FC00F03F20808F500100361A30EF2728A81EEF
:10D30C0040781700372728A80040EB140037D1804D
:10D31C0080C08080808F500D0032D0808081ED23C2
:10D32C00614F78D080800000E8D08088D18080F078
:10D33C003F20808F500100361A30EF1E40780300DA
:10D34C00370040EB0100370040EB0080FA0000068C
:10D35C000200FA000F789E0078618E880080FA0037
:10D36C0000060600FA4047985147980000EB000F62
:10D37C00780000EB000F781000371E00783C030794
:10D38C001007981E00909040905E409080CF500700
:10D39C00003A1E0090A040904E409080CF5002006A
:10D3AC003A1E00900500371E0FE83A03079E0F50F7
:10D3BC00EDFF3E0000EB0080FA0000060800FA20AA
:10D3CC0047983147984247983307982B0007000F2E
:10D3DC00781E0078BE40901140981E0078AE4090A8
:10D3EC002140983E00908040781E00780148781EBD
:10D3FC0000786001903E00906300B9000078000056
:10D40C00E98000411E00787100981E00788040EB86
:10D41C004140981E00787000900000E8E902071E59
:10D42C00007801C8B32148980208200308201E0088
:10D43C00782200071E0078CE4090314098708E8084
:10D44C000000E8708E881E00780080FA000006024A
:10D45C0000FA020307C400DD80D524008F40DF02F0
:10D46C00079E0078E000981E00780080FA00000605
:10D47C000200FA000F781E00788040EB41409800C3
:10D48C0080FA0000060200FA000F781E007811C026
:10D49C00B34140980080FA0000060C00FA3007985F
:10D4AC004207985307980000EB000F783E00904E0F
:10D4BC000190DE01903200984300983E0090204885
:10D4CC00900080FB8000EB1007982107980000EB80
:10D4DC00000F785400373E00906001901E00786376
:10D4EC0000B90000780003413E0090004890008095
:10D4FC00FB8000EB1E01900191B9020178AE019006
:10D50C00009AB98401780301419E01900018B8017A
:10D51C000141820078C809DD4800DE008071C8082E
:10D52C00DE004078004B783E00906001901E007841
:10D53C006300B90000780000E80003413E009070E1
:10D54C0040900080FB8000EB1E01900191B902011C
:10D55C0078AE0190009AB98401780301419E019044
:10D56C000018B80101418200784809DD4800DE004E
:10D57C000071C808DE004078004B783E00906001D6
:10D58C00901E00786300B90000780080E800034129
:10D59C003E00906040900080FB8000EB1E019001EB
:10D5AC0091B9020178AE0190009AB9840178030117
:10D5BC00419E01900018B8010141820078C809DD34
:10D5CC004800DE008071C808DE004078004B781EF1
:10D5DC000FE83E00901040780080FB9E0F50A7FF94
:10D5EC003E0080FA0000060A00FA889FBE8A9FBEA1
:10D5FC002007983107984207980000EB000F782E0F
:10D60C0000901040780080FBCF80DE77D4070004B8
:10D61C00BE3E00908000EB76D4070005BE4E009015
:10D62C008000EB72D4070001BE0A00BE0BD40700C9
:10D63C0001BE0800BEC1D4074DD4071007982E00B8
:10D64C00901040780080FB6300B90000788000786F
:10D65C002E00906000900101788000EB93D60700BB
:10D66C0000EB000F785700372E00906001901E00E1
:10D67C00786300B90000780004412E0090004890B7
:10D68C000081FB8001EB2E00902048900080FB80F5
:10D69C0000EB009AB9040278028BB9860278050275
:10D6AC00420010B80102428400784809DD4800DECF
:10D6BC00000071C808DE004078004C782E009060A5
:10D6CC0001901E00786300B90000780000E80004A7
:10D6DC00412E00907040900081FB8001EB2E009059
:10D6EC002048900080FB8000EB009AB9040278027D
:10D6FC008BB98602780502420010B8010242840000
:10D70C00784809DD4800DE000071C808DE0040786A
:10D71C00004C782E00906001901E00786300B900D8
:10D72C0000780080E80004412E0090604090008159
:10D73C00FB8001EB2E00902048900080FB8000EBDA
:10D74C00009AB9040278028BB9860278050242006D
:10D75C0010B80102428400784809DD4800DE000060
:10D76C0071C808DE004078004C781E0FE81E00904F
:10D77C009E0078808F50A5FF394F05BE4F04BE0028
:10D78C0080FA0000060A00FA300798014F98000052
:10D79C00EB000F783E00908E48902148983E009008
:10D7AC002048900080FB8000EB1007982107980020
:10D7BC0000EB000F786500373E00906001901E0072
:10D7CC00786300B90000780003413E00906001903E
:10D7DC001E00786300B9000078000041104078000A
:10D7EC0080FB8000EB1E01900191B9020178AE0123
:10D7FC0090009AB98401780301419E01900018B8F9
:10D80C000101418200784809DD4800DE000071C842
:10D81C0008DE004078004B783E00906001901E00BE
:10D82C00786300B90000780000E80003413E0090E6
:10D83C006001901E00786300B90000780000E800D9
:10D84C0000411040780080FB8000EB1E019001919C
:10D85C00B9020178AE0190009AB9840178030141B4
:10D86C009E01900018B80101418200784809DD48FA
:10D87C0000DE000071C808DE004078004B783E00E6
:10D88C00906001901E00786300B90000780080E879
:10D89C000003413E00906001901E00786300B900C7
:10D8AC0000780080E80000411040780080FB800088
:10D8BC00EB1E01900191B9020178AE0190009AB96A
:10D8CC008401780301419E01900018B80101418246
:10D8DC0000784809DD4800DE000071C808DE004011
:10D8EC0078004B781E0FE83E00901040780080FBCB
:10D8FC009E0F5096FF3C0080FA0000060C00FA8840
:10D90C001F782007983107984207985307984E01C3
:10D91C0090DE0190028FBE2E00906001903E009030
:10D92C006300B90000780004412E40900081FB8018
:10D93C0001EB2E00902048900080FB8000EB009AB9
:10D94C00B9040278028BB98602780502420010B83D
:10D95C00010242840078C809DD4800DE008071C8ED
:10D96C0008DE004078004C782E00906001903E005C
:10D97C00906300B90000780000E80004411E40905C
:10D98C000081FB8001EB2E00902048900080FB80F2
:10D99C0000EB009AB9040278028BB9860278050272
:10D9AC00420010B80102428400784809DD4800DECC
:10D9BC00000071C808DE004078004C782E009060A2
:10D9CC0001903E00906300B90000780080E80004EC
:10D9DC00411E40780081FB8001EB2E009020489086
:10D9EC000080FB8000EB009AB9040278028BB986A8
:10D9FC0002780502420010B8010242840078C8097E
:10DA0C00DD4800DE008071C808DE004078004C78EC
:10DA1C004F04780080FA0000060400FA000F781119
:10DA2C0007981E00781040780080FB6300B9000056
:10DA3C00788000781E00786000900101789E00903C
:10DA4C0040D5070080FA0000060200FA000F78208B
:10DA5C0056806100600000E017003A1E007880409C
:10DA6C00EB4140981E0078720007C40AA80088A9F0
:10DA7C002088A81E0078600090405688802B20508B
:10DA8C0056880148A91E00781040780080FB63007E
:10DA9C00B9000078605688C50AA810C0B3010037D9
:10DAAC000040EB0080FA0000060200FA000F781E1E
:10DABC0000781040780080FB6300B900007880008B
:10DACC00781E00786000900101788000EB18D50773
:10DADC000080FA0000060600FA881F782007982EAE
:10DAEC0000909040902147982E009020449007D6AB
:10DAFC00073CD607804F5403003A03D607000F7833
:10DB0C001100372E0090204490F6D50733D60780AD
:10DB1C004F5403003AF2D507000F780800372E0057
:10DB2C0090204490F1D5072AD607804F542C003A08
:10DB3C00EDD507000F782E4090B5D50730479821CA
:10DB4C007C80F00B2000816060042071052043F87C
:10DB5C00208049788149788249783E40908080FBCA
:10DB6C001E01782003200088B90000786A0040620A
:10DB7C0000780001783E40908080FB9E0178200365
:10DB8C00200088B9000078700040630078000041E4
:10DB9C008040EB014878207C800001780260A06016
:10DBAC00042071052043F820804978814978824906
:10DBBC00780100370000004F04780080FA0000065E
:10DBCC000600FA881F782007982E0090904090212C
:10DBDC0047982E0090204490B9D507EED507804F7A
:10DBEC005403003AB5D507000F781100372E00907A
:10DBFC00204490A8D507E5D507804F5403003AA4DC
:10DC0C00D507000F780800372E0090204490A3D53C
:10DC1C0007DCD507804F543C003A9FD507000F789E
:10DC2C00508E800000E0020032508E808DFF07AED7
:10DC3C0040901E0078AD1107AE40901E0078C211C6
:10DC4C0007AE40901E00782B12072E409059D50736
:10DC5C00304798217C80F00B20008160600420719B
:10DC6C00052043F8208049788149788249783E40E4
:10DC7C00908080FB1E01782003200088B90000787A
:10DC8C006A00406200780001783E40908080FB9EE4
:10DC9C0001782003200088B90000787000406300F0
:10DCAC007800004181C2B3014878207C8000017863
:10DCBC000260A060042071052043F820804978811F
:10DCCC004978824978AE0090518E88010037000067
:10DCDC00004F04780080FA0000060200FA000F786A
:10DCEC008062259E0078808F5002003980E52400E8
:10DCFC000F789E00784190880080FA0000060000A2
:10DD0C00FA4090800080FA0000060200FA19000721
:10DD1C00000F780300071E00780080FA0000060050
:10DD2C0000FA708E800000E86F0060708E880080B2
:10DD3C00FA0000060200FA000F780A00079E0F5046
:10DD4C000500361E0078C400DD80D524008040011B
:10DD5C00003780D5240080FA0000060000FA708E8F
:10DD6C00800080FA0000060000FA002029C07D889F
:10DD7C00900120D07D88217C80F00B200081606098
:10DD8C00042071052043F820804978814978824924
:10DD9C007880C4B360EDB7207C800001780260A06D
:10DDAC0060042071052043F82080497881497882ED
:10DDBC004978400020100688000820000688500092
:10DDCC0021500688A0002240068840302320068877
:10DDDC000041EB8040EB10C0B3781307C1E0A8C43E
:10DDEC000AA911002076210AC40A00C42AA811002D
:10DDFC002032210AC40A00C52AA9BDEAA8BC0AA877
:10DE0C00F0FF26105688310020E8210AC60A0000CF
:10DE1C000021005688FAD40701C1B3DFDE07F7D41E
:10DE2C00072CD5075300200041EB01C1B384FC073C
:10DE3C00F1D407F2C0B301C1B3B4DE070080FA001D
:10DE4C0000060000FA0200070080FA000006040039
:10DE5C00FAADFF071007981E00900000E008003292
:10DE6C00818E801E00900001780500098280D88088
:10DE7C0000FD808E88010037D031EF0AD2BF0080C0
:10DE8C00FBE20F501A0032E30F501F0032E10F502B
:10DE9C0020003A818E80010F780B00371E007886A7
:10DEAC00FF07908E88908E80404090E14F50030089
:10DEBC003A20C0B30AF2B70500371E0FE81E0090D7
:10DECC009E0078808F50F1FF39808E800000E880B2
:10DEDC008E880A0037908E807AFE070004E00500D9
:10DEEC003230C0B30AF2B70300370000000100372C
:10DEFC000000000080FA0000060600FA881F782057
:10DF0C0007980000EB000F782E00901040780080EE
:10DF1C00FB6300B9000078100798404D80AFD30721
:10DF2C000000EB000F780700372E00906000901E69
:10DF3C000440AFD307004078004C781E0FE81E0059
:10DF4C00909E0078808F50F5FF394F04780080FA4E
:10DF5C000000060000FAD4D1BF0080FA00000600D1
:10DF6C0000FAB08E80E10F500D0032E10F50050029
:10DF7C0039E20F50120032E30F501800321F0037F5
:10DF8C00AF0D070004E0190032100020B08E881984
:10DF9C000037210E070004E01500321A0E07C08E60
:10DFAC0088200020B08E881E0E07100037100E0738
:10DFBC00000178C18E80608E80B9FC07300020B0E3
:10DFCC008E88080037608E803EFC07D631EF00004B
:10DFDC00000300370000000100370000000080FA49
:10DFEC000000060A00FA20479831479842479833B8
:10DFFC000798044F982E40908080FBC00820008822
:10E00C00B9800078002B26008040BE4090014878F3
:10E01C002E40908080FBC008200088B980007800DA
:10E02C002B260080408040EB1140980000EB000F45
:10E03C00781D00372E40908080FB3E00901E0040E3
:10E04C00104178C008200088B90000789E004080FC
:10E05C002B260080400248782E40900081FBC0089F
:10E06C00200090B90000788080E8002B26008040CA
:10E07C001040908041E8C008200090B980007820C2
:10E08C002B260080401340981E0FE80E489000800D
:10E09C00FB9E0F50DFFF3E2E40908080FBC008207F
:10E0AC000088B9800078402B26008040CE4090112B
:10E0BC0040982E40908080FBC008200088B98000DA
:10E0CC0078602B2600804021C0B31140980080FA64
:10E0DC000000060400FA004F781147982247983345
:10E0EC0047989E80FBC008200088B9800078002BE0
:10E0FC00260080409E40900148789E80FBC00820FE
:10E10C000088B9800078002B260080408040EB11FD
:10E11C0040989E80FBC008200088B9800078802B36
:10E12C0026008040AE40900148781E81FBC008203C
:10E13C000090B90000788080E8002B260080401009
:10E14C0040908041E8C008200090B9800078202BD6
:10E15C00260080401340989E80FBC008200088B9A0
:10E16C00800078402B26008040BE40901140989E45
:10E17C0080FBC008200088B9800078602B260080C6
:10E18C004021C0B31140980080FA0000060400FA48
:10E19C00004F781147982247983347989E80FBC0D0
:10E1AC0008200088B9800078002B260080409E4013
:10E1BC00900148789E80FBC008200088B9800078C8
:10E1CC00002B2600804011C0B31140989E80FBC0EC
:10E1DC0008200088B9800078202B26008040AE40B3
:10E1EC00900148789E80FBC008200088B980007898
:10E1FC00202B26008040BE40901140989E80FBC092
:10E20C0008200088B9800078402B26008040804090
:10E21C00EB0148789E80FBC008200088B98000780C
:10E22C00602B2600804021C0B31140980080FA007A
:10E23C0000060400FA004F7811479822479833479C
:10E24C00989E80FBC008200088B9800078002B269F
:10E25C000080409E40900148789E80FBC0082000C2
:10E26C0088B9800078002B2600804011C0B3114083
:10E27C00989E80FBC008200088B9800078202B264F
:10E28C00008040AE40900148789E80FBC008200082
:10E29C0088B9800078602B2600804011C0B30148FB
:10E2AC00789E80FBC008200088B9800078202B263F
:10E2BC00008040BE40901140989E80FBC00820001A
:10E2CC0088B9800078402B260080408040EB0148C4
:10E2DC00789E80FBC008200088B9800078602B26CF
:10E2EC0000804021C0B31140980080FA0000060263
:10E2FC0000FA004F789E80FBC008200088B980008F
:10E30C0078402B260080408040EB0148789E80FBB3
:10E31C00C008200088B9800078202B26008040801F
:10E32C0040EB1140980080FA0000060200FA004F02
:10E33C00781147989E81FB9E80FBC008200088B90D
:10E34C000000788080E8002B260080401040900070
:10E35C0081FBC008200098B9000078820040802B17
:10E36C00260080409E40900148781E81FBC008200A
:10E37C000090B90000788080E8002B2600804010C7
:10E38C0040908041E8C008200090B9800078202B94
:10E39C00260080401340980080FA0000060400FA22
:10E3AC002047982E40900080FBE20F50070032E38C
:10E3BC000F50080032E10F5009003A002020000FE6
:10E3CC0078060037C02120000F78030037C0F520F5
:10E3DC00000F780000001E0078310C200108981EF8
:10E3EC0000780120210108781E00788000EB41089C
:10E3FC00981E00788000EB2108981E0078012029D7
:10E40C000108781E007890007801F0A00108782EA1
:10E41C0040908080FBC008200088B9800078602B79
:10E42C002600804011C0B31140981000200080FAE3
:10E43C000000060400FA2047982E40900080FBE272
:10E44C000F50070032E30F50080032E10F50090063
:10E45C003A002020000F78060037C02120000F78EA
:10E46C00030037C0F520000F780000001E007890E4
:10E47C00007801F0A10108780080FA000006040081
:10E48C00FA2047982E40900080FBE20F5007003294
:10E49C00E30F50080032E10F5009003A0020200031
:10E4AC000F78060037C02120000F78030037C0F525
:10E4BC0020000F780000001E00789000780100A06A
:10E4CC000108780000001E007810007861006000E0
:10E4DC0000E0FBFF3A1E007820009033800A000019
:10E4EC00000080FB0080FA0000060400FA20479828
:10E4FC002E40900080FBE20F50070032E30F5008D3
:10E50C000032E10F5009003A002020000F7806007D
:10E51C0037C02120000F78030037C0F520000F789A
:10E52C000000001E00789000780110A0010878000F
:10E53C0000001E00781000786200600000E0FBFF15
:10E54C003A1E007820009033800A0000000080FB07
:10E55C000080FA0000060400FA2047982E40900034
:10E56C0080FBE20F50070032E30F50080032E10F3E
:10E57C005009003A002020000F78060037C02120F7
:10E58C00000F78030037C0F520000F780000001E44
:10E59C0000789000780120A00108780000001E008F
:10E5AC00781000786400600000E0FBFF3A1E0078F1
:10E5BC0020009044800A0000000080FB0080FA00DC
:10E5CC0000060400FA2047983147982E40900080AE
:10E5DC00FBE20F50070032E30F50080032E10F50FE
:10E5EC0009003A002020000F78060037C0212000D7
:10E5FC000F78030037C0F520000F780000003E4074
:10E60C00908080FB1E00782108980000001E007886
:10E61C002000906100600000E0FBFF3A1000200039
:10E62C0080FA0000060400FA2047982E40900080E3
:10E63C00FBE20F50070032E30F50080032E10F509D
:10E64C000A003A002020000F78060037C021200075
:10E65C000F78030037C0F520000F78000000010090
:10E66C00370000001E0078A000900000240080609D
:10E67C000000E0FAFF3A1000200080FA00000608C3
:10E68C0000FA2047983147984247983307982E4014
:10E69C0090DBFF072E40904CFF07BE40902E409021
:10E6AC00B5FF072E4090D4FF072E4090F4000700D2
:10E6BC000F78CE40902E4090ADFF072E4090CCFFAF
:10E6CC00072E4090EC0007000F782E4090C7FF07F4
:10E6DC002E409038FF073E40900004A08040782EDA
:10E6EC0040909FFF072E4090BEFF0712C0B3BE00A4
:10E6FC00902E40904101072E4090F300072E409041
:10E70C0071FF070080FA0000060800FA20479831D4
:10E71C0047984247985347983407982E4090ACFF3F
:10E72C00072E40901DFF07BE40902E409086FF079D
:10E73C002E4090A5FF072E4090C50007000F78CE05
:10E74C0040902E40907EFF072E40909DFF072E405C
:10E75C0090BD0007000F782E409098FF072E409038
:10E76C0009FF073E40900004A08040782E40907036
:10E77C00FF072E40908FFF075E4190BE00902E4009
:10E78C00901201072E4090C400072E409042FF07C4
:10E79C000080FA0000060600FA204798314798429C
:10E7AC0047985347982E40907EFF072E4090EFFEDF
:10E7BC0007BE40902E409058FF072E409077FF07E1
:10E7CC002E4090970007000F78CE40902E4090502E
:10E7DC00FF072E40906FFF072E40908F0007000F11
:10E7EC0078DE40902E409048FF072E409067FF0740
:10E7FC002E409020FF070080FA0000060A00FA4025
:10E80C004798514798320798034F980000EB100730
:10E81C00984E40905AFF074E4090CBFE075E4090BA
:10E82C000040408040784E409032FF074E4090515F
:10E83C00FF070040EB004F780D00374E40906E0004
:10E84C00071007981E80FBBE009000804010407897
:10E85C008040784E409023FF074E409042FF071EA9
:10E86C004FE80E48909E407880CF50EFFF394E40D5
:10E87C00908080FBC008200088B9000078E400403C
:10E88C00002B260080401040900004E002003A4E1D
:10E89C004090EBFE071E00900080FA00000602007C
:10E8AC00FA004F789E80FBC008200088B980007861
:10E8BC00602B2600804011C0B30148780080FA001C
:10E8CC0000060200FA004F789E80FBC008200088EA
:10E8DC00B9800078602B260080408040EB0148789E
:10E8EC000080FA0000060800FA004F7811479822C1
:10E8FC0047982307986447981E40780DFF071E40E1
:10E90C00787EFE079E80FBC008200088B900007846
:10E91C00E60040002B26008040104078E14F500E5E
:10E92C0000321E40900040408040781E4078DBFE54
:10E93C00071E4078FAFE07AE40901E4078D6FE07C0
:10E94C001E4078F5FE071E40788AFE071E40900098
:10E95C0080FB0000400040780004A08040781E40FE
:10E96C0078CAFE071E4078E9FE076E4190AE009013
:10E97C001E40786C00071E40781E00071E40789CD5
:10E98C00FE071000200080FA0000060400FA204761
:10E99C00982E40900080FBE20F50070032E30F509E
:10E9AC00080032E10F5009003A002020000F7806D1
:10E9BC000037C02120000F78030037C0F520000F6E
:10E9CC00780000001E00782000900080EA4F00DEE6
:10E9DC000080FA0000060400FA2047982E409000B0
:10E9EC0080FBE20F50070032E30F50080032E10FBA
:10E9FC005009003A002020000F78060037C0212073
:10EA0C00000F78030037C0F520000F780000001EBF
:10EA1C0000789000780150A00108781E00789000D2
:10EA2C00780140A00108780000001E0078100078E2
:10EA3C007000600000E0FBFF3A1E00789000780147
:10EA4C0050A10108781000200080FA000006040094
:10EA5C00FA2047982E40900080FBE20F50070032BE
:10EA6C00E30F50080032E10F5009003A002020005B
:10EA7C000F78060037C02120000F78030037C0F54F
:10EA8C0020000F780000001E00789000780150A143
:10EA9C000108781E00789000780140A001087800E9
:10EAAC0000001E00781000787000600000E0FBFF92
:10EABC003A1000200080FA0000060800FA2047985F
:10EACC002107986247982E40900080FBE20F500778
:10EADC000032E30F50080032E10F5030003A0020B2
:10EAEC0020000F78060037C02120000F7803003774
:10EAFC00C0F520000F780000002700372E40903220
:10EB0C0000078040782E00900148782E009000007D
:10EB1C00E82007981E0078A000900040200080603C
:10EB2C000000E00200320080EB2200376E409000C3
:10EB3C0004E00200322E4090B1FF072E409000817D
:10EB4C00FBC008200090B9000078E40040002B26A0
:10EB5C000080401040788041E8C008200090B980C7
:10EB6C000078402B260080400348780100370000D5
:10EB7C00006E40900080FB0000EA4F00DE00407801
:10EB8C00EE40908140E96147980004E0CFFF3A00E5
:10EB9C0000EB0080FA0000060400FA2047982E4093
:10EBAC00900080FBE20F50070032E30F5008003258
:10EBBC00E10F5009003A002020000F78060037C002
:10EBCC002120000F78030037C0F520000F780000DB
:10EBDC00001E00789000780130A001087800000039
:10EBEC000000001E00782000906200600000E0FB36
:10EBFC00FF321E00784008900080FA0000060200E8
:10EC0C00FA004F789E80FBC008200088B90000787D
:10EC1C00E60040002B260080401040900080FA0057
:10EC2C0000060200FA004F781E80FB0000E9E20F9C
:10EC3C005007003E9E80FBC008200088B9800078F9
:10EC4C00002B260080400100370000EB0080FA000A
:10EC5C0000060000FA8062250080FA000006000021
:10EC6C00FAB08D800080FA0000060000FAB631EF91
:10EC7C000080FA0000060200FA004F78B08D808107
:10EC8C0062251E4178827078B08D800000E8B08DCE
:10EC9C00880080FA0000060000FA80A2250080FAA5
:10ECAC000000060000FAC08D800080FA000006000B
:10ECBC0000FAB831EF0080FA0000060200FA004FAB
:10ECCC0078C08D8081A2251E4178827078C08D809D
:10ECDC000000E8C08D880080FA0000060200FA00EF
:10ECEC004F781E80FB1100200008DD6101B9908D6A
:10ECFC0080A18D80000071818071908D88A18D889C
:10ED0C000080FA0000060000FA201B210080FA00A7
:10ED1C0000060000FAB231EFB431EF0080FA0000C7
:10ED2C00060000FA5B07070080FA0000060000FAF4
:10ED3C005B07070080FA0000060400FA1007980031
:10ED4C0040EB004F781E80FB800040A01B21008010
:10ED5C00401000780000E00A003A1E80FB80004062
:10ED6C00A01B210080409E00900108781E0090801E
:10ED7C0000EB2100980E00371E80FB800040E01B4A
:10ED8C00210080401000789E00903100981E80FB7E
:10ED9C00800040E01B210080409000781E009021F4
:10EDAC0000981E80FB800040E01B210080409E00EC
:10EDBC00900108781E00908000EB3100981E80FBBB
:10EDCC00611C218100409140788140E8621C210245
:10EDDC0000400148780080FA0000060600FA10078F
:10EDEC00982107980040EB004F782E0090B00090CF
:10EDFC001E00903100981E0090AE00902100982EBD
:10EE0C0000903000900000E00500322E00903000A1
:10EE1C00909E00902100980600371E80FB800040D9
:10EE2C00E01B210080409E00900108782E00909EEF
:10EE3C0000903100981E80FB611C218100409140A4
:10EE4C00788140E8621C210200400148780080FA79
:10EE5C000000060400FA1007980040EB004F781EE3
:10EE6C0000902000900000E008003A1E80FB9E00FD
:10EE7C0090B10090000140A01B21000041010878D6
:10EE8C000500371E00902000909E0090B10090313C
:10EE9C0000981E00903000900000E008003A1E80A0
:10EEAC00FB9E0090A10090000140E01B210000415E
:10EEBC000108780500371E00903000909E0090A14C
:10EECC0000902100981E80FB611C21810040914024
:10EEDC00788140E9621C210200400148780080FAE8
:10EEEC000000060400FA1007980040EB004F781E53
:10EEFC0080FB800040C01B21008040100078000087
:10EF0C00E00A003A1E80FB800040C01B21008040BC
:10EF1C009E00900108781E00908000EB2100980E56
:10EF2C0000371E80FB800040001C21008040100038
:10EF3C00789E00903100981E80FB800040001C21C0
:10EF4C000080409000781E00902100981E80FB806D
:10EF5C000040001C210080409E00900108781E009B
:10EF6C00908000EB3100981E80FB711C21810040C9
:10EF7C009140788140E8721C2102004001487800E1
:10EF8C0080FA0000060600FA100798210798004046
:10EF9C00EB004F782E0090B000901E00903100983E
:10EFAC001E0090AE00902100982E00903000900032
:10EFBC0000E00500322E00903000909E0090210061
:10EFCC00980600371E80FB800040001C210080400A
:10EFDC009E00900108782E00909E00903100981EA3
:10EFEC0080FB711C218100409140788140E8721CAB
:10EFFC00210200400148780080FA0000060400FA63
:10F00C001007980040EB004F781E009020009000F5
:10F01C0000E008003A1E80FB9E0090B100900001B9
:10F02C0040C01B210000410108780500371E0090EC
:10F03C002000909E0090B100903100981E009030FE
:10F04C0000900000E008003A1E80FB9E0090A1009A
:10F05C0090000140001C2100004101087805003798
:10F06C001E00903000909E0090A100902100981EF0
:10F07C0080FB711C218100409140788140E9721C19
:10F08C00210200400148780080FA0000060400FAD2
:10F09C001007980040EB004F781E80FB800040204A
:10F0AC001C210080401000780000E00A003A1E800D
:10F0BC00FB800040201C210080409E0090010878BD
:10F0CC001E00908000EB2100980E00371E80FB8004
:10F0DC000040401C210080401000789E00903100C0
:10F0EC00981E80FB800040401C21008040900078DE
:10F0FC001E00902100981E80FB800040401C2100C7
:10F10C0080409E00900108781E00908000EB31003A
:10F11C00981E80FB811C218100409140788140E841
:10F12C00821C21020040014878C9D1BF0040E8C9C7
:10F13C00F1B70080FA0000060600FA1007982107C4
:10F14C00980040EB004F782E0090B000901E00907D
:10F15C003100981E0090AE00902100982E00903047
:10F16C0000900000E00500322E00903000909E00D0
:10F17C00902100980600371E80FB800040401C2127
:10F18C000080409E00900108782E00909E009031E7
:10F19C0000981E80FB811C218100409140788140A9
:10F1AC00E8821C21020040014878C9D1BF0040E828
:10F1BC00C9F1B70080FA0000060400FA10079800A5
:10F1CC0040EB004F781E80FB800040201C2100800B
:10F1DC00409000781E80FB000140401C2100004143
:10F1EC00100078808F5020003A1E80FB8000402059
:10F1FC001C210080409000781E0090808F501800D9
:10F20C003A1E80FB800040201C210080408000EBD7
:10F21C000108781E80FB800040401C21008040804B
:10F22C0000EB0108781E80FB811C2181004091407D
:10F23C00788140E9821C21020040014878C9D1BF85
:10F24C000040E9C9F1B72D00371E00902000900056
:10F25C0000E008003A1E80FB9E0090B10090000177
:10F26C0040201C210000410108780500371E009049
:10F27C002000909E0090B100903100981E009030BC
:10F28C0000900000E008003A1E80FB9E0090A10058
:10F29C0090000140401C2100004101087805003716
:10F2AC001E00903000909E0090A100902100981EAE
:10F2BC0080FB811C218100409140788140E9821CB7
:10F2CC0021020040014878C9D1BF0040E9C9F1B71B
:10F2DC000080FA0000060200FA000F781E0078E9A0
:10F2EC0005070080FA0000060400FA000F781107E9
:10F2FC00989E00901E00785306070080FA000006C6
:10F30C000200FA000F781E0078FD06070080FA0054
:10F31C0000060000FA0040EB0080FA000006120024
:10F32C00FA000F980E08901000901040780074A10D
:10F33C001047980E08901000780000E94300DE207A
:10F34C0047980E08901000780040780040E967401C
:10F35C00603047981E40900080FB2007980000EB1F
:10F36C003007982E00908000EB0001EB821F788014
:10F37C0003EB3E0190CE01905E0290EE02907E0374
:10F38C00906FEC078F87E90040EB004F7853003704
:10F39C000E08909000901E80FB4300DD0000E800FA
:10F3AC008040104078004F980E08909000901E807E
:10F3BC00FB4300DD0080E8008040104078104F983F
:10F3CC000E08909000901E80FB4300DD630040000F
:10F3DC008040104078204F980E08909000901E802E
:10F3EC00FB4300DD640040008040104078304F98B3
:10F3FC000E08909000901E80FB4300DD65004000DD
:10F40C008040104078404F980E08909000901E80DD
:10F41C00FB4300DD660040008040104078504F9860
:10F42C000E08909000901E80FB4300DD67004000AA
:10F43C008040104078604F980E08909000901E808D
:10F44C00FB0000E84300DD008040104078704F98CE
:10F45C001E40900080FB00A0A02007988000203068
:10F46C0007982E00908000EB0001EB821F78800340
:10F47C00EB3E0190CE01905E0290EE02907E0390E6
:10F48C001AEC078F87E91E4FE82E40909E4078803B
:10F49C00CF50A9FF390040EB004F780F00371E808A
:10F4AC00FB8E0890110190AE40908180FBC308DD6B
:10F4BC008101789E80FB8180418100E8810041912F
:10F4CC0040780000470148981E4FE83E40909E400F
:10F4DC007880CF50EDFF391E40900080FB00A0A03B
:10F4EC002007983E40900080FB3007982E009080BB
:10F4FC0000EB0001EB821F788003EB3E0190CE0104
:10F50C00905E0290EE02907E0390ECEB078F87E901
:10F51C001E40908080FB0070200100702007980036
:10F52C0000EB3007982E00908000EB0001EB821F5F
:10F53C00788003EB3E0190CE01905E0290EE02903B
:10F54C007E0390D9EB078F87E90080FA0000060252
:10F55C0000FA000F7800000000000000000000809E
:10F56C00FA0000060400FA0040EB004F7811003757
:10F57C001E80FB800040A01B210080409000781171
:10F58C0007981E00900000E00700321E00902FFF2D
:10F59C00071E009094FD071E009013FF0704003710
:10F5AC001E4FE81E40780004E0ECFF320080FA00A9
:10F5BC0000060400FA0040EB004F781100371E8063
:10F5CC00FB800040C01B2100804090007811079800
:10F5DC001E00900000E00700321E0090D0FF071EB6
:10F5EC00009008FE071E0090F9FE070400371E4F1E
:10F5FC00E81E40780004E0ECFF320080FA000006C0
:10F60C000000FA0003200018881000201018885001
:10F61C004C202018880623EF0823EF0001205018F7
:10F62C00880C23EF0E23EF1023EF1223EF1423EF9C
:10F63C001623EF1823EF1A23EF1C23EF1E23EF20C2
:10F64C0023EF2223EF2423EF2623EF2823EF20019F
:10F65C00205019880010206019883423EF8000EBAB
:10F66C0043210A340300006420701A88400620905D
:10F67C001A88000120901988200120001B88001096
:10F68C0020101B886A23EF8000EB43210A6A0300D9
:10F69C00006420201C88703821401C880001204008
:10F6AC001B882001201020880010202020880C248A
:10F6BC00EF8000EB43210A0C040000642030218809
:10F6CC00703821502188000120502088200120C052
:10F6DC002188001020D021884224EF8000EB4321A8
:10F6EC000A420400006420E022887038210023883C
:10F6FC000001200022882001207023880010208027
:10F70C0023887824EF8000EB43210A7804000064FE
:10F71C0020902488703821B02488000120B02388E0
:10F72C00200120202588001020302588AE24EF8071
:10F73C0000EB43210AAE0400006420402688703898
:10F74C00216026880001206025880080FA000006D0
:10F75C000C00FA2007986147984207985307984E77
:10F76C000090DE009002402B434C2028CA07400733
:10F77C00985107986E40904BCC072047984E0190BB
:10F78C00DE0190404C20010020800F51818F592EBA
:10F79C00003E2E40908080FB2E019020032000889C
:10F7AC00B90000787600406201782E40908080FB92
:10F7BC00AE01902003200088B900007876004063E9
:10F7CC00007890007870F82F0080600009782E4047
:10F7DC00908080FB2E01902003200088B9000078D7
:10F7EC007600406201782E40908080FBAE01902024
:10F7FC0003200088B9000078760040630078100080
:10F80C00788001B30009784E0190DE019000FF2F43
:10F81C00010020E0C907000F782D00372E409080A2
:10F82C0080FB2E01902003200088B9000078760020
:10F83C00406201782E40908080FBAE019020032026
:10F84C000088B900007876004063007890007870EA
:10F85C00F82F0080600009782E40908080FB2E01EC
:10F86C00902003200088B90000787600406201786F
:10F87C002E40908080FBAE01902003200088B900C0
:10F88C0000787600406300781000780030A0000902
:10F89C00784E0190DE019000402B414C20B2C907FC
:10F8AC00000F781E0178EE40902E009005020700A4
:10F8BC0080FA0000060600FA1007984147984E405F
:10F8CC0090DDCB07004F78217C80F00B200081600D
:10F8DC0060042071052043F82080497881497882A2
:10F8EC0049789E80FB1E01902003200088B90000FF
:10F8FC00787400406201789E80FB9E01902003206A
:10F90C000088B90000787400406300789001789EFC
:10F91C0080FB1E02902003200088B90000787E0036
:10F92C00406400780080EA0080610009789E80FBCA
:10F93C001E01902003200088B900007876004062F8
:10F94C0001789E80FB9E01902003200088B9000066
:10F95C007876004063007810007800F0A1000978F8
:10F96C00207C800001780260A06004207105204397
:10F97C00F8208049788149788249780080FA000023
:10F98C00060600FA1007984147984E409099CB070D
:10F99C00004F78217C80F00B200081606004207186
:10F9AC00052043F8208049788149788249789E80E7
:10F9BC00FB1E01902003200088B9000078740040E1
:10F9CC006201789E80FB9E01902003200088B90084
:10F9DC0000787400406300789001789E80FB1E02D2
:10F9EC00902003200088B90000787E0040640078E5
:10F9FC000300700009789E80FB1E019020032000FC
:10FA0C0088B90000787600406201789E80FB9E01E8
:10FA1C00902003200088B9000078760040630078BD
:10FA2C0010007800F0A0000978207C80000178029A
:10FA3C0060A060042071052043F82080497881493A
:10FA4C00788249780080FA0000060000FA3B6EA923
:10FA5C003B4EA93AAEA93A8EA9008EA9028EA8A84F
:10FA6C000007217C80F00B20008160600420710570
:10FA7C002043F82080497881497882497870238026
:10FA8C0000F0A1702388B02380C000B3B02388108D
:10FA9C00208000F0A1102088502080C000B350209E
:10FAAC0088207C800001780260A060042071052011
:10FABC0043F8208049788149788249780041EB806D
:10FACC0040EB10C0B31A00070041EB8040EB20C0A4
:10FADC00B3160007217C80F00B20008160600420AD
:10FAEC0071052043F8208049788149788249780350
:10FAFC00E4A86FE4A8207C800001780260A0600478
:10FB0C002071052043F82080497881497882497812
:10FB1C000080FA0000060600FA2047983147984208
:10FB2C004798CE409030C6B380CF5002003640C6C6
:10FB3C00B34047982E40900080FBE10F50030032F9
:10FB4C00E20F502D0032590037B024806101B84EBD
:10FB5C0040900080FB8000EB009AB9040278028B85
:10FB6C00B98602780502420010B80102428400787E
:10FB7C00420620030020BFC807000F783E409000CB
:10FB8C0080FBE10F50050032E20F500800320000FC
:10FB9C00E00B00320D00379A24EF9E0078912488F8
:10FBAC007264A80C00379E0078D124889224EF72DE
:10FBBC0064A80700379A24EF9224EF7264A800001F
:10FBCC00000000000000000000002D0037502180D4
:10FBDC006101B84E40900080FB8000EB009AB904A4
:10FBEC000278028BB98602780502420010B8010235
:10FBFC004284007842062003002093C807000F7847
:10FC0C003E40900080FBE10F50050032E20F50089F
:10FC1C0000320000E00B00320E00372E24EF9E0065
:10FC2C00783121880664A80D00379E0078712188F0
:10FC3C002624EF0664A80800372E24EF2624EF06AE
:10FC4C0064A8040037000000000000000000000061
:10FC5C00000000000080FA0000060000FA562EA9F1
:10FC6C00602EA95A2EA90080FA0000060000FA5650
:10FC7C002EA9602EA95A2EA80080FA0000060000BA
:10FC8C00FA20708044800A0000000080FA00000610
:10FC9C000000FAECFF07000000000000000000006C
:10FCAC000000000000000000000000000000E9FF60
:10FCBC00070080FA0000060A00FA881F78100798DF
:10FCCC004147983207984307984E409084CA0700E2
:10FCDC004F7818C0B302002003F8233E0090CE00EA
:10FCEC009068C7070000E001003C0044EB0804E00A
:10FCFC0005003200002001F8233007984107980DC9
:10FD0C00003718C0B36011B83E0090CE009057C7B2
:10FD1C00070000E00100350044EB0804E00300326A
:10FD2C006000B83007984107989E80FB1E01902018
:10FD3C0003200088B90000787A00406204789E8025
:10FD4C00FB1E01902003200088B900007878004049
:10FD5C006200781000788000EB60C7073E0190CEFF
:10FD6C000190B2C7073EC707000078000C789E8050
:10FD7C00FB1E01902003200088B90000787C004015
:10FD8C006201789E80FB9E01902003200088B900C0
:10FD9C0000787C00406300781000780030A00009E7
:10FDAC00784F04780080FA0000060E00FA300798AD
:10FDBC00014F985207986307980E489034CA072051
:10FDCC0047982E40908080FB3E01902003200088B5
:10FDDC00B90000780002B0620078800040E0922602
:10FDEC000080409000782107985E0090EE00900211
:10FDFC00402B434C20FAC7075007986107985E01C7
:10FE0C0090EE0190304C20010020800F51818F59D1
:10FE1C000F0036AE009011409020400A0002009076
:10FE2C0040982E009076400A1000005E0190EE0182
:10FE3C009000402B414C20D4C707000F782400378A
:10FE4C005E0190EE0190A00F20010020800F5181E7
:10FE5C008F590F0036AE009011409020400A0002DE
:10FE6C00009040982E009076400A1003005E01909E
:10FE7C00EE0190002D21310120BEC707000F780E36
:10FE8C000037AE009011409020400A0001009040D5
:10FE9C00982E009076400A1003005E0190EE0190BF
:10FEAC00801A26010020AFC707000F781E01788E3C
:10FEBC0048903E00900200070080FA0000060800FF
:10FECC00FA1007984147983207984E4090D9C907C5
:10FEDC00004F789E80FB1E01902003200088B90003
:10FEEC000078780040620078BE00900108780080AD
:10FEFC00FA0000060400FA0040EB004F783F003790
:10FF0C001E80FB800040E09226008040900078111B
:10FF1C0007981E00909000780140A10108781E00FF
:10FF2C009030400A1005001E00909000780150A1FE
:10FF3C000108781E009090007801B0A10108789E0D
:10FF4C00009011409020400A0000009040981E0044
:10FF5C009076400A1000001E00909000900170A155
:10FF6C001100989E009021409040400A000000A093
:10FF7C0040981E0090B000900180A03100981E00A7
:10FF8C0090D000900150A15100981E00908000EB81
:10FF9C000108981E009001C4292108981E00908029
:10FFAC0000EB4108981E00908000EB6108981E0041
:10FFBC009090007801F0A10108781E4FE81E40785F
:10FFCC00E44F50BEFF360080FA0000060000FA0D28
:10FFDC00D2BF0080FB4192266140780080FA00007D
:10FFEC00060000FA0DD2BF0040E80DF2B70DD2BFEB
:04FFFC00E44F50017D
:020000040001F9
:1000000000360D72EF0080FA0000060000FA0ED2F2
:10001000BF0040E80EF2B70ED2BFE44F50010036E9
:100020000E72EF0080FA0000060400FA000F78213B
:1000300047980080FA0000060A00FA300798014F3E
:10004000980CD2BFE44F502100360ED2BF0080FB87
:10005000800040809326008040100F780ED2BF00B1
:1000600080FBC1912661407854C9072047980ED281
:10007000BF0080FBC19126E140780ED2BF0080FB1B
:100080000001408093260000411000789D00072E5B
:1000900040908080FB1E01782003200088B900007A
:1000A000780000410003B031C0B30148780E489099
:1000B0003CC9073047983E40908080FB0DD2BF007E
:1000C00080FB4292266240780081FBBE01902003B3
:1000D000200088B90000780080410002B002087852
:1000E0000DD2BF0080FB800040809326008040BE80
:1000F00000900108780DD2BF0080FBC191260E4907
:1001000090827078A2FF070CD2BF0040E80CF2B7D3
:100110003E40908080FB3E01902003200088B90083
:1001200000780002B0620078800040E092260080F3
:10013000409000782107982E00908000EB410898AD
:100140003E40908080FB2E0090740140BE019020C4
:1001500003200088B9000078008041780040020840
:10016000783E40908080FB2E00907C0140BE019044
:100170002003200088B90000780080417A00400206
:100180000878217C80F00B200081606004207105DC
:100190002043F8208049788149788249783E409010
:1001A0008080FB3E01902003200088B90000786A1F
:1001B00000406200780001783E40908080FBBE01E4
:1001C000902003200088B900007870004063007818
:1001D0000001413E40908080FBBE01902003200042
:1001E00088B90000780002B06300789192266140DF
:1001F00078004978207C800001780260A0600420AB
:1002000071052043F8208049788149788249780037
:1002100080FA0000060800FA2007986147986E40AF
:1002200090C1C807004F789E80FB2E0190200320CC
:100230000088B90000780002B0620078800040E0D9
:1002400092260080409000781107981E0090800050
:10025000EB0108981E009090007801F0A00108784A
:100260000080FA0000060800FA2007986147986E9F
:100270004090A6C807004F789E80FB2E0190200377
:10028000200088B90000780002B062007880004049
:10029000E092260080409000781107981E00909010
:1002A000007801F0A1010878EE40902E0090EBE17B
:1002B000070ED2BF0081FB9E80FBAE019020032081
:1002C0000088B90000780002B06300788040784070
:1002D000922601707911FF070CD2BF0040E90CF2A1
:1002E000B70080FA0000060400FA0067261007989D
:1002F0008200208000EB006726B8C707120020802C
:1003000000EB801E21B4C7071200208000EB901E76
:1003100021B0C707EA71EFEB71EF0040EB004F78B7
:100320000600371E00908000071E009068004010F5
:1003300007981E4FE81E4078FF4F50F7FF360080A9
:10034000FA0000060000FA208F800080FA00000604
:100350000000FAEBD1BF0080FA0000060400FA109A
:1003600007980040EB004F781E80FB800040C01DC6
:10037000210080401000780000E00A003A1E80FB57
:10038000800040C01D210080409E00900108781E22
:1003900000908000EB2100980E00371E80FB80004B
:1003A00040E01D210080401000789E0090310098B0
:1003B0001E80FB800040E01D210080409000781EE0
:1003C00000902100981E80FB800040E01D210080ED
:1003D000409E00900108781E00908000EB3100984C
:1003E0001E80FB811E218100409140788140E8827F
:1003F0001E210200400148780080FA000006040037
:10040000FA1007980040EB004F781E80FB800040F8
:10041000001E210080401000780000E00A003A1E13
:1004200080FB800040001E210080409E009001085B
:10043000781E00908000EB2100980E00371E80FB94
:10044000800040201E210080401000789E009031E6
:1004500000981E80FB800040201E210080409000FC
:10046000781E00902100981E80FB800040201E21F5
:100470000080409E00900108781E00908000EB31C3
:1004800000981E80FB911E218100409140788140A0
:10049000E8921E21020040014878EAD1BF0040E8FE
:1004A000EAF1B70080FA0000060200FA000F788235
:1004B00000208000EB1E007823C707208F800000FB
:1004C000E006003A9E0078218F881E00788000EBBD
:1004D000210098060037308F809E007831009831D7
:1004E0008F801E00782100989E0078318F881E0032
:1004F000788000EB310098EBD1BF0040E8EBF1B71A
:100500000080FA0000060600FA10079821079800FC
:1005100040EB004F782E0090B000901E009031000C
:10052000981E0090AE00902100982E009030009010
:100530000000E00500322E00903000909E009021D7
:1005400000980600371E80FB800040E01D210080DF
:10055000409E00900108782E00909E0090310098F7
:100560001E80FB811E218100409140788140E882FD
:100570001E210200400148780080FA0000060600B3
:10058000FA1007982107980040EB004F782E009052
:10059000B000901E00903100981E0090AE00902197
:1005A00000982E00903000900000E00500322E00F0
:1005B000903000909E00902100980600371E80FB2E
:1005C000800040201E210080409E00900108782E6F
:1005D00000909E00903100981E80FB911E218100AA
:1005E000409140788140E8921E2102004001487805
:1005F000EAD1BF0040E8EAF1B70080FA0000060443
:1006000000FA000F781107982200208000EB1E00EE
:1006100078B0C6071E0090B000901E007831009898
:100620001E00789E00902100981E009030009000DF
:1006300000E00500321E00903000909E00782100FE
:10064000980200379E0078318F881E00909E0078B7
:10065000310098EBD1BF0040E8EBF1B70080FA0021
:1006600000060400FA1007980040EB004F781E00C7
:10067000902000900000E008003A1E80FB9E009051
:10068000B10090000140C01D210000410108780523
:1006900000371E00902000909E0090B10090310025
:1006A000981E00903000900000E008003A1E80FB89
:1006B0009E0090A10090000140E01D21000041013A
:1006C00008780500371E00903000909E0090A10031
:1006D000902100981E80FB811E218100409140786E
:1006E0008140E9821E210200400148780080FA0022
:1006F00000060400FA1007980040EB004F781E80B7
:10070000FB800040001E210080409000781E80FB8E
:10071000000140201E21000041100078808F5020F1
:10072000003A1E80FB800040001E210080409000A7
:10073000781E0090808F5018003A1E80FB80004089
:10074000001E210080408000EB0108781E80FB80A5
:100750000040201E210080408000EB0108781E80B0
:10076000FB911E218100409140788140E9921E2139
:10077000020040014878EAD1BF0040E9EAF1B72D14
:1007800000371E00902000900000E008003A1E8014
:10079000FB9E0090B10090000140001E210000412E
:1007A0000108780500371E00902000909E0090B14F
:1007B00000903100981E00903000900000E008008A
:1007C0003A1E80FB9E0090A10090000140201E2157
:1007D0000000410108780500371E00903000909E0F
:1007E0000090A100902100981E80FB911E218100A5
:1007F000409140788140E9921E21020040014878F2
:10080000EAD1BF0040E9EAF1B70080FA0000060231
:1008100000FA000F781E00782000900000E004002D
:100820003A1E0078300090208F880500371E00782F
:100830002000909E0078B100903100981E00783022
:1008400000900000E004003A1E0078200090308FF5
:10085000880500371E00783000909E0078A1009037
:10086000210098EBD1BF0040E9EBF1B70080FA001E
:1008700000060200FA000F78EBD1BF0004E006008A
:10088000321E0078D8FF071E007845FE0710C0B35F
:100890000100370040EB0080FA0000060000FA80FB
:1008A000D1BF0080FA0000060000FA00000000003E
:1008B00000000000100028E046882B68A999E9A9EB
:1008C0009889A951002030210A98090098A9A9996E
:1008D00069A9110020A8210A9809008000EB76215F
:1008E0000A9809009AE9A98000EB40210A9A0900B8
:1008F000A2A9A9A829EF800C20604D88AE29EFB0ED
:1009000029EF700C20A04D8899E9A80468A9BDEAD8
:10091000A8BC0AA8D80AA98000EB76210AD80A0048
:1009200011002054210AD80A00D82AA91100203227
:10093000210AD80A00D92AA8F0FF26105688810279
:1009400020E8210ADA0A00B0C020005688400620BC
:10095000005788007726F05688C0C020E056883EB1
:1009600000071B000710C0B34AF0B70080FA000070
:10097000060000FAE14680100028010070E0468879
:100980000080FA0000060000FAE14680E0FF270040
:100990008060E046880080FA0000060000FA10C07F
:1009A000B380F1B70080FA0000060000FA8071EF12
:1009B0000080FA0000060000FA0248A92248A8D8E0
:1009C0000AA84B70EF0080FA0000060000FA4BD036
:1009D000BF0080FA0000060000FAD80AA92248A940
:1009E00010C0B34BF0B70080FA0000060000FA0018
:1009F00006200080FA0000060000FA908C8000803B
:100A0000FA0000060000FA81D1BF0080FA0000065B
:100A10000000FA8171EF0080FA0000060000FA8CF5
:100A200031EF8E31EF9031EF10C0B34CF0B7008052
:100A3000FA0000060000FA6060800080FA000006FC
:100A40000000FA10C0B376F1B70080FA000006008B
:100A500000FA7671EF0080FA0000060000FA76D105
:100A6000BF0080FA0000060200FA000F789E0078AE
:100A70004182880080FA0000060000FA408280006F
:100A800080FA0000060000FA77D1BF0080FB0080EA
:100A9000FA0000060000FA7771EF0080FA00000605
:100AA0000000FA10C0B377F1B70080FA000006002A
:100AB00000FAF9FF0778D1BF0080FB0080FA000040
:100AC000060000FA10C0B378F1B70080FA00000603
:100AD0000000FAEEFF077871EF0080FA00000600D0
:100AE00000FA0300077000070080FA000006020009
:100AF000FA881F7879D1BF0080FBE20F501E0032C8
:100B0000E20F5005003C0000E0080032E10F500CFD
:100B100000325E0037E30F50460032E40F504800C9
:100B200032590037BCFF070004E04B003210C0B35D
:100B300079F1B753003799FF070004E04700329A74
:100B4000FF0791FF07000478BAFF07800F544300A6
:100B50003620C0B379F1B747003789FF0700047822
:100B6000B2FF07800F543D003630C0B379F1B7E0D3
:100B7000C507000F789E007800A720008040300253
:100B8000BE2003BE8000200100206011B80000627A
:100B9000818062020163838163E00F50E08F58E03F
:100BA0000F59E08F592A00329E007880A6200080DD
:100BB000403002BE2003BE8000200100206011B83A
:100BC0000000728180720201738381739E027884B7
:100BD000A620048242009ABE0292BE9E007870A6B1
:100BE0002000804011C0B30148781600379BFF07F2
:100BF00040C0B379F1B712003783FF070000E00E61
:100C0000003299FF0784FF077971EF0B003700006E
:100C1000000900370000000700370000000500371A
:100C20000000000300370000000100370000004F03
:100C300004780080FA0000060400FA889FBE0000D5
:100C4000EB000F780000EB10079882D1BF0080FB0B
:100C5000E30F508B0032E30F5007003CE10F503B95
:100C60000032E10F5068003C0000E00800329700BD
:100C700037E70F501C0032E80F50090032E40F50E4
:100C800086003290003716FF070004E08A003280A9
:100C9000C0B382F1B78A00377A31EF8831EF8A31F9
:100CA000EF4CD0BF0004E0080032808C80F30F507E
:100CB00003003E70C0B382F1B77E00374C70EF7C0A
:100CC000003710C0B382F1B77900370000EB000F96
:100CD000780D00371E0078800040007726008040A5
:100CE0001000786101B8408C80518C8002004083F4
:100CF0008048408C88518C881E0FE83006209E006A
:100D000078808F50EFFF36E4FE0720C0B382F1B742
:100D1000610037D08B808000400077260080401033
:100D20000178608C80718C80000078000051100781
:100D3000989E009090FC2F808F500600359E00906A
:100D4000700320808F5002003C0000EB1007984099
:100D50008C80518C8010C2070004BE1E0090CF8092
:100D6000DE09C2070001BE5FC2070001BE0800BE67
:100D700046C107E8C107408C88518C88D08B800021
:100D800000E8D08B88D18B80300620808F503600D1
:100D900036B6FE0720C0B382F1B77A31EF320037A2
:100DA000408C80518C80420620030020B1C2072075
:100DB0008C88318C884CD0BF0004E0100032608CED
:100DC00080718C800001BE208C80318C80020040BC
:100DD0008380488100D10080D3608C88718C8880AA
:100DE0008C800000E8808C888271EF18003730C05A
:100DF000B382F1B7150037208C80318C80D8C107C1
:100E000060C207B8C107000078908C8840C0B382E8
:100E1000F1B70B003700000000000000000010C018
:100E2000B381F1B78271EF000000030037000000CA
:100E30000100370000004F04BE0080FA00000600E9
:100E400000FAE094260080FA0000060000FAB5EFF0
:100E5000A911002050210A860F00910120B0210A1B
:100E6000880F0051002064210A8A0F001100202001
:100E7000210A8A0F00320020800720A1092053F8A0
:100E800020804978814978824978207C80000178E7
:100E90000200A060042071052043F8208049788179
:100EA0004978824978000000207C80610060000061
:100EB000E0FCFF3A000000217C80000220008060FE
:100EC0000000E0FBFF320080FA0000060200FA5743
:100ED000CEA857AEA9578EA91ECEA91EAEA91F8EA9
:100EE000A8298EA81F6EA8296EA85AAEA956AEA929
:100EF0001F4EA8294EA8562EA8602EA80F6EA82B0C
:100F00006EA8476EA8636EA80FEEA82BEEA847EE5A
:100F1000A863EEA80048A90068A90268A90968A901
:100F20002048A82068A82268A82968A8870107DEA9
:100F3000C40797C407000F789E007830A82000806F
:100F400040104078D9E6079E007890A820008040A5
:100F500010407812C0B38040EBFC02079E0078B0CE
:100F6000A8200080401040786AF10788C407000F6D
:100F7000789E007830A820008040104078C6E607B0
:100F80009E007890A82000804010407812C0B38066
:100F900040EBE902079E0078B0A820008040104096
:100FA0007857F10779C407000F789E007830A820A1
:100FB000008040104078B3E607A30707E4E5072662
:100FC000E1076DF70768FA07D9F8079EFD072F05B7
:100FD0000735EF070080FA0000061000FAB5EFA908
:100FE000201020A0028800F42B000F781E0078103B
:100FF00000BA8000EB1007982107981E0078108037
:10100000BA8000EB3007984107983E0090CE0090E0
:10101000C001DD0200201E0090AE00900000718132
:1010200080715007986107985E0190EE01908003EF
:101030002001002002027803017880017801007805
:101040000302620000618000EBC000DD00002000B0
:1010500001BE6120B8000171818171520798630758
:10106000985E0190EE0190000120010020800F5158
:10107000818F590F0032AC060701802B200020AF72
:101080000607604F986E48900004A20004E0050037
:101090003202802B210020E0A729CA0607604F9862
:1010A0000000FE0080FA0000060200FA19C40700E2
:1010B0000F789E0078D0A8200080401040780080F3
:1010C000FA0000060200FA14C407000F789E0078A8
:1010D000D0A8200080401040780080FA000006026E
:1010E00000FA0FC407000F789E0078D0A820008077
:1010F000401040780080FA0000060000FA12D2BFCB
:101100000080FA0000060200FA004F781E417821A4
:1011100021218248780080FA0000060000FA12724D
:10112000EF0080FA0000060600FA10079841479881
:101130004E4090BBC307004F780041EB9E40781EA5
:1011400000901CC3070080FA0000060600FA100792
:10115000984147984E4090AFC307004F780041EB4D
:101160009E40781E00903AC3070080FA00000606F1
:1011700000FA1007984147984E4090A3C307004FCC
:101180007812C0B39E40781E009004C3070080FA16
:101190000000060600FA1007984147984E409097C5
:1011A000C307004F7812C0B39E40781E009022C340
:1011B000070080FA0000060400FA000F7821479823
:1011C000AE40901E0078D6FF07AE40901E0078DF3C
:1011D000FF070080FA0000060600FA100798414752
:1011E000984E409080C307004F7862C0B39E40780D
:1011F0001E0090E1C2070080FA0000060600FA1007
:1012000007984147984E409074C307004F7862C0DA
:10121000B39E40781E0090FFC2070080FA000006CF
:101220000600FA1007984147984E409068C307009F
:101230004F7852C0B39E40781E0090C9C20700800C
:10124000FA0000060600FA1007984147984E4090B1
:101250005CC307004F7852C0B39E40781E0090E7F1
:10126000C2070080FA0000060600FA1007984147FE
:10127000984E409050C307004F7822C0B39E4078EC
:101280001E009027C3071047981E40900080FA0068
:1012900000060400FA000F78214798AE40901E0027
:1012A000788DFF07AE40901E0078A2FF070080FAFD
:1012B0000000060600FA1007984147984E40903704
:1012C000C307004F7832C0B39E40781E009098C28A
:1012D000070080FA0000060600FA100798414798B8
:1012E0004E40902BC307004F7832C0B39E40781E0B
:1012F0000090B6C2070080FA0000060600FA100748
:10130000984147984E40901FC307004F7832C0B3B2
:101310009E40781E0090D3C2070080FA00000606A7
:1013200000FA1007984147984E409013C307004FAA
:101330007842C0B39E40781E009074C2070080FAC5
:101340000000060600FA1007984147984E409007A3
:10135000C307004F7842C0B39E40781E009092C2EF
:10136000070080FA0000060000FA5AAEA80080FAD2
:101370000000060000FA5AAEA90080FA000006003C
:1013800000FAF10020B8210A020C0001EBA800ECE1
:10139000A80000000160800000280080600000E0DC
:1013A000FBFF320AEBA8000CA800000001608000DF
:1013B00010200080600000E0FBFF320A0BA80080D4
:1013C000FA0000060000FA8000EBFE210A0A0B007A
:1013D0008000EBD8210A0A0B0001022060210A04D8
:1013E0000B0031002090210AD80B008000EB602117
:1013F0000ADA0B0031002098210AD60B00A10F2039
:1014000090210A060B008000EBFD210A080B000268
:10141000EBA931002065210A020B00108BA911CB2A
:10142000A9128BA912CBA9130BA9134BA9138BA932
:1014300013CBA9140BA9144BA9148BA914CBA9BFC6
:10144000FF070080FA0000060000FAE28F80F38FA9
:1014500080F07022010020800F51818F5907003EDB
:10146000E08F80F18F80610040E08048E08F88F15C
:101470008F880900374158800004200080600000F8
:10148000E004003A08CBA81072EFFC31EFFE31EF18
:101490000080FA0000060800FA2007986147986E5D
:1014A000409096C2072047982E40908080FB2E01E6
:1014B000902003200088B900007864004062007822
:1014C0001001782E40908080FBAE01902003200018
:1014D00088B90000784002B0630078000061000025
:1014E000E04000322E40908080FB2E0190200320AF
:1014F0000088B90000786400406201782E40908036
:1015000080FBAE01902003200088B90000786400C1
:10151000406300789001782E40908080FB2E0290EE
:101520002003200088B90000784002B064007800F1
:1015300080EA0080610009782E40908080FB2E01B7
:10154000902003200088B90000788002B0620F78F4
:101550002E40908080FB2E01902003200088B9004F
:1015600000786400406201782E40908080FBAE01DC
:10157000902003200088B900007864004063007860
:101580009001782E40908080FB2E02902003200056
:1015900088B90000784002B0640078030070000948
:1015A000780800372E40908080FB2E019020032089
:1015B0000088B90000788002B0620F781E007800C1
:1015C00080FA0000060600FA100798414798524733
:1015D00098CE40901E00906FFE07CE40901E009067
:1015E00084FE074E40902AC207004F789E80FB1E63
:1015F00001902003200088B9000078660040620056
:10160000780001789E80FB9E01902003200088B91D
:101610000000782002B06300780001419E80FB9EAC
:1016200001902003200088B9000078A002B0634038
:10163000780049789E80FB1E01902003200088B925
:101640000000780080E86201789E80FB9E01902077
:1016500003200088B90000780080E86300789001DA
:10166000789E80FB1E02902003200088B90000783D
:101670004002B06400780080EA0080610009789E32
:1016800080FB1E01902003200088B90000786400D0
:10169000406201789E80FB9E01902003200088B963
:1016A0000000786400406300789001789E80FB1E03
:1016B00002902003200088B90000784002B0E400C6
:1016C000785E40900080FB0088B9000078030070CD
:1016D0000009789E80FB1E01902003200088B9003D
:1016E00000786800406201789E80FB9E0190200394
:1016F000200088B900007868004063007890017885
:101700009E80FB1E02902003200088B900007860B4
:1017100002B06400780300700009780080FA0000CD
:10172000060600FA1007984147984E4090BDC10741
:10173000004F789E80FB1E01902003200088B90096
:1017400000786600406200780001789E80FB9E0170
:10175000902003200088B90000782002B063007850
:101760000000418040EB0148789E80FB1E019020E4
:1017700003200088B90000786800406201789E80EC
:10178000FB9E01902003200088B90000786800408B
:101790006300789001789E80FB1E02902003200059
:1017A00088B90000786002B06400780080EA0080A8
:1017B000610009789E80FB1E01902003200088B9FB
:1017C0000000780080E86201789E80FB9E019020F6
:1017D00003200088B90000780080E8630078900159
:1017E000789E80FB1E02902003200088B9000078BC
:1017F0004002B06400780080EA0080610009789EB1
:1018000080FB1E01902003200088B900007864004E
:10181000406201789E80FB9E01902003200088B9E1
:101820000000786400406300789001789E80FB1E81
:1018300002902003200088B90000784002B06400C4
:10184000780080EA0080610009780080FA000006D4
:101850000600FA2047983147984247982E4090005A
:1018600080FBE20F50070032E30F50080032E10F17
:101870005009003AC02A20000F78060037802C203B
:10188000000F78030037402E20000F780000001E64
:10189000007890007801F0A10108781E0078C0005F
:1018A000900160A14100981E007871022001089803
:1018B0001E00789000780150A00108781E007890F2
:1018C000007801B0A10108781E007890007801A08E
:1018D000A10108781E00789000900140A0110098A6
:1018E0003E40906140606140606140609E007800D1
:1018F00080FB6100604800DD1101780280A10200D8
:10190000708008784E409061406061406061406046
:101910009E00780080FB6100604600DD11017802C6
:1019200060A10200708008782E4090E14F500B00BB
:101930003A1E0078A008900130A02108981E007877
:101940009000780120A00108781E00788000EB014B
:1019500008981E007890007801F0A00108780080B7
:10196000FA0000060400FA2047982E40900080FB01
:10197000E20F50070032E30F50080032E10F500928
:10198000003AC02A20000F78060037802C20000F74
:1019900078030037402E20000F780000001E0078EA
:1019A00090007801F0A10108780080FA0000060498
:1019B00000FA2047982E40900080FBE20F5007006D
:1019C00032E30F50080032E10F5009003AC02A20DC
:1019D000000F78060037802C20000F780300374076
:1019E0002E20000F780000001E007890007801F093
:1019F000A00108780080FA0000060600FA20479847
:101A00002107982E40900080FBE20F50070032E340
:101A10000F50080032E10F5009003AC02A20000F91
:101A200078060037802C20000F78030037402E20E6
:101A3000000F780000001E0078AE009001089800AA
:101A400080FA0000060200FA004F781E80FBE20FC9
:101A500050190032E30F502C0032E10F503F003A92
:101A6000000000A015806100600000E0FCFF32A0D3
:101A700015806100600000E0380032B4C2A9611531
:101A8000800040200080600000E0020032C015802D
:101A9000360037C11580F00F20008060320037001B
:101AA00000008016806100600000E0FCFF328016BC
:101AB000806100600000E0250032D0C2A94116809C
:101AC0000040200080600000E0020032A01680216B
:101AD0000037A11680F00F200080601D0037000045
:101AE000006017806100600000E0FCFF326017803A
:101AF0006100600000E0120032ECC2A921178000F2
:101B000040200080600000E00200328017800C005E
:101B100037811780F00F2000806008003700000038
:101B20000500370000000300370000000100370007
:101B300000000080EB0080FA0000060600FA204753
:101B4000982107982E40900080FBE20F501C003235
:101B5000E30F50350032E10F504B003AC1158001C0
:101B60000F78D11580010F7861158000402000802A
:101B7000600000E0040032AE0090C11588BA22EF88
:101B8000060037AE0090F00F20008060C01588BAC4
:101B900022EF000000A015806100600000E0FCFF63
:101BA00032330037A11680010F78B11680010F780B
:101BB00000000000000000000041168000402000EE
:101BC00080600000E0040032AE0090A11688D622AA
:101BD000EF060037AE0090F00F20008060A016885E
:101BE000D622EF0000008016806100600000E0FC5B
:101BF000FF32180037811780010F78911780010F8D
:101C0000782117800040200080600000E00400324E
:101C1000AE0090811788F222EF060037AE0090F0F8
